:020000040800F2
:1000000000A0002009320108197500083D220108EE
:10001000177500081575000813750008000000002A
:100020000000000000000000000000001175000842
:100030000F750008000000000D750008EBE50008D2
:100040007132010871320108713201087132010800
:1000500071320108713201087132010871320108F0
:1000600071320108713201087132010871320108E0
:1000700071320108754B0008D5C8000871320108BB
:1000800071320108713201087132010871320108C0
:10009000496D00087132010871320108713201089E
:1000A00055750008D9C6000843750008FDC600084C
:1000B000CDC60008BDC6000885750008713201086C
:1000C0007132010871320108713201087132010880
:1000D00071320108CDC80008C5C800087132010896
:1000E000F9E5000871320108396D00087132010824
:1000F00065750008713201087575000871320108D4
:100100000000000000000000000000007132010843
:10011000713201087132010871320108713201082F
:10012000713201087132010871320108713201081F
:100130007132010871320108000000000000000067
:1001400071320108713201087132010800000000AB
:10015000000000000000000000000000000000009F
:100160000000000000000000713201087132010837
:1001700071320108000000000000000000000000D3
:080180000000000071320108CB
:100188002DE9F04F2DED028B754D764B2B60AFB0FE
:1001980000236B6010F0EAF918B910F00BFA0BF0B5
:1001A80045F80BF001F9704B704C1A7842F00102D7
:1001B8001A706F4A4FF47001C2F888100022099231
:1001C8000A92226842F4803222600493236803F47E
:1001D80000330A93099B013309930A9B1BB9099BB6
:1001E800B3F5A04FF2D1236813F4003318BF0123ED
:1001F8000A930A9B012B00F089805D4F5D4BFB60E1
:10020800636AAB60636ADFF8A4B1DFF8A481DFF842
:10021800A49143F080736362636943F4FC032EAED8
:10022800636103238DF86A3041F6FF7326F8503D69
:100238004FF09040314604F08FFD4FF6FF734E4863
:10024800ADF86830314604F087FD4C48314604F07B
:1002580083FD4B48314604F07FFD5846314604F093
:100268007BFD3146474804F077FD304608F0B4FD81
:100278001A9B454AB3FBF2F3444A1360444B454A80
:100288004FF0000AC3F800A0434B5A60F02287F8E9
:1002980023200722C3F808A0404F1A60D8F8083076
:1002A8003B6099E80F0086E80F0063691A9843F4E9
:1002B80000136361636943F4001363614FF4885367
:1002C800ABF828304FF48843ABF828301BA904F06A
:1002D80043FD1DA91C9804F03FFD64200EF077F93A
:1002E8004FF4A0722E48514615F0DDF9E3692D4A06
:1002F80043F00703E361A36943F4E523A36163695A
:1003080043F4BC03636102F5907E55E0264B12224C
:100318001A606368636063686360636843F480635A
:100328006360636823F47C136360636843F4E813D1
:100338006360236843F08073236022680B4B92014B
:10034800FBD55A6822F003025A605A6842F002024A
:100358005A60636803F00C03082BFAD14DE700BF1D
:1003680088010020DBAA0008CC2D002000100240E4
:1003780000ED00E00005FA05000400480008004808
:10038800000C00480014004840420F0010260020CE
:10039800142600203F19010010E000E098290020F1
:1003A8005C260020849A01080020024000100048C2
:1003B80044130020387A0108937B506892F80FC0E4
:1003C80003F00701DB0800EB83038900186A4FF08C
:1003D8000F0A0CFA01FC0AFA01F120EA010119627C
:1003E800196A10324CEA010172451962E4D10022FF
:1003F800B849002353540132122AF9D1DFF814A363
:100408000AF11E02FF2199540133082BF6D1B24A92
:10041800B24B1360DFF800B3B14A039303211170A4
:1004280058460021242215F03EF914228BF80020AA
:10043800AC49039B3F6801228BF8182098F805B057
:1004480081F800B0A3F5F071CAF82810A649A3F501
:1004580090730B60A54B03EBCB035B78CAF82C3089
:10046800BB0648BFCAF82C200023A14A40F2DC5141
:1004780022F813100133082BF7D113A800211C22EE
:1004880015F011F9BBF10E0F03D00BF0EF03082B99
:1004980002D101238DF85C30022009F0D7FB18B196
:1004A8004088003018BF0120C7F340038DF8523050
:1004B800C7F380138DF85430C7F340338DF84C30B0
:1004C800C7F3C03300F001008DF84F3017F4006314
:1004D8008DF8510007D098F8863103F1FF3EDEF120
:1004E800000343EB0E038DF85030C7F300438DF83B
:1004F8005530EB6AB8F84801ADF86000003318BF12
:1005080001238DF85630C7F300538DF85730B8F8EB
:100518004A31ADF85A30B8F85631ADF8583007F0CE
:100528000101C7F38043C7F3C002FF0448BF714805
:100538008DF85330B8F8543144BFB0F85001ADF8D5
:100548006000B3F5FA7FADF85E3084BF0023ADF8E4
:100558006030694898F8D63185F83030002385F83E
:10056800313043709DF85C308DF84D10002B8DF8BC
:100578004E200CBF0023022301B902B1013309EB5D
:1005880083094FF0000AD9F810309A1E22330392DB
:100598000593039A32F8023F03924FF6FF72934293
:1005A80000F05E81DAB2190A9DF8553033B11301B3
:1005B8005248C058524B984200F04D819DF8523035
:1005C80053B14E4B4F4F03EB02135868B84203D157
:1005D8001B89012B00F03F819DF84F3053B1474BE9
:1005E800484F03EB02135868B84203D11B89042B08
:1005F80000F031819DF8503053B1404B414F03EB2F
:1006080002135868B84203D11B89022B00F02381DA
:10061800022902D19DF84C3003E0012904D19DF84C
:100628004D30002B00F01781344F9DF857304FEABA
:1006380002194F4433B19DF85C301BB9043A032AC0
:1006480040F2F2800129CBB268D1FF2385F87830D7
:1006580085F87930294BC5F8887003EB09024FF00B
:100668000008517B50688DF86A1002F1080B128956
:10067800ADF868201AA9022285F87C8006938DF8C7
:100688006B2085F83480C5F83880C5F83C80C5F8FB
:100698004080C5F8748085F87A8085F87B8004F0FE
:1006A8005BFB069B9BF8021053F80900424604F0D6
:1006B800A7F9384610F056FB134B1449C5F88C308F
:1006C800134BC5F89030C5F8948038460A1D0CF0D5
:1006D8009BF8C0E094010020581E00203815002027
:1006E80019130020900A002018280020489E0108AD
:1006F8008812002044130020B9010020849A0108C0
:1007080000440140000800489D47000814020020EA
:100718007D480008880100205C1E0020022B49D17A
:100728005FFA8AF21C2101FB02FC9D4ACDF81CC02D
:1007380002EB0C089B4A88F87DA0012188F87C1000
:1007480002EB09014FF0000B91F80DE0486888F8BA
:100758007EB001F108020989ADF8681088F886B002
:100768001AA9C8F888708DF86AE006928DF86B307F
:1007780004F0F2FA8B4B069A53F8090091785A461E
:1007880004F03EF9384610F0EDFA854BDDF81CC050
:10079800854AC8F88C2003EB0C01844AC8F89020DD
:1007A8008C31C8F894B038460A1D0CF02DF80AF1BF
:1007B800010A50E0032B35D19DF85330DFF8E08172
:1007C800DFF820923BB198F832B0384608214FF64E
:1007D800FF7200231AE0BDF85E2098F832B0BDF829
:1007E8006030B2F5FA7F0BD97149B1FBF2F23846A5
:1007F800082192B204F0D9FA6E4B49F82B000AE0AE
:100808006D49B1FBF2F23846012192B204F0CDFAFB
:100818006A4B49F82B00C36098F83230013388F8E6
:10082800323018E0042B16D195F83180BDF85820E5
:10083800614B93FBF2F23846BDF85A30012192B26F
:1008480004F0B3FA95F8313005EB88080133C8F89D
:100858005C0185F83130039B059A93427FF499AE89
:1008680095F8312085F87C21554A564B92F800E0DE
:10087800AEF117020027022A1F709C461AD8AB6AED
:100888003B44D3ED007AF5EE407AF1EE10FA02D14E
:10089800EB6A63BB26E04C4A07EB02080FCB88E8FB
:1008A8000F009CF8003010370133C02F8CF800304F
:1008B800E5D1EDE7454B13F83E908CF8009003EB3B
:1008C800CE03D3F804A0BAF1000FE1D04F45DFDA28
:1008D8003D4A3B0103EB020853440FCB013788E83C
:1008E8000F00F3E73A4D2B68D80424D41DE0394BA8
:1008F800394A13F83E00107003EBCE035D68002DF3
:10090800F0D000238342EDDAC3EBC3016A18DFF8A5
:10091800D880D2F8009041F8089001EB0807918838
:10092800B9809279BA710133ECE70EF0EF03082B26
:100938002A4B20D122E09CF80020012AF5D9284B27
:1009480003EB0212103210339342EED053ED047AC7
:10095800B6EE007A67EE877A43ED047A53ED057AAE
:1009680067EE877A43ED057A53ED037A67EE877A67
:1009780043ED037AE7E7BEF10E0F09D11A7842F08A
:1009880010021A70BEF1180F30D10EF093F82DE056
:100998001A7822F010021A70BEF1190FF4E700BF9E
:1009A80088010020849A0108054B00087547000853
:1009B80000127A009D48000840420F008D48000848
:1009C800900A002058260020CC090020489E0108E3
:1009D8009829002048850108A4270020301B002002
:1009E800D409002028260020A52700200EF046F86C
:1009F8002B68A848DFF8C8A2DFF8C8B259035EBF61
:100A0800A54B01221A70049B049A1B7843F0040337
:100A180013704FF40853ADF8683002238DF86B302B
:100A28006369012543F4001331468DF86A50636108
:100A380004F092F9994B9A4A1A6000200DF0E0FDF3
:100A4800A36943F48053A361E36843F48053E360EC
:100A580063694FF0904943F400336361D9F820305B
:100A680023F47003C9F82030D9F8203043F4A003E8
:100A7800C9F82030D9F8203023F07063C9F8203045
:100A8800D9F8203043F0A063C9F82030D9F82030D5
:100A980023F07043C9F82030D9F8203043F0A04340
:100AA800C9F82030D9F8203023F47023C9F8203051
:100AB800D9F8203043F4A023C9F82030E0234FF0C0
:100AC80000080327484631461A9302238DF86C30F4
:100AD8008DF86D708DF86E808DF86F8008F0F2FAE1
:100AE8001022484631461A9204928DF86D708DF89E
:100AF8006C508DF86E808DF86F8008F0E3FAE1682D
:100B080041F48051E160E16821F48051E160654978
:100B1800888820F480500004000C8880888880B27F
:100B280040F480508880088800F4415040F44570B3
:100B380038430880888820F470600004000C40F472
:100B4800E0608880888B20F400600004000C4FF07F
:100B580007098883A1F81090088880B240F0400007
:100B680008805149C1F800A0616941F480216161A0
:100B7800E16941F40011E161216B21F01001216369
:100B8800216B41F010012163DBF8201021F0706126
:100B9800CBF82010DBF8201041F08061CBF8201052
:100BA800DBF8201021F07041CBF82010DBF8201082
:100BB80041F08041CBF820104021022358461A9179
:100BC80031468DF86C308DF86D708DF86E808DF82B
:100BD8006F8008F077FA802158461A91314608F05C
:100BE80071FADAF80010314B049A21F00101CAF8C1
:100BF8000010DAF800002E490140CAF800102D490B
:100C0800CAF81010DAF800102943CAF80010CAF818
:100C18000880CAF80C80CAF80880DAF8081041F48D
:100C28000041CAF80810DAF80010CAF80010DAF81B
:100C3800041021F0784121F40041CAF80410DAF8D0
:100C480000102943CAF800101B4903930E68184680
:100C5800414614F028FD022306F4004B06F4006A0E
:100C68008DF83D301E40039B8DF83C708DF83E801A
:100C78008DF83F801F4627D010480E950EA908F022
:100C880021FA06223A7087F8018087F80390BD7030
:100C98001BE000BF00100048F80E0020DC2D0020EB
:100CA80075E100080030014054120020B01E0020F9
:100CB800FFE0CF007A25E0009829002000080048CE
:100CC80000540040000400483546BBF1000F0ED028
:100CD8000423BF480E930EA908F0F4F908233B71CA
:100CE8000723FB7101237D711D44BB71EDB2BAF17D
:100CF800000F0DD00223B6480E930EA908F0E2F9B2
:100D080007233B73FB7301237D731D44BB73EDB253
:100D18000EA90823AE480E9308F0D4F909233B72B4
:100D280007237D72FB720123BB721D44E36AA94845
:100D380023F4F873E362E36A43F4D873E362636904
:100D480043F0805343F00103636107F08EFF1AA854
:100D580007F060FFA04B1A93EDB2A04B1B93012D37
:100D68004FF000030CBF1A4680221F924FF4807286
:100D7800984C20924FF480622192202220462292A1
:100D88001AA94FF400521C931E9323922493ADF892
:100D9800745007F04CFF236843F0010323604FF0C1
:100DA800A0440A20A36823F04053A360A36843F03B
:100DB8008053A3600DF00BFCA36823F08043A3606D
:100DC800A368A360A36843F00043A3604FF0A04268
:100DD8009368002BFADB9368814923F040539360B2
:100DE800936843F00053936088687E4B034043F454
:100DF80068338B60D1687C4B0B4043F40053D3605D
:100E0800136B013D23F00F031D43156300240123D9
:100E18003A19917800296CD05D1C042B3E5DD0787E
:100E2800EDB24FF0A04E0ED803EB4302DEF83010BF
:100E380052001F23934021EA030106FA02F30B43F1
:100E4800CEF8303031E0092B0ED8053B06225A4344
:100E5800DEF834101F23934021EA030106FA02F357
:100E68000B43CEF8343020E00E2B4FF006010ED89D
:100E7800A3F10A024A43DEF838C01F2393402CEA44
:100E8800030106FA02F30B43CEF838300DE00F3BAE
:100E980001FB03F2DEF83CC01F2393402CEA030158
:100EA80006FA02F30B43CEF83C30092E4FF0A0426D
:100EB8000FD99369A6F10A0303EB43039669072147
:100EC800994026EA0101916191699840084390612F
:100ED8000EE05369731E03EB4303566938219940AA
:100EE80026EA010151615169033398400843506172
:100EF8002B460434102C8BD14FF0A042936843F05A
:100F0800010393604FF0A0431A68D207FAD5DA6854
:100F1800364C22F00202DA60DA6842F00202DA6045
:100F2800DA6842F00102DA609A6842F004029A60D4
:100F3800B4F85C31002B40F08287B4F95E21002AB6
:100F480040F07D87B4F96021002A40F07887284A6C
:100F580094F863311268DFF8B8B005930021B2F84D
:100F68005630244803930C22B4F8647194F86B61EA
:100F780094F86C51B4F80C9094F80FA0DFF89480B2
:100F880014F091FB00211422584614F08CFB1A4AE5
:100F9800049200211170C8F8801107F0FDFA049A34
:100FA800059B1146002800F02187144ACBF8002041
:100FB800134ACBF80420134ACBF80C20B7F5807FEE
:100FC800114ACBF81020114A26D100203BE000BF7F
:100FD800000800480800024040000050C01E0020E1
:100FE80000030050E010FCFF07C0FFFD4413002081
:100FF800981200206429002050080020ED7B00088A
:10100800F97A00085579000890C1793D0000002060
:10101800902D002088010020BB2F01D9012012E06B
:10102800612F01D902200EE0292F01D903200AE0FF
:10103800132F01D9042006E0092F01D9052002E069
:10104800002FC2D00620107001220A700222B34974
:101058000A70B3490A6842F001020A609B46B14A25
:101068000023BBF1090F1370F8D8012202FA0BF321
:1010780040F2B2311940002960D113F0450F09D16F
:101088001B075BD50023C8F8803107F085FA0028D4
:1010980054D00DE0192027211AAB03F073FF002864
:1010A800F0D0A14BA14A1A60A14A5A6006234BE02E
:1010B800062168200A460DEB000303F063FF9DF844
:1010C8006D1001F001029DF86B1001F001014B0059
:1010D80043EA82019DF8692002F001030B430AD01C
:1010E8005BB2012B01D1002302E0022B0ED10123B8
:1010F80088F8843111E00EAB68200C21012203F03E
:1011080041FF9DF8383013F00F0303D103200DF091
:10111800D3FA02E0042BEAD1E5E7834B854A1A604B
:10112800854A5A6098F88421002A0CBF6F226E22E3
:101138001A727C4B01221A70032305E0BBF1010FE0
:1011480009D94FF0000B8AE7744A5370744A136840
:1011580043F002031360042D00F2A380DFE805F0DA
:1011680003AA6B036B000A200DF031FA7720A02147
:1011780001220EAB03F006FF00285CD01E210122DD
:10118800772003F07BFF4FF42F600DF015FA4FF036
:10119800000BABF160010025C9B202221AAB77201F
:1011A8008DF868508DF8695003F0ECFE9DF86930B1
:1011B8009DF8682043EA0222604B03F5C3712BF8BF
:1011C80001200BF1020BBBF1100FE2D1B3F894210F
:1011D80002F47F4EA3F894E102F00F0101202B46A0
:1011E800DFF858C125F001026244B2F88621002ACE
:1011F80018BF002015F0010F03D0D2B253400822C7
:1012080002E083EA1223FAE713F4004F18BF83F4CD
:10121800C053013A4FEA4303F6D10135102DDFD10F
:10122800464D4EEA0102A5F8942120B9C3F30333D1
:10123800994200F0E985414D95F896B1BBF1000F50
:1012480040F0F48514200DF0C2F905F297137620CA
:10125800D021012203F096FE95F89731582B29D119
:1012680005F5CC7388211822762003F08BFE3122F5
:101278007620F42103F002FF012385F89631304BE4
:10128800304A9A60304A5A6045F6D8125A802F4A36
:10129800DA602F4A1A612F4AA3F800B05A6100F0A9
:1012A800C5BD012D06D01D4B1D4A9D70136843F026
:1012B800040313601A4D2B689B0702D51A4B1B6851
:1012C8009847DFF878B0244ABAF1000F46D017F0F3
:1012D800FF0F0AD12B6813F0020F4FF07D0140F287
:1012E800712308BF4FF4FA7302E04FF47A7319467A
:1012F800994505DBB9F57A6FA8BF4FF47A6900E024
:1013080099464B1E4B44B3FBF1F3013BDBB203FBA5
:10131800011188F8B431116024E000BF10010020E9
:101328002C1B0020F82D002064290020EF6B0008FA
:10133800996B00085D7C00083B7B00088801002051
:10134800F00600209177000893770008B579000827
:10135800677A000895750008DC2900208BF8B4A18D
:10136800C2F800902F4F3B6898472F4A002313700C
:1013780091461EB1B21E012A00F25B854FF00008AB
:101388000C20414601221AAB8DF8688003F0FAFD63
:10139800002800F07C859DF86830482B0FD1234B3E
:1013A800234A1A60234A5A60062389F80030224BE0
:1013B8000322DA702B6843F008032B6002E04046F2
:1013C80000F065BD94F858310BB11C4A137094F8BD
:1013D80059310BB11A4A137094F85A310BB189F884
:1013E80000302B68174913F0080F2FD0BDF90C00F7
:1013F800DFED156A642290FBF2F302FB130212B2CE
:1014080007EE902AB8EEE77A07EE903AF8EEE77A18
:10141800E7EE267AB2EE047A67EE877AC1ED007AB3
:1014280016E000BF902D0020F92D0020CC060020EA
:101438007D7B0008D37900081001002050080020A7
:10144800F82D0020242800208988883C00230B6080
:10145800BB4E337843F002033370BA4B4FF48842E3
:101468009A614FF488521A854FF00A09DFF8D4823E
:10147800B8F814309BB283F48843A8F81430B8F84D
:1014880014309BB283F48853A8F8143019200DF057
:101498009EF801200DF0B4F819200DF098F809F124
:1014A800FF3900200DF0ACF819F0FF09DED14FF438
:1014B8008853A8F828302B684FF488491807A8F8EB
:1014C800289009D5A04BC8F818901B6898479F4BDF
:1014D800A8F8289001221A709D4B9FED9E8A1B68E0
:1014E800DFF8B8821B7B00EE103AB8EEC00A20EE97
:1014F800080A09F0A5FDB8F8003007EE903AF8EEB2
:10150800E77A27EE800A14F0DDFA934B9FED937A81
:101518001880B8F8003007EE903AF8EEE77A904B6A
:10152800C7EE277AFF211B229FED8E7AC7EE877AB6
:101538009FED8D7AC3ED007AD7ED047A8B4F8C4BF3
:1015480067EE887A384667EE877AC3ED007A14F03A
:10155800AAF800223A702A68864B012112F0020F7D
:1015680019701FBF797003211970022118BFB97053
:10157800510741BF19784D1C1D70032548BF7D5484
:1015880012F00A0F38460CD01A780421B954511CAD
:10159800C9B205257D54D11C0232D2B21970062178
:1015A800B954754D29688F0641BF1A78571C1F70AA
:1015B800072748BF87540A0608D51A780927875489
:1015C800971C0132D2B21F700A2787546779082FF7
:1015D80001D00E2F08D11A7802F1010E83F800E02D
:1015E8004FF00B0E00F802E01A7811F4803F4FF02C
:1015F8000C0C00F802C002F1010E1CBFDFF874C128
:1016080002325FFA8EFE83F800E01FBF8CF80020DC
:10161800564A4FF00E0C02F80EC04A0741BF1A781E
:1016280002F1010E83F800E04FF0100E48BF00F8F9
:1016380002E01A7802F1010E5FFA8EFE4FF0120CEA
:1016480011F4806F83F800E000F802C00ED094F81F
:1016580010C2BCF1000F09D0DFF818C102328CF8B3
:101668000020424A4FF0130C02F80EC01A7811F409
:10167800007F4FF0140C00F802C002F1010E1CBFED
:10168800DFF8F0C002325FFA8EFE83F800E01FBF79
:101698008CF80020354A4FF0150C02F80EC0182FB0
:1016A80013D11A784FF0160E00F802E002F1010E7D
:1016B8005FFA8EFE4FF0170C00F80EC002F1030E11
:1016C8000232D2B283F800E087540A0341BF1A7885
:1016D800571C1F70192748BF8754CF0541BF1A7878
:1016E800511C19701A2348BF83540021982223489B
:1016F80013F0D9FF06F0FBFF214B224A1A60224B58
:10170800B4F852111980214900230B808B702049AD
:101718000A60B4F8982190B21E4921F813000133E9
:10172800122BF9D12B68D8045EBF1B48B0F89E0174
:1017380008801B0740F1F980174B93F892312FE08E
:10174800CC2D002000100048CC060020E406002024
:10175800DC08002035FA8E3CF80800200AE81C4115
:101768001408002000401C46BD3786356112002051
:10177800D80800206012002098290020B41D0020FD
:101788002C100020CE14002030100020602D0020E6
:10179800542D0020802C0020441300201600002027
:1017A800062B00F2BC80DFE803F004070E3D5877F3
:1017B800770045F2F05201E042F6F822814B1A8098
:1017C80007F04BF8AAE007EE902ADFED7F6A7D4B21
:1017D800B8EEE77ADFED7D7AE7EE267A42F6F82171
:1017E80019800023FCEEE77A794A17EE901A42F83E
:1017F80023100133122BF7D1764A77491160774AC3
:101808004020137008F00AFB002800F088800123AC
:101818004FF0070890F90000714A8DE8080140214F
:10182800704B76E0674B42F6F8221A80694B6E4A95
:101838001A606A4B102240201A7008F0EFFA00284C
:101848006DD001234FF0000C90F90000674A8DE835
:10185800081040214FF4E1335BE05A4B42F6F8227E
:101868001A805C4B624A1A605C4B082240201A704E
:1018780008F0D4FA002852D001234FF0000E90F956
:1018880000005C4A8DE8084040214FF4E13308F03D
:10189800A1F8CBF8B8013EE04A4ADFF89081DFF8BA
:1018A80090C1DFF890E1544F544C554842F6F82166
:1018B80011804A490C22062B0A700ED0002388F8A2
:1018C80000308CF800308EF800301B233B70052365
:1018D800227003704FF4E1340BE0002188F8001007
:1018E8008CF800108EF8001022702121454C3970B8
:1018F8000370384B444A1A60402008F08FFA70B1E0
:1019080001230027414A90F9000040218DE8880012
:10191800234608F05FF8003018BF012028B90820D6
:1019280009F052FC2B4B3A4A1A602B682B4A13F4E5
:10193800804F1FBF082111702649364818BF08601C
:1019480042F20101194003F0010003F4005479B197
:101958001C4944F620670F8024B1082111701D49E5
:101968002D4C0C6020B10C2111701A492B480860CD
:10197800117804395170190640F195800027284CD8
:10198800DFF8B4902748DFF8B480CBF8BC9139462B
:10199800152267706760A76013F085FEA9F105033B
:1019A8003846C8F8003006F069FC1F4B02201B6857
:1019B800E36008F033FA002842D1802009F004FCE3
:1019C80069E000BF38090020CDCCCC3F0000B0C48E
:1019D800382C00201C000020AD160108501E0020E5
:1019E8002D190108A086010099160108811801081F
:1019F8008116010835180108C62C0020C52B0020C7
:101A0800C72C002090D00300A9150108151701085C
:101A180011170108E116010801170108F11601085C
:101A28002808002048030020BC290020C62B0020DD
:101A3800C52C0020C42C00203815002048080020A0
:101A480047796378C4490C2202FB03125278BA42E0
:101A580004D00133DBB2042BF4D900236370D8F827
:101A6800003062781B7890F90000002B4FF00C03CF
:101A780003FB021314BF0327012700225B7800979A
:101A88000192022107F0A6FFB44B1860002894D0F9
:101A9800012006F0F3FBB24B1868B24B00F5C57293
:101AA8001A6006F099FCB04AB04B1360B04AB14FC7
:101AB800803313602B680024DA033C7040F1AD805A
:101AC8000DF028F9DFF818C3DFF81893CDF810C027
:101AD80040F22A3B4FF00108604621465A4687F8F3
:101AE800008013F0E0FDD9F81430A348A34F43F465
:101AF8008023C9F81430436A23F00F034362436A12
:101B080043EA08034362022203234FF4807A0CA9B4
:101B18008DF8342003928DF835308DF83640CDF8A5
:101B280030A08DF8378007F0CDFAD9F81830039A2D
:101B380043F40033C9F818303B8823F440731B047E
:101B48001B0C3B801D23FB620EA93A8560233C8653
:101B58003846C7F814800E93ADF83E401094ADF89F
:101B68004440ADF84640ADF84840ADF84A40ADF8BD
:101B78003C8007F0F3F8BB6943F00803BB617B6C5A
:101B880043F400437B64D9F8143043EA0803C9F8E6
:101B98001430A9F57D69484607F067F81AA807F0D8
:101BA80039F8774B1A9310231C938023DDF810C063
:101BB8001F931AA94FF400534846CDF86CC02393DD
:101BC800ADF874B01E94CDF880A02194229424948A
:101BD80007F02DF8FB6843F40073FB60D9F8003078
:101BE80043F00203C9F800300BA80D238DF82C3000
:101BF8008DF82D808DF82E408DF82F800FF094F8F9
:101C08002146604B1A68604B43F821200131202996
:101C1800F7D102F0C3FF02F0C1FF2B685B0556D570
:101C28005A4F5B4BD7F80085C3F80080042008F0B2
:101C3800F5F80421C7F8040508F0CAF8554B87F8E9
:101C480008050820C3F8008008F0E8F8524B534C08
:101C58001860082108F0BCF8002187F809052C2233
:101C6800204613F020FD8E2363704FF07C0AE0239A
:101C78004FF07D09E37084F800A084F82B90484C5D
:101C88002C220021204613F00EFD8A2363701020B9
:101C9800A023E37084F800A084F82B90C7F80C8583
:101CA80008F0BCF81021C7F8100508F091F887F87B
:101CB80014052020C7F8188508F0B0F82021C7F8C7
:101CC8001C0508F085F887F820050FF071FF2B68D0
:101CD800344A13F4002318BF012313700CF050FC8E
:101CE800314B1860314B5A79052A194602BF304BDF
:101CF8004FF4C8721A802F4B4FF47A721A802E4B09
:101D0800C8221A802D4A137843F0080313702C4A0E
:101D1800137823F0020313702A6840F60203134075
:101D28006BB1284B284A1A60284B03221A70284B9B
:101D380001221A70274A00231380274A13808B68D0
:101D48002B60264B01221A70337863F07F033370BF
:101D58002FB0BDEC028B47E0C87A0108EC1F0020C9
:101D680098120020881000202820002064150020E8
:101D780024200020F90E00200004004800440140FF
:101D880034440140587A0108FA0E002088010020E6
:101D9800201B0020781B0020C41B0020481B0020AB
:101DA8007D1B0020D829002018090020441300209A
:101DB8003E100020F22D0020F02D0020301B0020C6
:101DC800FB2D0020181B0020C01400207C1B0020C5
:101DD80008010020281100202A110020F80E0020F8
:101DE8005D03002000100240BDE8F08F2C49CBF8BD
:101DF80000102C49CBF804102B49CBF81010042103
:101E080011700522FFF723B9284B42F210721A808D
:101E18005A80274A5A60274A9A60274ADA60274A2E
:101E28001A61274A5A610325FFF73DBA0425FFF7CF
:101E38003ABA012E7FF6C6AA1E46FFF796BA1BB21B
:101E480007EE903ADFED1F6AB4F95E311E4AF8EEEC
:101E5800E77A07EE103A67EEA67AB4F96031CDED6D
:101E68001A7A07EE903AB8EEC77AF8EEE77A0021C8
:101E780027EE267A67EEA67A11701AA813498DED17
:101E88001B7ACDED1C7A09F0E3F8FFF760B8012E54
:101E98007FF698AA002689F80000FFF76FBA00BFFE
:101EA8008D6C0008316C0008295C8F3DF00600201D
:101EB800C9790008E97A0008BF790008D97A0008CA
:101EC8009577000835FA8E3C800000208C1E002093
:101ED800954A2DE9F04F1568944C05F59C4320333D
:101EE8002DED028B2360924B196889B011F4804F55
:101EF8000592984605D10FF0A9FD10B92379013351
:101F080023718C4B1F78C7B18B4A1268954240F2F7
:101F1800DF80013F1F70DBE0D9F800308748072DCC
:101F280098BF595D864B88BF29461B689847032D83
:101F38000BD904EB45050137E880804BDFF81C928C
:101F48001E78FDB2AE42E7D820E0D9F8002005F1AE
:101F58000E0302EB83039988DA880028E9D04FF44E
:101F68007A73401A5843531A90FBF3F040F6C903AA
:101F780000F57A70984205DC40F2EE239842B8BF2B
:101F8800184601E040F6CA0080B2D2E70F2327794D
:101F980084F82A3094F82B300193032594F82C30D8
:101FA800B7FBF5F505EB45057D1B0393D9F8003024
:101FB8000293DFF8B0A1EBB204930025B54254DADE
:101FC8006049019B31F815B04FEA450953B90FF044
:101FD8003DFD28B1039B002B08BF4FF0000B01E02B
:101FE800DDF804B0029B988A584502D8D88A58452B
:101FF8000ED2E8B20FF0D4FC032D8346DFBF94F86D
:102008002AE00120A8402EEA0000D8BF84F82A0060
:102018000FF01CFD18B14C4829F800B021E0049BD2
:1020280094F876002AF813B028B9022F15D93F4939
:10203800012081F87600BAF80210BAF800000844C6
:10204800BAF804100844414980B229F8010000B2E6
:10205800032190FBF1F080B200E058463A4929F894
:10206800010001350AF1060AA8E794F82A20384841
:10207800384BA2F10F014A424A4184F890206AB1D4
:10208800354A1268520109D40268D9689A60521A0E
:10209800C82A1DD9012283F8212019E0026898680E
:1020A800DA605B68121A9A4288BF2A4B4FF0000127
:1020B80084F82B1088BF83F821100025B54207DA71
:1020C800E8B20FF06DFC204B23F815000135F5E759
:1020D800D8F80030DF0405D51F4B1B68DE0701D494
:1020E8000FF02AFA059B19681C4B1868837A002B95
:1020F8003AD0013B144D027B35F813301AB1C3F5C1
:102108003B6308339BB21BB2A3F57A73B3F57A7FAE
:10211800A8BF4FF47A7323EAE37307EE903A9FED72
:10212800107AF8EEE77A58E0D82D0020800F0020CA
:10213800982900205C2D0020582D0020501E0020DA
:102148001C000020860F0020802C0020F80F0020A3
:10215800BC290020602D00205C120020542D002096
:1021680000007A44AE0F0020D8F80020150440D5AE
:10217800D4F89420934E8A1A002A3ADB01F59C423F
:102188002032C6F89420904AC07A55798F4A32F89E
:10219800152096F89850013592B292FBF0F205F0AE
:1021A8000F0086F89800304480F899201A4688482D
:1021B800185C01330244102B92B2F8D112B292FB90
:1021C800F3F31BB2642BA8BF642323EAE37307EE7F
:1021D800903A9FED807AF8EEE77AC7EE877A7E4AE2
:1021E8009FED7E7A67EE877AFCEEE77A17EE903AF3
:1021F8001380D8F800307A4F13F4807F00F00981FB
:10220800784BDFF8E491994205D999F8022012B980
:10221800012289F8022099F80220002A00F0F980AA
:10222800714A3E7892F821506A1E554255416F4ACC
:102238001168002DC1F38063C6F3800601939246AE
:1022480014BF4FF0000B4FF0030B99F82020052A1C
:1022580000F2D980DFE802F0034D527584A1002E08
:102268003AD0D4F8AC00B4F8B0100CF044F9012816
:1022780009D15F495F4A09681268C988642000FB70
:102288000122C9F81020019B6BB1594A12681279D2
:102298004AB10FF0B1FF032289F820204FF47A7277
:1022A800C9F81C20D1E7002D40F0AD80514AD9F87B
:1022B800101010684C4A88420AD902920FF09CFF0D
:1022C800029A032182F8201040F6B831D161BCE7A8
:1022D800012182F82010B8E7019B4FF4806013B108
:1022E80008F062FF01E008F04EFF0022C9F8102054
:1022F80089E0002D46D10FF07FFFA6E725B1052222
:1023080089F82020012000E0284666B1D4F8AC20E6
:10231800D189394A118051809180354909684988A5
:10232800D1804FF0020B334A1168D9F8142091423A
:1023380001D8002E64D147F23052C9F81C2003227C
:1023480021E03A7842F002023A700FF0F5F8294A93
:10235800D9F81C1012680A44C9F81820042212E09F
:10236800244A9DB11168D9F8182091424BD9234AC3
:1023780012781AB9DAF80020D30744D43A7822F050
:1023880002023A70052289F820205EE71268D9F81F
:102398001C100A44C9F8182035E01549154A09687F
:1023A8001268C988642000FB0122C9F810204FF484
:1023B8008060002289F8202089F8032008F0E3FED5
:1023C80043E700BF800F0020B01E0020C01E002081
:1023D800191000200000C842B812002000C07F4435
:1023E800FB2D0020404B4C00602D00205C1200208B
:1023F800C82D0020BC290020802C002014000020BB
:1024080000287FF422AFBBF1000F02D058460CF031
:1024180015F9934D05F5C570B5F852110CF06BF828
:10242800834668B90FF0DAFE8E4BC3F800B0C3F8E4
:1024380004B0C3F808B08C4B00221A605A609A6046
:102448003B785E0736D5D8F80030D80632D5874BAA
:102458001B78D9062ED4864B1B7893B195F8E231B8
:10246800BBF1000F15D17BB1824B1A68D4F8B43098
:102478009B1A002B08DA0FF05FF87F4B83F8B8B08F
:1024880018E0BBF1000F0DD110200CF0D7F8012394
:102498000EE03BB1774A12684FF47A7101FB0323CF
:1024A800C4F8B43094F8B83023B10CF0AFF8002376
:1024B80084F8B830002295F8E0A195F8E111B5F854
:1024C8009AE1B5F89CC113466C4E019636F9120094
:1024D8009B087045C4BF63F07F03DBB201326045DF
:1024E800B8BF43F04003042AEED194F8B9206248FB
:1024F8009A4205D190F8BA20F92A04D8013200E0AE
:10250800002280F8BA2084F8B930594B5C4E1A780A
:102518009946E2B93368DA0708D5BBF1000F16D13E
:102528003B78DB0713D50EF073FE10E03B785807B5
:102538000DD5514B93F82B304BB1524BDB7833B957
:1025480011B10EF0F9FF02E0BBF1000FF9D094F8D9
:10255800BA30494ADFF840B1142B40F0AF8099F8FF
:1025680000301AF1000A18BF4FF0010A6BB392F855
:10257800B9305F2B11D13B7803F0040303F0FF015E
:1025880013B10EF0D9FF08E00B20039102920CF072
:1025980055F8029A039982F8BA10BAF1000F14D0CC
:1025A80094F8B9307D2B10D13B7803F0040303F085
:1025B800FF0213B10EF0C0FF07E00B2002920CF0EF
:1025C8003DF82D4B029A83F8BA203B7803F00403B8
:1025D80003F0FF01002B71D194F8B930264A572B2C
:1025E80016D1294B4FF47A721A80D8F800301906A0
:1025F80001D505F053FF254B1B685A0742BF244AF3
:102608000A21118013F0080358D1224A138055E09B
:10261800D8F80000400717D55A2B15D192F8BB30CF
:102628002BB1012382F8BB1082F8BC3046E092F847
:10263800BD3083F0010382F8BD300BB10C2000E0FF
:102648000D200BF0FBFF39E05D2B00F028855B2B9C
:1026580000F027855E2B21D1032000F023BD00BFA9
:10266800441300208C25002000250020301B00206A
:1026780014000020BC290020800F0020802C00209E
:102688005C120020602D0020F22D00202C1B002061
:10269800F02D00203413002098120020562B01D171
:1026A80009F038F899F80030002B00F0108594F8FC
:1026B800B9306F2B40F005850EF0AAFDD8F8003030
:1026C800580736D594F8BD30B84A93B13B785907C6
:1026D8000FD5019BB3F90610B5F89A31994208DD78
:1026E800336813F0010302BF3221A2F8C01082F848
:1026F800BD303368DA030DD594F8C220AB4B2AB944
:1027080093F8BB2012B93222A3F8C020012384F821
:10271800C2300EE094F8BB30A44A53B13B7803F0C2
:10272800040303F0FF0123B9012382F8BB1082F8E8
:10273800BC30DBF800A0002333600AF17B090AF102
:10274800CB0B99F8002099F8013019F8010C9A423E
:102758000BD249460BF098FE38B119F8022C012328
:1027680003FA02F233681343336009F10409D945C7
:10277800E7D18F4B1B7853B18E4B8F4E1A68DFF819
:1027880050A212F0020F994640F0408337E30AF155
:10279800CA060AF589793278737816F8010C9A42D4
:1027A80025D231460BF070FE08B3B37896F804E0F2
:1027B800824A96F803A07D480C21013B01FB0E419B
:1027C80003EB43031344D1F8C8209A420FD0C1F851
:1027D800C830002390F8F420C1F8CC30012303FA64
:1027E8000EF322EA030381F8C4A080F8F430063619
:1027F8004E45D0D1724B1E68724B1B68039394F8F8
:102808002B300493704B029300230193029B1B68A7
:10281800002B00F0E98293F800A0BAF1000F00F055
:10282800E382029A039952688A1A002A0CDB01F59E
:10283800FA7202994A60019901228A4094F8F410C8
:1028480021EA020284F8F420049A002A00F0CC82DB
:10285800029A597812F8042C0432D2B2002940F0B6
:1028680082825A4931F91210B5F8982102F1C8004C
:10287800814202DD93F802B015E0C83A914203DACA
:102888009978C1F1000B0EE0019A0123934094F866
:10289800F42022EA030384F8F430039B029A03F538
:1028A800FA735360A0E294F8F430019A1341DB07FD
:1028B80000F19A82BBF1000FCCBF022001200BF07F
:1028C800E3FE0AF1FF33DFF8E490132B00F2848271
:1028D800DFE813F01400250037004B006400860081
:1028E800ED005001B701E701170282024B005A00C0
:1028F8008600ED005001BD002201870196F8009086
:10290800D944B9F1FA0FA8BF4FF0FA0929EAE979D1
:10291800304686F800900BF09DFD01200FE096F8F8
:102928000190D944B9F1640FA8BF4FF0640929EAAE
:10293800E979304686F801900BF08CFD0220494673
:10294800DCE196F803A0DA44BAF1640FA8BF4FF0AF
:10295800640A2AEAEA7A86F803A03046D9F8F81019
:1029680007F064FA03205146C8E171795944642993
:10297800A8BF642121EAE17171710D200BF0ECFD13
:10298800BAF10D0F00F02882317959446429A8BFA3
:10299800642121EAE17131710E20AFE1B179594426
:1029A80081F30801B1710520A8E100BF800F002064
:1029B800FE2D00205C1200202C1B00200C7C01083E
:1029C800BC120020BC29002048100020802C0020C8
:1029D800F41B002000007A440000C84200000000F8
:1029E800D9F8FC301A78022A22D107EE90BAF8EE0C
:1029F800E77AB2EE040A87EE800AD3ED097A30EE60
:102A0800270AB5EEC00AF1EE10FA09D45FED0E7A86
:102A1800B4EE670AF1EE10FAC8BFB0EE670A01E03B
:102A28001FED120A83ED090A0F200BF07FFD0AE063
:102A380099785944C829A8BFC82121EAE171997039
:102A48000F200BF089FDBAF10F0F00F0C581D9F8FE
:102A5800FC301A78022A20D107EE90BAB8EEE78A3D
:102A6800B2EE040A88EE008A93ED080A38EE000AEE
:102A7800B5EEC00AF1EE10FA09D45FED297AB4EE8A
:102A8800670AF1EE10FAC8BFB0EE670A01E01FED61
:102A98002D0A83ED080A122058E159785944C829AB
:102AA800A8BFC82121EAE1715970122026E1D9F89E
:102AB800FC301A78022A20D107EE90BAB8EEE70A5D
:102AC8005FED3B7A93ED0C7A80EE270A30EE070A29
:102AD800B5EEC00AF1EE10FA07D4B4EE670AF1EECB
:102AE80010FAC8BFB0EE670A01E01FED440A83ED93
:102AF8000C0A10200BF01AFD0AE0197B5944C8296A
:102B0800A8BFC82121EAE171197310200BF024FD38
:102B1800BAF1100F00F06081D9F8FC301A78022A57
:102B28001ED107EE90BAB8EEE78A5FED557A93EDBD
:102B38000B0A88EE278A38EE000AB5EEC00AF1EED5
:102B480010FA07D4B4EE670AF1EE10FAC8BFB0EE77
:102B5800670A01E01FED5F0A83ED0B0A1320F5E019
:102B6800D97A5944C829A8BFC82121EAE171D97284
:102B78001320C3E0D9F8FC301A78022A22D107EED4
:102B880090BA1FED6C0AF8EEE77A87EE800AD3ED6B
:102B98000F7A30EE270AB5EEC00AF1EE10FA09D422
:102BA8005FED737AB4EE670AF1EE10FAC8BFB0EEC3
:102BB800670A01E01FED770A83ED0F0A11200BF079
:102BC800B5FC0AE0997D5944C829A8BFC82121EA63
:102BD800E171997511200BF0BFFCBAF1110F00F0EB
:102BE800FB80D9F8FC301A78022A20D107EE90BA77
:102BF8001FED880AB8EEE78A88EE008A93ED0E0A80
:102C080038EE000AB5EEC00AF1EE10FA09D45FED0D
:102C18008E7AB4EE670AF1EE10FAC8BFB0EE670A12
:102C280001E01FED920A83ED0E0A14208EE0597D13
:102C38005944C829A8BFC82121EAE171597514204F
:102C48005CE0D9F8FC301A78022A20D107EE90BA55
:102C5800B8EEE78AB2EE040A88EE008A93ED0A0A13
:102C680038EE000AB5EEC00AF1EE10FA09D45FEDAD
:102C7800A67AB4EE670AF1EE10FAC8BFB0EE670A9A
:102C880001E01FEDAA0A83ED0A0A09205EE0D9785F
:102C98005944C829A8BFC82121EAE171D97009207F
:102CA8002CE0D9F8FC301A78022A1ED107EE90BA27
:102CB800B8EEE78A5FEDB87A93ED0D0A88EE278AB9
:102CC80038EE000AB5EEC00AF1EE10FA07D4B4EEF9
:102CD800670AF1EE10FAC8BFB0EE670A01E01FED0F
:102CE800C10A83ED0D0A0A2030E0597B5944C829EE
:102CF800A8BFC82121EAE17159730A200BF02CFC06
:102D08006AE0D9F8FC301A78022A22D107EE90BA84
:102D18001FEDD00AB8EEE78A88EE008A93ED100A14
:102D280038EE000AB5EEC00AF1EE10FA09D45FEDEC
:102D3800D67AB4EE670AF1EE10FAC8BFB0EE670AA9
:102D480001E01FEDDA0A83ED100A0B200BF0EEFB11
:102D580042E0D97D5944C829A8BFC82121EAE171B8
:102D6800D9750B20CAE7012936D19878B84B33F9C1
:102D78001230B3F5617F05DB40F633029342A8BFFA
:102D8800134601E04FF46173BAF10C0F24D14FF4EC
:102D9800966292FBF0F0AF4AA3F5617393FBF0F3F0
:102DA8005FFA83F913784B4516D0B9F1040F34BF95
:102DB8004B4602231370A84A0AFB035303F2AA7373
:102DC800136008F0CDFA504649460BF0C5FB09F1EF
:102DD8000100C0B20BF058FC019A0123934094F80B
:102DE800F420134384F8F430019B01330193029BD0
:102DF8000C330293019B042B7FF408ADBCE4D8F894
:102E08000030D80510D5954BDB786BB1336899073E
:102E18000AD5BAF8003013F0010B0AD10FF0DEF929
:102E2800012008F0C1F904E0012008F0ACF9012301
:102E380000E00023D9F8002052070DD563B1012026
:102E480008F0A1F9BAF800309B0708D40FF0C6F9CA
:102E5800022008F0A9F902E0022008F094F9BAF873
:102E680000307F4A13F0030F4FF4884114BF91617B
:102E78001185326812F00A0F27D0D9F80020D00641
:102E880009D559070AD4042008F08EF9754B1B8818
:102E9800A4F8003102E0042008F075F9D9F80030F0
:102EA8009A0607D5BAF800305B0606D4402008F029
:102EB8007BF902E0402008F066F9D9F8003058069E
:102EC80042BF684B1B88A4F802313368990609D4BD
:102ED800D9F800301A0540F191804FF4807008F05D
:102EE80063F98FE0604B1B789B0753D55F4B1B78CA
:102EF800042B4FD9D9F8003013F4007B0FD0BAF85F
:102F08000030DE063AD4102008F04EF9202008F0F0
:102F18003AF95748011D05F015FA02232AE0BAF8D4
:102F2800006006F01006B6B22EB1102008F02BF99A
:102F3800012684F804B1D9F80030580512D5D4F820
:102F480008314C495A89B1F90030002BB8BF5B42AF
:102F5800934207DAB1F90230002BB8BF5B429342C3
:102F6800C0F2F880BAF80030990608D5202008F099
:102F78000AF9002384F80431012600E0002694F8B9
:102F88000C31BBB90E200BF059FB3B4B012283F8E7
:102F98000C210FE0BAF8003003F03003002B97D073
:102FA800102008F0F0F8202008F0EDF8002384F84D
:102FB800043101E0002E8BD0304B002003F12806AD
:102FC80003F150042E4A002122F810102D4A5960AE
:102FD80022F810100432716022F8101000221A60D2
:102FE8009A603260B26022606160A2601433143665
:102FF800143400287FF46CAF0120E3E74FF48070AD
:1030080008F0C1F86B79082B01D00E2B02D14020B3
:1030180008F0B9F8D8F800305A0540F1B18095F8B1
:1030280010321BB93B7813F0040F03E0D9F80030D5
:1030380013F4002F2AD0144B00221A703C2005F0FC
:1030480055FC002800F09C800CF086FFF6E700BFD6
:10305800802C002044290020BC120020602D002074
:103068000010004834130020301B0020361B0020BD
:10307800C41200203C130020800F00209010002074
:10308800F42D002008110020551E00200EF090FDA0
:1030980009B0BDEC028BBDE8F04F05F028BB01205C
:1030A80000E002205FFA80F909F1FF3385F8A837BC
:1030B80008F0BCF808F078F948460BF0E5FAFFF795
:1030C800FDBABAF1000F02D07E2B3FF4F5AA94F8AE
:1030D800B930972B06D12D4B4FF4C872A3F8BE20F8
:1030E800FFF7ECBAA72B06D1294A137843F004035B
:1030F8001370FFF7E3BA0022BB2B079201D102231A
:1031080003E0B72B04D14FF6FE73ADF81E300AE08A
:10311800BE2B01D1022304E0BD2B7FF4CFAA4FF6CA
:10312800FE73ADF81C30DBF80030BDF81C10B3F8A6
:1031380058200A44A3F85820BDF81E10B3F85A20A6
:103148000A44A3F85A2008F0E5FA002384F8BA30B4
:10315800FFF7B4BABAF800309B063FF510AF20204D
:1031680008F022F80B480C4B011D1A685B68436095
:10317800026005F0E7F8054B012683F80461FEE6D6
:1031880009B0BDEC028BBDE8F08F00BF800F0020B6
:10319800301B0020CC120020381B00202DE9F04FF6
:1031A800C14BB3F90610C14B2DED028B1F687A890C
:1031B80085B0914201930EDBB1F5FA6FFC79BDBF82
:1031C8008B1A6343A2F5FA64C4F16404BCBF93FB91
:1031D800F4F4643400E06424B54BB64AB3F898B10B
:1031E80093F96231126802929BB21546039300224A
:1031F800AD4B33F912E0CBEB0E0303F2F31640F2BA
:10320800E63086424FEA420C03D8002BB8BF5B4237
:1032180001E04FF4FA73022A2ED0029E96F811614B
:103228001EB1B342CCBF9B1B0023A34E6FF0630AB1
:10323800642093FBF0F836F818900AFB083A08F176
:10324800010836F918600FFA89F8C8EB060606FB7C
:103258000AF696FBF0F699484E4420F80C60BE1822
:10326800642036797343964E93FBF6F364339BB22E
:10327800634393FBF0F02DE0029890F812611EB1C1
:10328800B342CCBF9B1B0023DFF860926FF063084A
:10329800642093FBF0F008FB003A39F91060013024
:1032A800002B39F91000A0EB060000FB0AFABDF864
:1032B8000C009AFBF8FAC6EB0A0A1AFB00FA7F48D8
:1032C800A0F804A0B879B8BF5B4243437C4893FB9D
:1032D800F0F064306B787B4E4FF06408434393FB07
:1032E800F8F3B354784EEB7A434393FBF8F3B354B3
:1032F8006B7D724E5843754B90FBF8F0022A985438
:10330800734B0ED1DE4583F802800DDB684CB4F8B0
:103318009A21914214DBB1F5FA6FA8BF4FF4FA6114
:103328000FE0DE459C5404DA36F80C305B4226F890
:103338000C300132032A05F101057FF459AFE5E7A6
:103348001146DFF8BCE15D4D891A4FF47A736FF0CE
:1033580063075943C2F5FA626423B1FBF2F191FBAA
:10336800F3F23EF8120007FB0211013207B23EF9F0
:103378001220D21B514391FBF3F30344F380554BC6
:103388001B885F0635D5544B544A1B881288DFEDDD
:10339800547A9B1A1BB208EE103AB8EEC88A28EE87
:1033A800278AB0EE480A07F04BFEF0EE408AB0EEEE
:1033B800480A07F0E2FDB5F9023006EE903AB5F991
:1033C8000030F8EEE66A07EE903A20EE667AF8EEFC
:1033D800E77AA7EEA87A67EE807ABDEEC77AE6EEBE
:1033E800A87A17EE103AFDEEE77A2B8017EE903A9E
:1033F8006B803C4D2B68980740F1A1803A4B3B4FBE
:103408001A687B6945F20721D31A8B4240F39780EB
:103418007A6105F02FFF364BDFF8E8901A78032A17
:103428009846B9F8003022D10A2B2AD9002328203F
:1034380088F800300BF0CBF805F01CFF2D4B1888EE
:103448000EF098FA2C4B1A68D37890FBF3F0013001
:1034580008282A4BA8BF08201870537980B213FB9C
:1034680000F33B83137913FB00F0788309E00A2B00
:1034780007D80323214A88F80030002313703B83C0
:103488007B8398F800301A4A012B3DD002D3022BD7
:103498004CD054E03A8BB9F800309A424FDD012302
:1034A80088F8003040E000BF802C0020BC120020CB
:1034B8004413002098120020002600203C1300200E
:1034C8000CFEFFFF142500201E11002017250020E8
:1034D8006C250020F41B00203413002082100020EB
:1034E80035FA8E3C98290020D82D00201011002094
:1034F8007C1B0020C81E0020181B0020080100208B
:10350800B21F00201C1B0020B9F800107B8B8B42D7
:1035180002DD022313700FE0A34B1B8B013399428A
:1035280002DD002313700AE0082006E07B8BB9F85F
:10353800002001339A42B2DC07200BF07FF82D6897
:10354800290577D5994B984F1A68FB69C3EB020890
:1035580045F2072398456DDD954BB6F906B0D3F8CB
:103568000090FA6199F80A30B4F85211914E012B83
:103578004FF47A70ABF57A7B98FBF0F803D042D31E
:10358800022B20D041E08C4B396A5A7B8B4B33F8A5
:1035980012204FF0080E92B291FBFEF3C91A8B1855
:1035A800BA843B6240F6E44293FBFEF39BB253437A
:1035B800B9F80820C2EB13335843B9F9063090FB29
:1035C800F3F0306021E07E4BB9F808A01B78C6F80C
:1035D80000A05A0719D57B480AF08DFF20B915F0CD
:1035E800100F18BF4FF0000B32220BFB0BF393FBAD
:1035F800F2F3B9F906205B445A434FF47A7392FB0D
:10360800F3F3534400E000233360D7E90A01336839
:103618006D4A03FB08F84FF47A7398FBF3F810EB44
:10362800080041EBE8710023C7E90A010EF01CFE0F
:10363800664B1860664E3368DB0427D52F0622D503
:10364800644B1B789D071ED5634B187804281AD93C
:103658000022624BD7180521951C4FF00A0E122A3A
:10366800D154E9B287F801E004D0B0EB510F2A46F3
:10367800EFD800E014215A18322002F8010CFF227A
:103688005A540F2000E00A200AF0D8FF544D2A6847
:10369800002A50D0534B544F1868396881429846D5
:1036A80049D8524BDFF8509119785268E1B94FF078
:1036B800010A83F800A0B9F80030D35C23B3504660
:1036C8000AF09EFF4A4B83F800A00EF0CBF9B9F838
:1036D8000030CBB92B681B78053B534514D80AF04A
:1036E8004FFF444B18600FE04FF0000A83F800A02A
:1036F800B9F80030D35C3BB150460AF081FF3C4B2F
:1037080083F800A00EF0AEF92A68B9F800305268C4
:103718003948D25CFE2A01D100230BE0FF2A02D1EE
:103728000AF074FF07E0D8F800500A2111FB025292
:103738003A6001330380224D2B78580704D52F4B6C
:103748004FF488529A6171E03268D1075CBF43F048
:1037580001032B701F4B1B781F075EBF2B7823F0CC
:1037680001032B70D60248BF2B78214A44BF23F0AF
:1037780001032B70224B1B6813F0040F02D0214960
:10378800098851B92049098809B1980705D41F4B00
:103798001B88003318BF0123D3B3022313702B787F
:1037A80023F001032B7038E010110020D82D0020E1
:1037B800181B0020241B0020B01E0020C01E002063
:1037C800FB2D0020CE140020407E0500281B002081
:1037D8005C120020301B0020361B002070290020BE
:1037E80024260020BC2900201C26002018260020A2
:1037F800842D00207C2B002020260020001000486B
:103808002C1B0020F02D00203E100020F22D00205F
:103818002978C90758BF022313700AF0B1FEB34BC9
:103828001B68C01A002801DB0EF01CF90EF0C0F965
:10383800AF4B1E789846002E00F0AA80AD4E336834
:10384800002B00F0DC8630680AF091FF002800F0B9
:10385800D686A84BA84C18680AF086FF092801D01C
:103868003F2850D14FF0000AD4F80090A34D574696
:10387800B9F1000F05D0A24829684A4611F060FF47
:1038880010B9AA4607B92F469E4B10359D42EFD373
:10389800C7B1D7F800E0DAF800C023681EF8035073
:1038A8001CF80300A8420DD15A1C954938B92D2B94
:1038B80005D8914D2A602025CD54885402E0CD5476
:1038C8002260EAE723680BB1574511D08E480CF007
:1038D80037FC574507D857F8100B0CF031FC092076
:1038E8000CF026FCF5E789480CF02AFC4FF000099B
:1038F80023689945A7D2824B13F809000CF018FCED
:1039080009F10109F4E72368002B40F05C860428DC
:1039180040F09E867A4808F04BF800F070BED9F85F
:103928000000DFF8F8A10AF022FF38B3DAF8000047
:103938000AF01AFFDBF8003093F848100246002915
:1039480034D124286BD1012283F84820DBF80030D9
:10395800DFF8C4A193F84820062AE0D193F849007B
:1039680001F0FAFB8346002800F083803B689879D1
:103978000CF02FFB3B68002283F84820644B93F837
:103988003530002B40F00D864C36982E00F03786E7
:10399800604BF21892F84A100129F5D15E4FF3589E
:1039A8003A605E4ABB4613609146B8E7012904D1E4
:1039B8004D2814BF00220222C6E7022904D13C2860
:1039C80014BF00220322BFE703290CD140284FF07F
:1039D800000102D983F84810B8E758711971D971F4
:1039E80098710422B0E7042906D1997983F849002F
:1039F8004A409A710522A7E70529A7D1587919796C
:103A08008842987906D950409871481C18710B441F
:103A18001A729BE790420CBF0622002294E72B788B
:103A28003F49580792D4232ADAF8003014D10120EC
:103A380088F800002F480391036035480292036319
:103A480038480CF07DFB31480CF07AFB0399029A58
:103A58000B7843F002030B70334B1B681B789342BF
:103A680001BF324B324A1A60324B04BF324ADA6025
:103A78006CE7DAF8002092F849304C2B00F0988473
:103A880000F28780332B00F0CE8421D8292B00F058
:103A98005B8409D8252B00F01584272B00F01984A6
:103AA800232B40F0D1853BE22D2B00F05E8407D814
:103AB8002B2B40F0C9850CF06FFA607100F06CBDDB
:103AC8002F2B00F01C85312B00F02E8500F0BCBD9B
:103AD8003E2B00F01B8146D8372B00F0D8842DD818
:103AE800352B00F0718200F0AFBD00BF882D00209B
:103AF800FE2D00206029002020200020408301089E
:103B0800F01F0020F0840108A39C0108A89C01086C
:103B180010110020B41D0020D41B0020D81B002049
:103B2800FB2D0020D89C0108581E0020FC9F002077
:103B3800EFBEADDE00ED00E00400FA05392B00F021
:103B4800D5833C2B40F08085DFF84C94D9F800A051
:103B58000CF022FA8AF80000D9F8003018780BF037
:103B680045F800F019BD432B00F06E8406D8412BB0
:103B780040F06A854FF0000900F05ABC442B00F071
:103B880007854A2B40F060850CF010FAA08100F000
:103B980003BDD02B00F00F8355D8CA2B00F0C0808E
:103BA80009D8C82B00F0858000F226834E2B00F040
:103BB8000C8400F049BDCD2B00F0088304D8CC2B31
:103BC80000F02A8200F040BDCE2B00F00883CF2BF6
:103BD80040F03A850CF0EAF96FF4AF6283189BB2B3
:103BE800C62B98BFA4F898010CF0E0F9A4F844019A
:103BF8000CF0DCF9A4F846010CF0D8F9A4F8480157
:103C08000CF0D4F9A4F8DA010CF0C6F984F8EF0145
:103C18000CF0C2F90CF0C0F984F8F0010CF0BCF912
:103C280084F887010CF0B8F984F894010CF0B4F921
:103C3800D94BD3F800900CF0B9F900EB80004000A4
:103C4800A9F8560052E3D62B00F039820AD8D22BB5
:103C580019D0C0F0F882D32B25D0D42B00F03B82AA
:103C680000F0F2BCEF2B41D005D8D82B40F0EC8403
:103C78004FF0000AE6E0F22B00F07582FA2B00F014
:103C8800B78200F0E1BC2B78590700F185840CF06D
:103C980083F9022884F8A80740F29382BF4B0022D8
:103CA80083F8A8278DE20CF081F9BD4B188000F04D
:103CB80073BC92F805904FEA5909B9F1120F03D96C
:103CC80004F010FE00F068BC4FF0000ACA4507D2A5
:103CD8000CF06CF9B34B23F81A000AF1010AF5E766
:103CE800B14B012283F8342000F056BCDFF8A892CB
:103CF800D9F800A00CF05AF9AAF85A00D9F800909F
:103D08000CF054F9A9F8580000F046BC0CF044F93E
:103D180084F8E2010CF040F984F8E10100F03CBCC1
:103D28009D4B1A681278022A824699466FD1D9F8B3
:103D380000B00CF031F907EE900AF8EE677AB2EEAF
:103D4800048AC7EE887A0BEB8A0BCBED087AD9F890
:103D580000B00CF021F907EE900A9FED947AF8EE86
:103D6800677A0BEB8A0BC7EE877ACBED0B7AD9F81B
:103D780000B00CF011F907EE900A9FED8D7AF8EE7D
:103D8800677A0BEB8A0BC7EE877A0AF1010ABAF158
:103D9800030FCBED0E7ACAD1BAF1070FD9F800B0EC
:103DA8001CD10CF0F9F807EE900AF8EE677AC7EE26
:103DB800887ACBED117AD9F800B00CF0EDF807EE5F
:103DC800900AF8EE677AC7EE887ACBED127AD9F8BE
:103DD80000B00CF0E1F88BF84C0012E00CF0DCF8C5
:103DE800D3448BF80100D9F800B00CF0D5F8D344CF
:103DF8008BF80B00D9F800B00CF0CEF8D3448BF850
:103E080015000AF1010ABAF10A0FC5D1C4E3D9F8BD
:103E180000B00CF0C1F8D3448BF80100D9F800B019
:103E28000CF0BAF8D3448BF80B00D9F800B00CF0BA
:103E3800B3F8D3440AF1010ABAF10A0F8BF8150056
:103E4800E5D1A9E3DFF850919FED598AD9F800B080
:103E58000CF0ACF807EE900AF8EE677A0BEB8A0BD9
:103E6800C7EE887ACBED087AD9F800B00CF09EF846
:103E780007EE900AF8EE677A0BEB8A0BC7EE887AA2
:103E8800CBED0B7AD9F800B00CF090F807EE900A59
:103E9800F8EE677A0BEB8A0BC7EE887A0AF1010A0B
:103EA800BAF1030FCBED0E7ACCD1BAF1070FD9F8DE
:103EB80000B01CD10CF07AF807EE900AF8EE677A99
:103EC800C7EE887ACBED117AD9F800B00CF06EF80D
:103ED80007EE900AF8EE677AC7EE887ACBED127A89
:103EE800D9F800B00CF062F88BF84C0012E00CF036
:103EF8005DF8D3448BF80100D9F800B00CF056F8FF
:103F0800D3448BF80B00D9F800B00CF04FF8D34429
:103F18008BF815000AF1010ABAF10A0FC5D13BE383
:103F28000CF03AF8132883463FF6CAAEDFF868A0CB
:103F3800DAF800900CF030F800231E4A0C2101FB3F
:103F48000322117A814222D10FFA8BFB09EB8B09EC
:103F5800137889F879300CF01FF889F87A000CF09A
:103F68001BF889F87B000CF017F8134B134A1A60FA
:103F780089F87C00124BDAF80000186000217930CB
:103F88000AF0A8FA0F4B80F00100187004E301331F
:103F98001C2BD2D194E600BF9812002044130020B5
:103FA80080100020802C0020101100200000C84242
:103FB80000007A44787C01087810002088140020DA
:103FC8007C100020140000200BF0E6FF0B2882462E
:103FD8003FF676AECE4BD3F800900BF0DDFF03280A
:103FE8003FF66EAE062303FB0A9989F8CE000BF064
:103FF800D3FF89F8C9000BF0CFFF89F8CA000BF08E
:10400800CBFF89F8CB000BF0C7FF89F8CC000BF089
:10401800C3FF89F8CD00BFE25379092B7FF650AE74
:10402800019BD3F800900BF0B7FF019B89F80000C3
:10403800D3F800900BF0B0FF89F801000BF0ACFF4B
:10404800019B64281B68A8BF642018710BF0A4FFAB
:10405800019B64281B68A8BF642058710BF09CFF63
:10406800019BFF281B68A8BFFF2098710BF094FFE5
:10407800019B6428D3F8009028BF642089F80700C2
:104088000BF08AFF019B89F80200D3F800900BF02F
:1040980083FF019B89F80300D3F800900BF086FF9B
:1040A8003B68A9F80A005B790A2B40F27582994BA4
:1040B800D3F800900BF070FF89F808006CE2824694
:1040C8000BF074FF944B23F81A000AF1010ABAF1B5
:1040D800080FF5D160E253790F2B7FF4F1AD0BF0A7
:1040E8005BFF072881463FF6EBADDFF824A2DAF83C
:1040F80000B00BF05BFF0E2303FB09F9CB44ABF8D0
:104108001901DAF800B00BF051FFCB44ABF81B01F2
:10411800DAF800B00BF04AFFCB44ABF81D01DAF82F
:1041280000B00BF039FFCB448BF81F01DAF800B070
:104138000BF032FFCB448BF82001DAF800B00BF01B
:104148002BFFCB448BF82101DAF800B00BF024FFE9
:10415800CB44DAF800A08BF822010BF031FFD144F0
:10416800C9F8230118E20BF017FF0F2881463FF624
:10417800A7AD0BF011FFC9EBC909A14489F8D40018
:104188000BF00AFF89F8D5000BF006FF89F8D60076
:104198000BF002FF89F8D7000BF0FEFE89F8D80073
:1041A8000BF0FAFE89F8D9000BF0F6FE89F8DA0070
:1041B8000AF080FCF0E12B785B0700F1ED810CF050
:1041C800F9F907F033F807F0EFF8E5E12B7858072D
:1041D80000F1E281514B4FF4C8721A80DCE12B7870
:1041E800590700F1D9814E4A137843F0040328E0B7
:1041F8002B785A07E5D527E20BF0CEFE484B1A7804
:1042080010B142F0020201E022F002021A700BF033
:10421800C3FE444BDFF82C9118700BF0D1FEC9F89F
:1042280000000BF0CDFEC9F804000BF0BFFE3E4BBA
:1042380018800BF0BBFE3D4B3D4A1880137843F0C5
:1042480002031370A8E10BF0A7FE02900BF0B8FE72
:1042580083460BF0B5FE82460BF0B2FE81460BF0AA
:10426800A5FE0BF0A3FE0BF097FE029BA3B9314B02
:104278001020C3F800B0C3F804A006F084FF284A51
:10428800137843F001031370B9F1000F00F0848133
:10429800294BC3F800907FE1102B40F07D81274B1C
:1042A800C3F800B0C3F804A0B9F1000F02D0224B44
:1042B800C3F800902148224B0222011D1A7004F015
:1042C80041F869E1A0600BF07BFEA3681843A06089
:1042D80062E10BF06BFEA4F85C010BF067FEA4F83A
:1042E8005E010BF063FEA4F8600155E10BF054FE8B
:1042F80084F87C010BF050FE84F880010BF04CFE32
:1043080084F87F010BF048FE84F8810144E100BF86
:1043180098120020BC120020462900203E100020E0
:10432800301B0020361B0020341B0020321B0020CD
:10433800C2120020C4120020D4120020CC12002087
:1043480084100020381B00200BF030FEA4F88201F6
:104358000BF02CFEA4F884010BF01EFE84F88601F5
:104368000BF024FEA4F8880116E10BF015FE84F882
:1043780092010BF01BFEA4F89C010BF017FEA4F8A9
:1043880098010BF013FEA4F89A010BF005FEDAF879
:10439800003084F893015B79082B40F2FD800BF024
:1043A80005FEA4F89E010BF001FEA4F8A001F3E0BD
:1043B8000BF0F2FD84F8D8010BF0EEFD84F8D9017A
:1043C8000BF0F4FDA4F8DA01E6E092F80590032377
:1043D800B9FBF3F9B9F1120F3FF672ACDFF888A315
:1043E8004FF0000BCB4580F0D7800BF0D5FD8AF855
:1043F800A2010BF0DBFD40F2ED23984205DD40F60B
:10440800CA039842A8BF184601E040F2EE20A0F285
:10441800EE2019230BF1010B90FBF3F00AF1020ACD
:104428008AF8A101DEE70BF0B7FD84F89401B3E048
:104438000BF0B2FD04EB090309F10109B9F1080F0A
:1044480083F88A01F4D1A7E00BF0A6FDC4F808B000
:1044580060710BF0B5FDA3681843A0600BF09CFDDC
:1044680084F892010BF0A2FDA4F85C010BF09EFD0C
:10447800A4F85E010BF09AFDA4F860010BF096FD1C
:10448800A4F882010BF092FDA4F8840184E053792A
:104498004FF0070AB3FBFAF2C2EBC2029A1A12F003
:1044A800FF0F7FF40DACB3FBFAFA0AF1FF3A5FFA9B
:1044B8008AFABAF1FF0F6FD00BF06EFD5FFA80FB3E
:1044C8004FFA8BF005F0C2FB814600283FF4F8ABA9
:1044D80080F800B00BF06AFDA9F802000BF05CFD53
:1044E80089F804000BF058FD89F805000BF054FD1D
:1044F80089F807000BF050FD89F80600D5E7DFF8CA
:10450800689209F1400A0BF051FDA9F8A0020BF0DE
:1045180043FD89F8A2020BF03FFD09F1040989F86F
:104528009F02D145EFD137E00BF036FD1F288146B9
:104538003FF6C6AB3B685B79082B7FF4C1AB0BF049
:1045480035FD09F1880904EB890A00F03F00AAF853
:1045580002000BF02BFDBAF80230800100F4FE5087
:104568001843AAF802000BF017FD000104F829000F
:104578000BF012FD14F8293000F00F00184304F86E
:1045880029000BF009FD8AF801000AF0C3FB03E0DB
:10459800624B012283F8352000200BF049FDFFF71C
:1045A800E5B95F4B98590AF0D9F818B932200AF0E2
:1045B8000EF8F6E70AF03EFA06F00EFE594B5A4A94
:1045C800DA60FFF7E1B90C2844D00A284BD1574DDF
:1045D80057480BF0B5FD2846232111F09AF808B189
:1045E800401B20602368002B60D1504823600021C5
:1045F800302211F058F898F80030002B2DD14D4B8F
:104608001B689B0615D54C4B44491B688A6B9A1A44
:10461800002A0EDB494A1278042A0AD9484A03F5C7
:10462800123303F5F8738B63938A9BB283F4884340
:104638009382444B9B68002B6BD0434805B0BDEC7C
:10464800028BBDE8F04F184704F04CF9FFF78EB91C
:104658000C2804D13D480BF073FD3D480DE07F2840
:1046680012D1FFF7F0B80D28B1D07F2809D1013B4E
:104678002E4A384823600021D1540BF061FDFFF722
:10468800E2B82F2B3FF6DFA8A0F12002D2B25E2AB3
:104698003FF6D9A813B920283FF4D5A85A1C2260A0
:1046A800224AD0540BF044FDFFF7CDB85A1EA95C3E
:1046B800202901D1134696E71C4A23600021D154D2
:1046C800254B264DD3F800A0D5F800B0DFF85C9054
:1046D800584611F02CF807463A464846594611F014
:1046E8002FF81F4A28B919F8073053445B785B073D
:1046F80003D010359542E7D306E0954204D2781CE2
:10470800EB684844984702E016480BF019FD00236F
:104718006BE705B0BDEC028BBDE8F08F10110020EF
:10472800B41D002000ED00E00400FA05F01F002091
:1047380087AA01082C1B0020D82D0020361B00203A
:1047480000100048902D00204C110020AD9C01085D
:10475800A89C0108D49C0108180100204083010886
:10476800F0840108B89C01084413002010F80A3CA2
:104778000133DBB20A2B84BF10F8131C044A00F87B
:104788000A3C82BF002322F8113000F80A3C704727
:10479800A42C0020334A136C90681944081A40F678
:1047A8008C23984270B513469160D06051603BD914
:1047B800127893F945108A4210460BD1111F082927
:1047C80008D893F84610182901D8013103E083F876
:1047D800442002E0002183F8461093F9444021491F
:1047E800A24219D191F84740B4B10C310024944247
:1047F80006DA1D4D51F8046F25F814600134F6E708
:104808000C2805D01849002421F810400130F7E79A
:10481800164801780131017083F8452000220121F2
:104828001A7083F8471070BD92F84710C9B1A0F20A
:10483800EF2440F2DA518C4208D811780B2905D8B8
:104848000B1D0131117042F8230070BD002283F85E
:104858004720074B03F13002002143F8041F93421D
:10486800FAD170BDBC010020A42C0020B4060020A1
:10487800C8010020024A136C0133194411647047BF
:10488800BC010020024B53F820301B6819607047A8
:1048980028260020064B53F820301A681B89A1F5FA
:1048A8007A7159434FF47A7391FBF3F111607047B1
:1048B80028260020054B98420CBF054A054A138854
:1048C80001339BB213800020704700BF00540040A2
:1048D800581200205A120020F0B5046D866823682B
:1048E80023F0010323608379054613F0020F407912
:1048F8000CBF4FF0000E4FF4005E13F0040F14BF0E
:104908004FF48067002710F0010F14BF0421002125
:104918008307206820F001002060626822F440527A
:104928004EEA02026260226822F4B05323F00C03BC
:1049380048BF41F008013B430B432360A36895B08F
:1049480023F44073A360684604F046FA284B9C425F
:1049580001D10C9B0EE0274B9C4201D10D9B09E035
:10496800254B9C4201D10E9B04E0244B9C420CBF7A
:104978000F9B109B2268A879170448BF5B00B3FB04
:10498800F6F206FB1233B3EB560F236828BF013249
:104998001E0441BF4FF6F073C2F34201134041EACF
:1049A80003026B7992B213F0020FA28100F00101A9
:1049B80014BF4FF400320022DC0748BF42F48032B3
:1049C8002B6D11B159680A4302E0596821EA0202C5
:1049D8005A609A6801074CBF42F0080222F00802A8
:1049E8009A601A6842F001021A6015B0F0BD00BF63
:1049F800003801400044004000480040004C00409E
:104A08003D4B1B78012B30B514BF00240324B1B9EA
:104A1800036A23F0010303628169036A21F0F30149
:104A280023F00A0341F0010142F001021A4341EA6E
:104A3800041181610262836923F00C031BE00429DD
:104A48001DD1016A4FF6EF730B4003628169056A55
:104A5800120121F473414FF65F7342F0100241F4E2
:104A680080712B4092B2134341EA043181610362A1
:104A7800836923F4406383618369836130BD0829B6
:104A8800016A1AD14FF6FF630B400362C169036ADA
:104A98009BB289B223F4206343F4807321F0F301BD
:104AA80043EA022241F0010192B241EA0411C161D4
:104AB8000262C2694FF6F37319E04EF6FF730B40BA
:104AC8000362C369056A40F6FF41194045F6FF7362
:104AD8002B4043F4805343EA023241F4807192B28E
:104AE80041EA0431C1610262C2694FF2FF331340E7
:104AF800C361C369C36130BDB801002038B510F87F
:104B08000E2C50F8043C044652B9012200F80E2C31
:104B180020F80C1C997A18680222BDE838406FE723
:104B280030F80C2C20F80A1C891A89B220F8081CC5
:104B3800074A10F80F0C002522F8101004F80E5C34
:104B48001868997A2A46FFF75BFF04F8065C38BDB7
:104B5800A42C0020044B53F820301BB107289CBF1D
:104B68001B681960704700BFE4020020084A1368F8
:104B78009B050BD5074B00211970074908684FF6AC
:104B8800FE7303400B604FF400735360704700BF1F
:104B980000000240FA2D0020300002402DE9F047C5
:104BA800664D2B6866490A78581C02F0FF068E4647
:104BB8000AB10346F6E72B60687BAB6895F80C8072
:104BC800AA7B374639B2202900F09B80DFF880C1E4
:104BD8000CEB81033CF82110DC789B78C3F1FF03D0
:104BE8009BB2002B65D0C3F1FF0363434FF03C0C2D
:104BF8001B12B1FBFCF9B9F1050F5DD8DFE809F02C
:104C0800030B1A293A4AE01ADAB24143B1FBFCF025
:104C18001044C0B251E0B1FBFCF00CFB101189B29A
:104C2800DAB2C1F13C01E31A4B432046B3FBFCFC6A
:104C380094442CE0B1FBFCF00CFB10115FFA83F8F4
:104C4800E21A89B24A43B2FBFCF24244D2B220468D
:104C580032E0B1FBFCF90CFB191189B25FFA83F859
:104C6800E01AC1F13C014843B0FBFCF04044C0B23B
:104C7800224621E0B1FBFCF80CFB1811D8B289B22E
:104C8800E31A01FB03F2B2FBFCFC224684445FFA00
:104C98008CF412E0B1FBFCF80CFB181189B2D8B205
:104CA800C1F13C01E31A4B43B3FBFCF20244D2B21C
:104CB80003E02246204600E044464FEA042C4CEA32
:104CC800004C4CEA020C172306F117014FF00108BB
:104CD80008FA03F8C91A18EA0C0F89B2DFF87480C9
:104CE80014BF4FF011094FF0090913F1FF3308F809
:104CF8000190E9D218360137B6B2BFB2114BA046BF
:104D080060E7AA73AB60104AE98001238EF800308F
:104D18000E4985F80C8040F22A336873AE805360E0
:104D280000234B620B889BB243F001030B8013688E
:104D380043F001031360BDE8F08700BF5011002065
:104D4800FA2D00205C110020300002400044014090
:104D5800FA0E00205D03002073B506460D460024B8
:104D680001232A88A34013421AD0AA78009302F09C
:104D780003038DF80430EB78022B03D0032B0CBF10
:104D8800032301238DF805303046C2F30113694629
:104D9800C2F381028DF806308DF8072004F092F9ED
:104DA8000134102CDCD102B070BD2DE9F04F734EE8
:104DB800F57B07460C4687B011469A4600686B1C7F
:104DC800914622464FF0020BF37307F09BFC3B8998
:104DD8007868ADF8043001A98DF806B08DF807B0F1
:104DE800FFF7BAFF0023ADF80A30ADF81230ADF87E
:104DF800163070230193BA7A3C68CDF80CA00123D1
:104E080006F110082D01ADF808304FF48073A8445E
:104E1800ADF810B0ADF814300C2A7ED8DFE802F0F7
:104E2800077D7D7D0F7D7D7D387D7D7D5E00204603
:104E380001A903F093FFA36943F0080326E0236A5E
:104E48004F4823F010032362236A6168A26922F0A5
:104E5800807222F4E642844242F4E04206D000F531
:104E68000060844202D043F0300307E023F0E003FF
:104E780021F4406143F0300341F480616160A26134
:104E8800C4F838A02362A36943F40063A36144E033
:104E9800236A3B4823F480732362226A6168E369CA
:104EA800844223F0730343F0700306D000F50060DA
:104EB800844202D042F4407207E022F4606221F496
:104EC800405142F4407241F480516160E361C4F89A
:104ED8003CA02262E36943F008031DE0236A2848E6
:104EE80023F480532362226A6168E369844223F4CD
:104EF800E64343F4E04342F4405203D000F5006037
:104F0800844201D141F480416160E361C4F840A06A
:104F18002262E36943F40063E3613A7B3B681AB1B8
:104F28005A6C42F400425A641A8892B242F0010262
:104F38001A80BA7A0C2A18D8DFE802F00717171770
:104F48000B1717170F1717171300721903F13401EE
:104F58000AE0721903F1380106E0721903F13C0105
:104F680002E0721903F14001116135444046A5F889
:104F780018906B6107B0BDE8F08F00BF501100209A
:104F8800002C0140F8B53A4E3A4C4000C7B24FF4F5
:104F980020453068C4F8D050D0F818E01EF4004F0F
:104FA80005D0AE46013DBEF1000FF5D116E0D0F8B0
:104FB80004E0314D0EEA050545F490353D43456062
:104FC8004FF42045C4F8D050D0F818E01EF0020F76
:104FD8002DD1AE46013DBEF1000FF5D1C4F8D05039
:104FE8001FE02946013D0029F8D081694906F8D516
:104FF800C4F8D05020494568294041F0007141F477
:10500800105141EA0241394341604FF42041A2B1B5
:10501800306885696D071ED411F1FF31F9D2C4F8E3
:10502800D010FFF747FC003018BF0120F8BD4FF43F
:1050380020458162C4F8D050D7E73068C4F8D01052
:105048000B46826992060CD41A46013B002AF8D115
:10505800C4F8D030E5E7416A03F8011B013AD2B23F
:10506800D3E7C4F8D0302023C3610120F8BD00BFC6
:105078005412002050110020009800FC400070B528
:10508800C5B23248324B00684FF42044C3F8D040D0
:105098008669360404D52646013C002EF8D113E073
:1050A80046682C4C344044F0807444F490342C43CB
:1050B80044604FF42044C3F8D0408669B60729D429
:1050C8002646013C002EF8D1C3F8D0401CE021460A
:1050D800013C0029F8D081690E06F8D544681D49BD
:1050E800214041F0007141F48031294341604FF47F
:1050F8002041C3F8D0108469A40711D40C460139A3
:10510800002CF8D1C3F8D010FFF7D4FB003018BF3B
:10511800012070BD4FF420448162C3F8D040DAE723
:1051280082624FF42042C3F8D0208169890606D4F0
:105138001146013A0029F8D1C3F8D020E4E7C3F8B2
:10514800D0202023C361012070BD00BF541200206D
:1051580050110020009800FC2DE9F0474D282DED56
:10516800028B044600F05E8600F2B980302800F019
:10517800DF8651D8222800F09D8423D8032800F028
:105188000B8214D8012800F0FB81022840F0088720
:1051980004200AF04DFF43200AF01BFF4C200AF0C0
:1051A80018FF46200AF015FF4C2000F061BE0428C5
:1051B80000F0FB81052840F0F3861A200AF038FF3A
:1051C800002402E2282800F0EC8515D8242800F0F5
:1051D800D385262840F0E486D14C06200AF028FF23
:1051E800B4F85C010AF027FFB4F85E010AF023FF67
:1051F800B4F8600100F0BDBD2C2800F0E5852E282C
:1052080000F066862A2840F0CB8601200AF010FFBD
:10521800C34B587900F02CBE3D2800F0FD821ED803
:10522800362800F036860BD8322800F01B86342842
:1052380040F0B68648200AF0FBFE002500F05CBC72
:105248003A2800F0C0823B2800F02D84382840F02E
:10525800A78604200AF0ECFEB14C00F093BD452867
:1052680000F08B8627D8402800F00586422840F0B9
:105278009786AB4C10200AF0DBFE60790AF0A9FE95
:10528800A0680AF0E1FE94F892010AF0A2FEB4F8D0
:105298005C010AF0D0FEB4F85E010AF0CCFEB4F866
:1052A80060010AF0C8FEB4F882010AF0C4FEB4F83E
:1052B800840100F05EBD492800F0B9824B2800F057
:1052C800A285462840F06C860D200AF0B1FE002029
:1052D8000AF07FFE00200AF0B7FE00F059BE7028E1
:1052E80000F0F68200F2E580692800F04C8200F2B6
:1052F800B680662800F0A68100F2A680642800F037
:105308007D81652840F04C86864C0B200AF090FE83
:1053180020880AF090FE6268834B9A420CBF20896D
:10532800608980B20AF087FE804B1B68C3F3C00017
:10533800C3F38002800040EA4200C3F340021043F6
:10534800C3F3401240EAC20003F0100318430AF006
:1053580072FE774B1A88E368247C02F0080103F494
:10536800475949EA010903F4804149EA010903F46C
:10537800004149EA010903F4803149EA010903F4CB
:10538800003149EA010903F4802149EA010903F4DB
:10539800002149EA010903F4801149EA010903F0EF
:1053A800007349EA0303DFF8A89199F8009012F016
:1053B800010FC9F3800914BF4FF002084FF000082D
:1053C80043EA090312F0020F43EA080314BF4FF03F
:1053D800040C4FF0000C12F0040F43EA0C0C14BF3D
:1053E8004FF0100E4FF0000E12F0400F14BF2027A0
:1053F80000274CEA0E0E12F0100F14BF4FF400767F
:1054080000264EEA070712F0200F14BF4FF48065FC
:1054180000253E4312F4807F14BF4FF40060002043
:10542800354312F4007F14BF4FF4001100212843C4
:1054380012F4806F41EA000114BF4FF0806300232B
:10544800002019430346E9E0672800F02381682813
:1054580040F0A68510200AF0EBFD00248AE16C28B4
:1054680000F0A48117D86A2800F008846B2840F05F
:10547800978505200AF0DCFD2E4B18880AF0DBFD25
:105488002D4B18880AF0D7FD264B93F8720000F0D0
:10549800010000F0EDBC6E28224D00F0988100F26A
:1054A800EF8106200AF0C4FD686E0AF0CDFD234B9B
:1054B80087E1782800F0FB8018D8742800F03D8335
:1054C8000AD8722800F09A83732840F0698508206A
:1054D8000AF0AEFD0124CAE3762800F0EF8300F25B
:1054E8006D832F200AF0A4FD154CD4E2A42800F007
:1054F8000C842FD87B2800F07482A02840F05085B7
:105508000C200AF095FD0F4B18680AF09DFD0E4B14
:1055180018680AF099FD0D4B186800F03DBD00BFF2
:105528004413002050120020005400402C1B00207F
:10553800F41B0020AA1B0020AC1B00202C13002009
:10554800477C0108ACF7FF1FB0F7FF1FB4F7FF1F38
:10555800FB2D0020F12800F0E680FE2800F0FC83F7
:10556800F02840F01D85B54C04200AF061FDA36CBD
:10557800B3F85A000AF05FFDA36CB3F85800F8E3DB
:1055880003200AF055FD00200AF023FD20460AF00A
:1055980020FD0D2000F06CBC0AF04AFD01200AF045
:1055A80018FD0A200AF015FDADE306200AF040FDBB
:1055B80043200AF00EFD48200AF00BFD46200AF0B1
:1055C80008FD33200AF005FDD2E39D4B185D013438
:1055D8000AF0FFFC0B2CF8D100249A4B185D01341B
:1055E8000AF0F7FC082CF8D10024974B185D013419
:1055F8000AF0EFFC072CF8D100F0D0BC07200AF025
:1056080017FDE7200AF0E5FC904B58790AF0E1FC19
:1056180000200AF0DEFC042000F0BEBCA3420AD23F
:105628008B4A9D5C012202FA05F50D421CBF9A4087
:1056380010430133F2E70AF007FD844B93F8A807FB
:1056480000F016BC12200AF0F3FC824B1B88B3F55D
:10565800806F8CBF0825012500247F4B33F9140087
:1056680090FBF5F0013480B20AF0E5FC032CF4D18C
:10567800724CA08D0AF0DFFCE08D0AF0DCFC208E75
:105688000AF0D9FC608E0AF0D6FCA08E0AF0D3FC92
:10569800E08E6EE310200AF0CBFC00246F4B185DFF
:1056A80001340AF096FC102CF8D100F077BC702079
:1056B8000AF0BEFC0026614D0E24AB6C74432344F3
:1056C8000136B3F819010AF0B6FCAB6C2344B3F801
:1056D8001B010AF0B0FCAB6C2344B3F81D010AF0BF
:1056E800AAFCAB6C234493F81F010AF072FCAB6C64
:1056F800234493F820010AF06CFCAB6C234493F824
:1057080021010AF066FCAB6C234493F822010AF0ED
:1057180060FCAB6C1C44D4F823010AF095FC082EFD
:10572800C9D100F03BBC7020484C0AF081FC04F160
:10573800700594F8D4000AF04CFC94F8D5000AF0EF
:1057480048FC94F8D6000AF044FC94F8D7000AF014
:1057580040FC94F8D8000AF03CFC94F8D9000AF010
:1057680038FC073494F8D3000AF033FCAC42E0D19B
:1057780000F014BC3A4B185D01340AF02AFC102CD6
:10578800F8D100F00BBC374D2878400000F0FE003F
:105798000AF04EFC00242B789C4280F0FF83324BA9
:1057A80033F814000AF047FC0134F4E72F4C0620C4
:1057B8000AF03EFC20880AF03EFC60880AF03BFCB8
:1057C8002B4B1888D5E204200AF032FCE3E30720CB
:1057D8000AF02EFC274B1888FF28A8BFFF20C0B26C
:1057E8000AF0F7FB244B186880F3100080B20AF027
:1057F80022FCB5F868000AF01EFC144B93F88721C8
:105808001E4B186822B10A23584380F3100001E0A8
:1058180000F30F0080B2ACE20C4C02200AF008FC46
:1058280094F8E2010AF0D5FB94F8E10120E30220A4
:105838000AF0FEFB054B98899BE200BF501200203E
:10584800109D01081C9D0108259D01084413002096
:105858006112002016000020261300208812002064
:105868009C120020501E0020802C0020902900202F
:10587800341300201C1B0020281B0020241B0020A0
:105888000B200AF0D5FBEB6E18780AF0A2FBEB6E42
:1058980058780AF09EFB0026EB6EC44C3344013660
:1058A80018790AF096FB032EF6D1E36ED8790AF040
:1058B80090FBE36E98780AF08CFBE36ED8780AF0D8
:1058C80088FBE36E58890AF0B6FBE36E187ACFE2DC
:1058D800B64C1E200AF0ACFBA36C1B78022B4FF0D1
:1058E80000056BD1A36C03EB850393ED080AB2EEB8
:1058F800048A20EE080A10F0E5F880F30800C0B228
:105908000AF067FBA36CDFEDAA7A03EB850393ED3E
:105918000B0A20EE270A10F0D5F880F30800C0B271
:105928000AF057FBA36CDFEDA37A03EB850393ED35
:105938000E0A20EE270A10F0C5F880F30800C0B25E
:1059480001350AF046FB032DCCD1072DA36C23D1DA
:1059580093ED110A20EE080A10F0B4F880F308005D
:10596800C0B20AF036FBA36C93ED120A20EE080AC7
:1059780010F0A8F880F30800C0B20AF02AFBA36C64
:1059880093F84C3000EE103AB8EE400A10F09AF84E
:1059980080F30800C0B20BE02B4458780AF019FBDA
:1059A800A36C2B44D87A0AF014FBA36C2B44587DC3
:1059B80001350AF00EFB0A2DC7D1EFE2A36C2B4488
:1059C80058780AF006FBA36C2B44D87A0AF001FB3E
:1059D800A36C2B440135587D0AF0FBFA0A2DEDD152
:1059E800DCE23C200AF024FB0024704D9FED718A14
:1059F800AB6C03EB840393ED080A20EE080A10F061
:105A080061F880B20AF017FBAB6C03EB840393EDEB
:105A18000B0A20EE080A10F055F880B20AF00BFBCA
:105A2800AB6C03EB840393ED0E0A20EE080A10F02A
:105A380049F8013480B20AF0FEFA032CD5D1072CBC
:105A4800AB6C16D193ED110A20EE080A10F03AF863
:105A580080B20AF0F0FAAB6C93ED120A20EE080A55
:105A680010F030F880B20AF0E6FAAB6C93F84C000C
:105A78000BE0234458780AF0DEFAAB6C2344D87A5A
:105A88000AF0D9FAAB6C2344587D01340AF0D3FAF2
:105A98000A2CD4D182E214F8010F002800F07E828B
:105AA8000AF097FAF7E701200AF0C2FA3F4B9B6C1D
:105AB8001878DDE150200AF0BBFA00253B4B9C6CBE
:105AC8003D4B04EB85040C2194F8792001FB02334B
:105AD800013593F838000AF07CFA94F87A000AF055
:105AE80078FA94F87B000AF074FA94F87C000AF0CB
:105AF80070FA142DE2D151E22C4B9C6C062303FB67
:105B08000544013594F8CE000AF063FA94F8C90008
:105B18000AF05FFA94F8CA000AF05BFA94F8CB002E
:105B28000AF057FA94F8CC000AF053FA94F8CD002A
:105B38000AF04FFA0C2DDFD130E24FF000080126B1
:105B480000271A4B1A7C974227DA11330024FA5C93
:105B5800194D0C2305F130016343595C914207D17B
:105B68002B44586B0FF0E3FD82462EB9B14605E091
:105B780001341C2CECD10EE080440CE0D1450ADA4B
:105B88000C2303FB04535B6B13F809000AF021FA9A
:105B980009F10109F2E70137D3E7002E00F0FE8191
:105BA8005FFA88F00AF044FA0026C9E7501200208C
:105BB8000000C84200007A44487C0108CF4D287C88
:105BC8000AF036FA00242B7C9C4280F0E781CC4B0B
:105BD800E65C0021CB480C2200F1300702FB01F300
:105BE800DA5DB24205D1034493F838000AF0F1F9BE
:105BF80002E001311C29EDD10134E4E7C24C162042
:105C08000AF016FAB4F898010AF015FAB4F8440143
:105C18000AF011FAB4F846010AF00DFAB4F848018E
:105C28000AF009FAB4F8DA010AF005FA94F8EF0173
:105C38000AF0CFF900200AF0CCF994F8F0010AF044
:105C4800C8F994F887010AF0C4F994F894010AF0A5
:105C5800C0F900200AF0BDF9A84B9B6C0A20B3F9E3
:105C6800563093FBF0F080B20AF0E5F98AE0E0B232
:105C780001340AF0AEF9092CF9D18FE110200AF0AD
:105C8800D7F9A24BA24C187800F002000AF0A1F94B
:105C9800A04B18780AF09DF920680AF0D5F96068D9
:105CA8000AF0D2F99C4B18880AF0C5F99B4B188862
:105CB8000AF0C1F9914BB3F870005AE00AF06CF998
:105CC800074612200AF0B4F98C4C17B9666FA56F15
:105CD80006E0102F13BF0025E66FD4F880502E463B
:105CE80038460AF076F930460AF0AEF928460AF046
:105CF800ABF9D4F884000AF0A7F900200AF09BF960
:105D080000200AF098F90020B2E07C4D95F8880050
:105D180080000130C0B20AF08BF995F888000AF0CB
:105D280058F900242E4696F888309C4280F0368137
:105D38007B4D285D0AF04DF905F11003185D0AF056
:105D480048F905F120033035185D0AF042F9285D5D
:105D58000AF03FF90134E6E708200AF069F9002063
:105D68000AF069F900200AF066F900200AF063F9E0
:105D780000200AF060F911E104200AF059F9624B99
:105D8800986809E194F87C010AF023F994F88001F5
:105D98000AF01FF994F87F010AF01BF994F88101C1
:105DA80066E0594C07200AF043F9B4F882010AF07A
:105DB80042F9B4F884010AF03EF994F886010AF031
:105DC80008F9B4F88801D4E74F4C0C200AF030F9F0
:105DD80094F892010AF0FDF8B4F89C010AF02BF946
:105DE800B4F898010AF027F9B4F89A010AF023F9EF
:105DF80094F893010AF0EDF8B4F89E010AF01BF943
:105E0800B4F8A001B5E7404C04200AF011F994F861
:105E1800D8010AF0DEF894F8D9010AF0DAF8B4F8F3
:105E2800DA01A6E73F4C404D207800EB4000C0B2B5
:105E38000AF0FEF8002623789E4205F1020580F05C
:105E4800AD8015F8020C0AF0C4F815F8010C00EB47
:105E5800800000EB800000F2EE2080B20AF0EBF840
:105E68000136E8E701200AF0E3F8274B93F894019C
:105E78000AF0AFF892E008200AF0DAF80024224B82
:105E88002344013493F88A010AF0A3F8082CF6D1C8
:105E980084E01A4B1C4C93F8C900C0EBC000C0B298
:105EA8000AF0C6F804F11805204A94F8F60192F9A8
:105EB800001043B2994275D092F90C10994271D0F2
:105EC80092F918209A426DD00834AC42ECD165E0C2
:105ED80040200D4C0AF0ACF804F14005B4F8A002DB
:105EE8000AF0A9F894F8A2020AF073F8043494F8B6
:105EF8009F020AF06EF8AC42F0D14FE05012002039
:105F080061120020487C010844130020301B002047
:105F1800381B0020361B0020341B0020321B0020B9
:105F2800D9120020501E0020E61400205C1E00201C
:105F3800E0202A4C0AF07CF804F18005B4F822022B
:105F480000F03F000AF077F8B4F82202C0F3861098
:105F58000AF071F894F8200200090AF03AF894F867
:105F6800200200F00F000AF034F8043494F81D02FF
:105F78000AF02FF8AC42E1D110E013200AF058F8EB
:105F88000024174B185D01340AF023F80B2CF8D1C4
:105F980000200AF059F800200AF056F8012018E00D
:105FA800002016E00AF015F8B4F8F8010AF043F8F2
:105FB80094F8FA010AF00DF894F8FB010AF009F8D0
:105FC80094F8FD010AF005F894F8FC010AF001F8CC
:105FD8007AE7BDEC028BBDE8F08700BF44130020D0
:105FE800109D01082DE9F047C94CCA4E237886B0A8
:105FF8000746002B00F0138232686368D31A7C2BA3
:1060080040F20D82237A6260013323724FF0000858
:1060180008F12400BE4DC0B20BF0BAFD05F10A0329
:1060280033F9183007EE903ABB4B1B88B8EEE77A85
:1060380007EE903AF8EEE77A08F10108C7EE277AFA
:106048009FEDB67A67EE877AFDEEE77ACDED037AB3
:10605800BDF90C000BF08AFDB8F1030FD8D1302040
:106068000BF096FDB5F910000BF080FD0BF088FDE4
:106078002B7A9A072CD16A6841F288339A4218D948
:1060880010200BF085FD4FF06408686990FBF8F06C
:1060980000B20BF06BFD21200BF07AFD686990FBD4
:1060A800F8F308FB13000028B8BF404200B20BF019
:1060B8005DFD14200BF06CFDB4F918000BF056FDD3
:1060C8001C200BF065FD00200BF050FD0BF058FD77
:1060D800237ADFF83C825B0740F07E8102200BF0D8
:1060E80057FDD8F81C00DFF848926423323090FB43
:1060F800F3F000B20BF03AFD0320B8F926500BF08C
:1061080047FD874B1B7813F0040F4FF0050A95FBEA
:10611800FAF5ADB20DD008F5D970394608F0EBF9AB
:1061280028B9D9F8003013F0100F18BF002528B28D
:1061380005E0D8F8FC379889B0FBFAF000B20BF00C
:1061480015FDD9F800309F0740F18A80DFF8E49107
:10615800B4F8027899F80030B4F800286C4D3F0183
:106168004FF06408BFB208FB02325B00B2FBF3F3E6
:1061780047EA0327BFB2C3F303231F4306200BF0EC
:1061880007FD38B20BF0F2FCB4F8023899F80010A9
:1061980001339BB293FBF1F201FB1233A4F80238EE
:1061A800D4F804389B7B012B05D139200BF0F0FC87
:1061B800B5F900081AE0B5F800586E233A205D4397
:1061C80015270BF0E5FC95FBF7F5AFB2B7FBF8F533
:1061D80028B20BF0CBFC08FB15753B200BF0D8FC64
:1061E800A8B2451D0A2095FBF0F000B20BF0BEFCEA
:1061F80028200BF0CDFCD4F80838454D0A2093FB35
:10620800F0F000B20BF0B2FC04200BF0C1FCD4F8A3
:10621800FC37D5F80C089A894FF6FF739842A8BF47
:106228001846C2B10028ACBF131A134607EE903ABD
:106238009FED3C7AF8EEE77A67EE877A07EE102A48
:10624800B8EEC77AC7EE877AFDEEE77A17EE900ABE
:106258006428A8BF642020EAE07000B20BF086FC36
:10626800D4F810382A4F9D0640F1AB8097F81438BF
:1062780098071DD511200BF08BFCB7F816082A4B90
:106288004FF4F365684390FBF3F000B20BF06EFC3B
:1062980019200BF07DFCB7F816084543642095FBE0
:1062A800F0F595FBF0F300FB135000B20BF05EFC29
:1062B80094F81438B4F8185813F0020F08BF0025E2
:1062C80001200BF065FC28B20BF050FC09200BF004
:1062D8005FFC00200BF04AFC144B94F81A581A88FB
:1062E800B2F5967F0AD90A4B1B7A03F00F03072BE6
:1062F80004D842F20F75954228BF154605200BF0C9
:1063080047FCD4F804385B7BC3B928B233E000BF3C
:106318001C130020BC2900201600002000007A442D
:10632800FB2D00200000C842A08601000A010020C1
:1063380098290020080100206666E63FA5F12003A1
:1063480007EE903A1FED047AF8EEE77AF6EE006A67
:10635800C7EE877ABEEE007AF5EEC07AF1EE10FA53
:1063680058BFB0EE667A77EE877AFDEEE77ACDED24
:10637800037ABDF90C000BF0F9FB94F81428C94B0B
:10638800910703D493F81B28012A04D1012384F828
:106398001B38C5481CE0D3F80438DFEDC46A93ED18
:1063A800017AD3ED027A27EE267A67EEA67ABDEE59
:1063B800C77AFDEEE77A8DED047ACDED057A04A86B
:1063C80006E0BB4A92E8030004AB83E803001846E2
:1063D80004F0C6FA0BF0D4FB237A282B1FD1B14B5B
:1063E80000221A723C2733684FF47A70B3FBF0F836
:1063F80017200BF0CDFBB8FBF7F5B5FBF7F007FB63
:106408001050000200B20BF0B1FB18200BF0C0FBDB
:1064180007FB158000B20BF0A9FB0BF0B1FB94F859
:106428002438A04D002B00F0628108F0A9F8D5F8B7
:106438002838A04AC31A9342074640F2C680002370
:1064480085F82E3885F83038B5F80038DAB21B0AE6
:1064580085F84A2885F84B3885F8402885F841386A
:10646800D5F8582833689A1AD5F85C38D97B4FF490
:106478007A734B439A420ED38F4B1B68C5F8583832
:1064880095F86038013B012B9FBF102385F82E3803
:10649800022385F830380A20D4F8082892FBF0F255
:1064A80084F84828121284F8492894F81428D4F853
:1064B8000C3893FBF0F384F84C381B1284F84D38F1
:1064C800920794F81A38774984F87B3803D42D2337
:1064D80081F87C3877E0042BD4F81C98D4F820682D
:1064E800DFF8E481754A8CBF3323322381F87C3886
:1064F8004FF0060C724B99FBF3F096FBF3F308FB95
:10650800009108FB036803EB83030CFB01F103EB29
:10651800830391FBF2FE642502FB1E119B0091FB95
:10652800F5F184F86D1809120CFB08FC84F86E1854
:106538009CFBF2F143FA81F39BB202FB11C292FB7E
:10654800F5F284F87228121284F8703884F87328E7
:106558001B0AB4F8162884F871382423534393FB94
:10656800F5F5B4F88E3884F8743800EB80001B0A0F
:1065780000EB8000800084F875380A22B4F81838D7
:10658800B3FBF2F303F5FA739BB240FA8EF080B2D4
:1065980084F876381B0A4FEAD97984F86B08F60F25
:1065A800000A84F8685884F87738C5F30725B4F8E2
:1065B800903884F86A9884F86C0884F86F6884F8CE
:1065C800695884F87D38C4F8287894F89288354D4D
:1065D800B8F1000F0DD1D5F8980808F0C8F80128CF
:1065E80007D90228374E00F0628204F0ABF9012384
:1065F800B370D4F89C282B4D002A78D095F892686F
:106608003EB1D5F8A43840F6B731FB1A8B4219D8F9
:106618006DE00123D5F8980885F8923803F0BFF9A2
:10662800D5F8A83893F9000002238DE8480008211E
:1066380032464FF4964303F0CDF985F8AC68C5F8B7
:10664800980852E095F8A068CEB9D5F89808C5F82A
:106658009C6885F8926803F0A2F9D5F8A83893F9F0
:10666800000001238DE84800082132464FF4964384
:1066780003F0B0F9C5F8980804F064F935E0013E74
:10668800F6B285F8A06895F8AC1895F8AD38EEB96B
:106698004A1C013385F8AC2885F8AD38D5F8980838
:1066A80021E000BF1C130020381B00208096184BE7
:1066B800D47D01083F0D0300BC29002040420F0093
:1066C8008096980016000020806967FF12F8016B19
:1066D800C5F89C28701885F8AC080133D5F89808D7
:1066E80085F8AD38314608F045F8C4F8A47894F830
:1066F800AE38A24DF3B1D5F8B038DBB1D5F8B4381F
:10670800C3B1C5F8B8381B689D4AC5F8BC38D5F878
:10671800C0381344187AFEF71FFDD5F8B8389879B1
:1067280009F057FCD5F8C0380133092B88BF00237E
:10673800C5F8C038934D94F8C4282E688F4B002AAA
:1067480000F0F081D3F8C828002A00F0EB8193F814
:10675800CC38013B012B00F2E581D4F8C808874FFB
:1067680008F005F8E0B1D7F8C80807F0FDFF97F87A
:10677800CD38D5F800907E2B80460ED102231B28F9
:1067880087F8CC3809D1D7F8C80807F0F0FF20B946
:106798000123C7F8D09887F8D43884F8CD88DCE787
:1067A800D7F8D0282B689B1A41F6583293421ED945
:1067B800032387F8CC38B5E1734A32F8130010B9CF
:1067C80003464FF403600133B0F5C06FDBB279D0F4
:1067D8001ED9B0F5006F7FD032D9B0F5036F3FD125
:1067E80084F8D538D4F81038644F99063FD494F813
:1067F800D41894F8D538002900F056812A68921BDD
:10680800012AD9D984F8D538002384F8D43889E105
:10681800B0F5007F43D007D8B0F5807F49D0B0F5F8
:10682800887F00F08D80E6E7B0F5806F00F0B080DB
:10683800B0F5826F00F0F580B0F5047FDBD123E07E
:10684800B0F5E26F00F08D80B0F5E46F00F08E8057
:10685800B0F5E06FCFD184F8D538B4F90A1089E0E3
:10686800B0F5046F76D0B0F5026FC4D105E197F8A2
:1068780014389A07BBD5B7F8161824234B4312339C
:10688800642193FBF1F109E184F8D5383F4B3B4F84
:106898001B689B07ABD5B7F800380A21FDE084F8E0
:1068A800D5383A4B354F1B681905A0D5D7F80818C5
:1068B800F4E084F8D538D4F81038304F5A0796D514
:1068C8007969EBE084F8D538304B2C4F1B681B05F1
:1068D8008DD5D7F80C18E1E0D4F81018274A84F8B9
:1068E800D5388F0683D592F8141888077FF57FAFBF
:1068F800D90712D5D2F8203883EAE371002BA1EB2F
:10690800E37101EB51014FF01902B1FBF2F1ACBF99
:1069180041F0004141F040410FE0D2F81C3883EAD1
:10692800E371A1EBE371002B01EB51014FF0190268
:10693800B1FBF2F1B8BF41F080414FF400608BE049
:1069480084F8D538D4F810380C4F5B077FF54FAF73
:106958003969A3E0B4F9181084F8D5386423594389
:106968007AE084F8D538B4F90C1003E0B4F90E10C5
:1069780084F8D5382C2391FBF3F16DE01C1300202B
:10698800D47D0108BC290020129E01089829002006
:1069980084F8D53894F8D638644A0133DBB2032B2F
:1069A80088BF012382F8D63894F8D61842F21073BB
:1069B80059435F4B1B78D80748BF01319A0748BF36
:1069C80002315F07B4F8D83848BF0431D80748BF48
:1069D8000A319A0748BF14311F0648BF2831D80525
:1069E80048BF28315A0748BF64311F0748BFC8311C
:1069F800980548BF01F5C8719A0648BF01F57A7134
:106A0800DF0648BF01F5FA61580648BF01F57A610B
:106A18004FF4806003F062FF444B002283F8D428CF
:106A2800E5E6D4F81018DFF8048184F8D53811F0B9
:106A3800200717D098F8142812F0020F14BF4FF44B
:106A48007A71002112F0010F14BF4FF4FA6300238A
:106A58000B4494F81A18194403F040FF002384F8F3
:106A6800D438C4E6334B1B6819067FF5C0AE3946E7
:106A780003F034FF88F8D478B9E684F8D538D4F828
:106A880010382A4F9A067FF5B2AE97F814389B074C
:106A98007FF5ADAEB7F818386421594303F01EFFEF
:106AA800002387F8D438A2E684F8D5383AE0B378DA
:106AB80023B1C5F8947886F802809AE5D5F8943819
:106AC800FB1AB3F57A6FFFF494AD0123D5F8980853
:106AD800B37007F049FE0646D5F8980807F044FE5B
:106AE80076067FF486AD8A2802D08E280DD080E500
:106AF800D5F8103898067FF57CAD95F89238002BBC
:106B08007FF477AD05F6610306E095F89238002B1F
:106B18007FF46FAD05F62C03C5F89C382D2385F856
:106B2800A03866E506B0BDE8F08700BF1C1300205A
:106B3800FB2D0020982900200D4B0E491A680E4B9A
:106B480092B213445B000D4A1B68C3F3090310B5E6
:106B5800136013689BB201335B1000229A4206D07F
:106B6800074851F8044B20F812400132F6E710BDEF
:106B7800505C0040206200401E300020F8280020B1
:106B8800FD280020014B00221A607047F4280020DD
:106B980013B506220446A82119206B46FEF7F2F920
:106BA800F8B19DF800309DF8012043EA0222022145
:106BB8009DF8033012B292FBF1F222809DF8022078
:106BC80042EA032212B29DF8053092FBF1F262808C
:106BD8009DF8042042EA03231BB2012093FBF1F342
:106BE800A38002B010BD08B5242180221920FEF729
:106BF80045FA642007F0EBFC202197221920FEF7C4
:106C08003DFA0A2007F0E3FC102223211920FEF7A1
:106C180035FA642007F0DBFC024B4FF480521A80EF
:106C280008BD00BF16000020154B37B508220546E1
:106C38001A85E8200AF050F8002400200AF04CF8E1
:106C48000DF804000134062CF7D10D4B08229A6187
:106C58009DF800209DF8013043EA02232B809DF81F
:106C680002209DF8033043EA02236B809DF804203C
:106C78009DF80530012043EA0223AB8003B030BD04
:106C880000100048274A73B55369274C43F4001392
:106C9800536103236946082501268DF805302046EF
:106CA80000238DF806308DF8073000958DF80460C4
:106CB80002F008FA1D4AA561138823F040031B045B
:106CC8001B0C1380138823F038031B041B0C2B4365
:106CD800138013889BB243F040031380242025853A
:106CE80009F0FAFF802009F0F7FFA561642007F09A
:106CF80063FC2585202009F0EFFFAF2009F0ECFFA9
:106D08003046A56107F058FC2585232009F0E4FFEB
:106D1800602009F0E1FFA561642007F058FC02B08B
:106D280070BD00BF00100240001000480030014054
:106D3800024B4FF480221A60704700BF14040140D0
:106D48002DE9F04F944D954C2B68954E9BB22380BE
:106D5800228831880A40900585B007D54FF6FF5341
:106D6800904A2B6013780133DBB2137023880B40F1
:106D7800190440F143830023ADF80A302B68874992
:106D88009AB21804228040F139830B8803F00F036C
:106D98008B70002B40F00483834A844F1368844827
:106DA8009BB23B803B8803F0300303803B8803F4AD
:106DB80040533B80D2F800E04BF6BF730EEA030362
:106DC80083F4005383F0200343F4004343F080032B
:106DD80013600B8813F0100F804626D1116848F60F
:106DE8000F730B40734913600B681A7A022A89469D
:106DF80001D0042A05D101F0D1FDD9F800301B7A61
:106E08003FE1062A6ED15A78052A09D11A78520626
:106E180006D1D87801F0A6FD674B1B681B6A984716
:106E2800664B1B689B6898475CE013689BB2ADF89B
:106E38000A30BDF80A301B0540F1F38111685D483E
:106E480040F68F730B405E4913600A685D4B92B23F
:106E580013445B0081461A68036893F808E0BEF1A2
:106E6800090F8A4617D092B2520002F1804202F509
:106E7800C04211781970517859709188C8B2090ABE
:106E880041EA002159801189C8B2090A41EA002162
:106E980099809289DA8001221A72DA8893F801B00F
:106EA800002A40F0F1801A7812F07F0250D1BBF12D
:106EB800090F10D1DA78012A00F2CA8099780029DE
:106EC80040F0C6809988002940F0C2809A723A4BF7
:106ED8001B685B68BAE0BBF1050F10D193F903207A
:106EE800002A01DA0823CCE09A78002AFAD19A8895
:106EF800002AF7D19B7A002B00F0B480F2E7BBF1AF
:106F0800030F0FD1DA78012A40F0A2809A88002A6C
:106F180040F09E805A7A42F020025A72264B1B6833
:106F2800DB6993E0BBF1010F40F09280DA78012A27
:106F380040F08E809A88002A40F08A805B7A980612
:106F480040F1868001F0D8FD002800F08B807FE0BA
:106F5800012A39D1BBF10B0F7AD1184A5879126836
:106F6800D97892699047D9F800309A7A002A6FD078
:106F780000286DD11A79002A6AD19B78002B67D135
:106F88000D4B1B68DB6898470A4B1B685A79DA7205
:106F9800DA781A7366E000BF445C0040F81B0020F2
:106FA8003E290020FC2D0020005C0040821E0020AD
:106FB800801E0020AC1D0020B01D0020AC1F00204A
:106FC800505C004004300020022A41D1BBF1010F7F
:106FD800B8D0BBF1030F3BD1587920F0800E4FEAAF
:106FE8008E0202F1804101F5B84110F0800F096866
:106FF80014BF01F0300101F44051BEF1030F27D84E
:10700800B3F802E0BEF1000F22D109B39B7AFBB1BD
:1070180002F1804202F5B842010613684BBF23F41F
:10702800E04323F4804323F0400323F070034BBF75
:107038009BB29BB283F0100383F4805343F4004364
:1070480043F080031360A94B1B689B69984709E0CC
:10705800A74B1B6858465B699847032810D000283F
:107068007FF440AFDAF80020A24B92B213445B00E1
:107078001A6800221A603023A8F80030062300E0BE
:107088000923D9F8002065E1BBF1060F13D11A785E
:1070980050067DD19A78964B012A02D11B68DB698C
:1070A8006AE0022A02D11B681B6A65E0032A6FD1D5
:1070B8001B685B6A60E0BBF1000F3AD15988002970
:1070C80066D15A6822F47F42B2F5003F60D11A783F
:1070D80012F07F0204D19B88002B00F0F48157E066
:1070E800012A0AD1824A5879126892699047002881
:1070F8004ED1D9F800309B7A17E0022A48D15A7944
:1071080002F00F010BB29B0003F1804303F5B84373
:1071180012F0800F1B6814BF03F0300303F44053D0
:10712800032935D812F0700F32D1002B40F0CB81F3
:107138002EE0BBF1080F04D11B78590600F0C58179
:1071480026E0BBF10A0F23D11A7802F07F02012A48
:107158001ED19A7AE2B15988D1B95A6822F47F428D
:10716800B2F5803F14D1624A587912689269904703
:10717800002800F0AC810BE053B1D9F800204FF0A3
:10718800000AA2F812A093615046984750460BE0B7
:10719800574BD9F800201B6850781B69984703287B
:1071A80002D1554B1B6806E0D9F800301A8A4FF611
:1071B800FF718A4201D1092203E0022800D012B9E6
:1071C80008221A72C7E093F90010002923DAD98837
:1071D80003910398DFF818E1824202D9039A1A82D0
:1071E80011E08A420FD2DEF8001091F82C0082429A
:1071F80001D2002105E092FBF0F100FB112212B947
:1072080001213E4A1170DEF8002092F82C209A8263
:1072180001F0C4FB9FE003221A724FF440533B80F5
:1072280099E0BDF80A301BB2002BBFF6A7AD116874
:1072380040F68F730B4013602F4AD2F8009099F8EC
:107248000830022B934600F08280042B7FD0032B5A
:1072580001D0052B75D1D9F81830B9F810209BB991
:10726800B9F81020002A4FD04FF440533B80244BEC
:107278001968204B89B20B445B001968002119601A
:107288003023A8F800303FE0002AE9D0B9F814A06C
:10729800924528BF92461FFA8AF2104601929847F3
:1072A800019AB9F810309B1AA9F81030B9F81230C1
:1072B8001344A9F81230124B1A68124B92B21344B5
:1072C8005B000AF1010A1B689BB203F1005303F546
:1072D80040534FEA6A0A5B0000215145C0D053F879
:1072E800212020F811200131F7E700BFB01D002050
:1072F800AC1F002002300020AC1D0020FD2D002016
:10730800505C004004300020B9F814309342DBF898
:10731800003001D8032201E012B105221A720CE0F4
:10732800062119726C4B19686C4B89B20B445B00CF
:1073380019681A603023A8F80030DBF800301B7A8F
:1073480006E0072B03D1664B1B68DB6898470823C8
:10735800DBF80020137201F0B3FB624B1A684BF69E
:10736800BF7313403A88D2043A8848BF83F48053E5
:107378009004B8F8002048BF83F40053D106B8F849
:10738800002048BF83F01003920648BF83F0200313
:1073980043F4004343F08003524A9BB213602DE04C
:1073A8009A0002F1804202F5B842116889B2ADF83C
:1073B8000A10BDF80A1009B2002909DA106840F667
:1073C8008F7101401160013B474A52F823309847BA
:1073D800BDF80A301F067FF5D1ACA1788B0003F108
:1073E800804303F5B84348F60F72186802401A60E4
:1073F8003D4B03EB81039B699847BFE422883388A0
:107408001340590505D54FF6FF332B60374B5B68A2
:107418009847228831880A40920444BF4DF6FF738A
:107428002B602388324A0B40DB0452D54EF6FF739B
:107438002B600023D370D378052B41D8DFE803F005
:10744800030D1418222DA368294D1BB908F068FCF8
:10745800062300E00523EB703BE008F061FC042301
:10746800E3700123A36034E002232371032328E09F
:107478002379013BDBB22371237953BB1C4B0422D4
:10748800DA7026E01B4A13689BB243F010031360BE
:107498000523E3700A2323711BE02379144A013B77
:1074A800DBB22371237903F0FF0093B911490C680B
:1074B8004FF6EF7323400B600623D370906008E00B
:1074C8000623E37005E00C4B57E60C4B55E60C4BD6
:1074D80053E605B0BDE8F08F505C00400230002054
:1074E800AC1F0020005C0040E87D0108200000205F
:1074F800F81B0020405C0040CF8500087586000816
:1075080055860008704770477047FEE7FEE7FEE7BC
:10751800704730B50024E3B293420DD2030F092B14
:1075280094BF3033373301F8143001EB440300259E
:1075380000015D700134EEE730BD0248024905F0F4
:1075480078B800BF0048014074270020014802496C
:1075580005F06FB800400140242700200148024987
:1075680005F067B800340140FC26002001480249B4
:1075780005F05FB800340140FC26002001480249AC
:1075880005F057B800080040D42600206D4B6E4A1D
:107598009FED6E7AD2ED007ADFED6D4ADFED6D3A40
:1075A80030B51C88B3F90AE01D8A06EE904AB8EE99
:1075B800E76AF8EE666ADFED687AB3F9044067EEC9
:1075C800E67AB7EE004AE6EE077A9FED647A67EE50
:1075D800666A9FED637AE6EE076A27EEA77A07EEFA
:1075E800904AB3F902409FED5F6AF8EEE77A67EEDA
:1075F800277A07EE104AB8EEC77ADC89E6EE877A72
:10760800B6EE007AFDEEE76A87EE866AC3ED066A93
:10761800F8EEE66AD2ED017A9A89E6EE874A06EE36
:1076280090EAB3F908E09FED507A05EE90EAF8EE9B
:10763800E66AF8EEE55A66EEA46A65EEA45A66EEC6
:10764800A46AB3F806E0E6EE875A65EE875AA5EE17
:10765800A34AF0EE445A04EE10EAB8EE444A25EE86
:10766800844AB5EE404AF1EE10FA5BD02DB205EE31
:10767800905A24B224EEA45A07EE104AF8EEE55ABE
:1076880012B265EE255AB8EEC75A65EEA35A64EEF3
:10769800854AB0EE007AE4EE875AB5EE007A65EED8
:1076A800875A07EE102AB8EEC75A9FED307ADFEDF9
:1076B800306AB3F91620E5EE075AF8EEE77A9FED3F
:1076C8002D7A76EEE77ADFED2C6AE5EEC77A05EEDD
:1076D800902AB0EE677ADFED297AB3F91420B3F96E
:1076E800123067EE277A07EE102AC7EE847AF8EE92
:1076F800E55AB8EEC77A65EEA75A27EE877A65EE9F
:10770800A75A27EE237AA5EEA67AF0EE476A07EE87
:10771800103AB8EEC77A36EE877ADFED196AE7EEE7
:10772800267A01E0DFED177A18B1FDEEE77AC0EDB1
:10773800007A31B1FDEEC67A642217EE903A5343CF
:107748000B6030BD20030020041C0020000000371F
:1077580000007AC700000038000000390000803AB5
:10776800000080380000A045000000360000804777
:107778000000804900008039000000300050C345F7
:107788000000803D00000000704770476C4B6D4A58
:107798002DE9F04F5E8994684FEA062AB4EB0A0A8D
:1077A8009C884FEA04481C894FF000054FF0000BF5
:1077B80065EB0B0BA4FB0A6704FB0B77F40944EA9F
:1077C800476418EB04065C884FF000094FEAE71598
:1077D8004FEAC438DC8849EB050787B0CDE9046770
:1077E800A4FB0A6704FB0B77340A44EA076418EB26
:1077F80004064FEA27259C894FF0000949EB050745
:10780800CDE90067AAFB046704FB0B77F40D44EA93
:10781800472414F5FA664FEAE75545F10007B6F52F
:10782800FA6F77F10003CDE90267964667DAA4FBA1
:10783800046704FB05F34FF0050C07EB4307DDE98C
:107848000489A6FB0C230CFB07335F104FEA3206B2
:10785800B8EB06084FEA920669EB070946EA837611
:107868009F10DDE90023921B63EB0703DDE9026744
:10787800CDE90023344A4FF0FF33964277EB0303F8
:10788800CDE9048928DA40F6AC52A4184FF0000379
:107898005D4104FB05F3A4FB044505EB43056FF0CC
:1078A8000602664202FB0566A4FB0223334418EB7A
:1078B800020649EB0307CDE904670B26A4FB062360
:1078C80006FB0533DDE900455B104FEA3202A41AD6
:1078D80065EB0305CDE900450AFB0BF3DDE902453D
:1078E800AAFB0AAB0BEB430B4FEADA7242EA4B02F4
:1078F800A41A4FEAEB7365EB0305CDE90245DEF800
:107908000C40009B019DA4FB032304FB05334FEAB5
:1079180052584FEA635948EAC328DDE90423B8EB13
:10792800020269EB03039946D30B43EA494300B1CA
:10793800036009B1029B0B6007B0BDE8F08F00BF80
:107948000E030020041C002024FAFFFF044A137CC5
:1079580023B1012303700023137470470370704729
:10796800041C002007EE900AF8EEE77ADFED0C6AB7
:107978009FED0C0AF5EEC07AF1EE10FAD4BFB1EE25
:10798800677AC7EEA67A08B5D8BFC7EE267A27EE7B
:10799800800A03F055FB044B83ED000A08BD00BFC5
:1079A8008096184B35FA8E3CAC0000207620F421E6
:1079B8003122FDF763BB772048210122FDF75EBB2A
:1079C800772058210122FDF759BB1FB50446022133
:1079D8000C2001220DF10703FDF7D4FA08B90020A5
:1079E8003BE09DF80730DB07F9D50321062202ABFF
:1079F8000C20FDF7C7FA0C20092101220DF107031D
:107A0800FDF7C0FA0028EAD09DF8073013F00C0FF4
:107A1800E5D19DF809209DF8083043EA0223C3EB1D
:107A280083339B009DF80B2023809DF80A3043EA9E
:107A38000223C3EB83339B009DF80D2063809DF8E0
:107A48000C3043EA0223C3EB83339B00A3800C2052
:107A58000A210122FDF712FB012004B010BD07B571
:107A6800F7216B4606227620FDF78CFA9DF8003048
:107A78009DF801100B4A1B0343EA01139DF80210FD
:107A880043EA111353609DF803309DF804101B035B
:107A980043EA01139DF8051043EA1113136003B07C
:107AA8005DF804FB041C002007B5002101AB03228C
:107AB8007720FDF767FA9DF805309DF804001B0252
:107AC80043EA00439DF80600184303B05DF804FB41
:107AD80008B5FFF7E9FF014BD86008BD041C00207A
:107AE80008B5FFF7E1FF014B986008BD041C0020B2
:107AF80013B506220446432168206B46FDF742FA77
:107B0800A8B19DF800209DF8013043EA02232380A4
:107B18009DF802209DF8033043EA022363809DF814
:107B280004209DF8053043EA0223A380012002B017
:107B380010BD13B5062204463B2168206B46FDF7AD
:107B480021FAA8B19DF800209DF8013043EA0223EC
:107B580023809DF802209DF8033043EA02236380C6
:107B68009DF804209DF8053043EA0223A3800120F4
:107B780002B010BD07B50A2100220C20FDF77EFADD
:107B8800142006F024FD0A210F220C20FDF776FAB6
:107B98000A2006F01CFD01AB102103220C20FDF782
:107BA800F1F90A2006F013FD0A2100220C20FDF746
:107BB80065FA0A2006F00BFD0DF1030302210122EC
:107BC8000C20FDF7DFF90DF10303092101220C2038
:107BD800FDF7D8F90A2101220C20FDF74FFA03B06E
:107BE8005DF804FB08B508F073F86B218022682063
:107BF800FDF744FA642006F0EAFC6B2103226820B2
:107C0800FDF73CFA0F2006F0E2FC104B19211A7818
:107C18006820FDF733FA0F2006F0D9FC0C4B1A2127
:107C28001A786820FDF72AFA1B2118226820FDF728
:107C380025FA1C2110226820FDF720FA6820372138
:107C48000022BDE80840FDF719BA00BF3C03002038
:107C58000000002008B508F03BF8074B1B7813B16B
:107C6800012B03D008BD4FF4006201E04FF48052AD
:107C7800024B1A8008BD00BF0C030020160000202C
:107C8800F8B59E4B1B680546187818B1012800F016
:107C98006B81E6E2242D9A4C0CD006D80A2D00F010
:107CA800DC800D2D00F0D98048E12A2D06D02C2D3E
:107CB80004D043E16074A074E07451E1914BA17C5D
:107CC800677C8F4A002058542FBB197817754729AD
:107CD80021D1597850291ED19978472907D1D978C7
:107CE800472904D11979412901D1012111759978C0
:107CF800844A522903D1D1784D2900F0B482997869
:107D0800804A472907D1D178532904D11279562AB4
:107D180004BF03222275227D794E022A3AD0032A13
:107D28004DD0012A40F08780BA1E072A00F28380CE
:107D3800DFE802F004080F131A25812B09F0CCF9AB
:107D4800A06178E01B78532B75D1A3695B42A361CE
:107D580071E009F0C1F9E0616DE01B78572B6AD139
:107D6800E3695B42E36166E01B78302B664B1A7867
:107D78008CBF42F0020222F002021A705BE000207F
:107D880009F00AFA84F8200055E0002009F004FA06
:107D9800608450E0072F06D0082F4CD1012009F04D
:107DA800FBF9F08447E0012009F0F6F941F21843A5
:107DB80058434FF47A73B0FBF3F0B0843BE0022FE2
:107DC80007D0032F0BD1002009F0E6F94F4B1870AC
:107DD80031E0002009F0E0F986F828002BE02AD9E4
:107DE8003A1F921096F828300132D2B2013B02EBCA
:107DF8008303DBB2102B1ED8F91EC2F1010201EB7E
:107E08008202D2B2012A0BD0042A11D100205E1EB0
:107E180009F0C2F93E4B98553E4B00229A5507E0AF
:107E28005E1E3D4A0020935509F0B6F93B4B985524
:107E3800E36A0133E362324B2A2D18BFDA7C07F17B
:107E480001074FF000000CBF012255406774A07471
:107E58000CBF83F83020DD7482E094F830000028ED
:107E680047D02F4B13F8012D2E495A708B42F9D168
:107E7800244A234D13785278402B85BF373B1B018A
:107E88001B01DBB298BF03F0F003402A8CBF373ADE
:107E9800303AD2B21344E27CDBB29A4226D1212393
:107EA8000B70287D6B6B1F4A013301286B630AD066
:107EB80002281DD1722313701B4BAA8C1A801B4BEE
:107EC800EA8C1A8014E0672313700F4B1B789F0706
:107ED8000FD5174BAA691A60EA695A60154B95F8CD
:107EE80020201A70144B6A8C1A8002E03F230B7012
:107EF8000020002384F8303032E000BF480800201A
:107F0800041C0020C4290020301B0020D8120020A7
:107F180009130020F9120020D9120020E9120020CC
:107F28005C03002048030020321B0020C012002000
:107F3800381B0020361B0020341B0020A37C94F83B
:107F480030000E2B9FBFAC4A591C9174AB4A98BFA6
:107F5800D554A94A18B9D37C5D40D57400E00020F7
:107F6800003018BF0120F8BDA34B93F83810002249
:107F7800082900F27681DFE801F0050C101A2B3B86
:107F8800607E8B00B52D40F06C8183F8392001228A
:107F980050E0622D08BF02224CE0032283F838200B
:107FA80083F83A5083F83B5083F83C5059E1042257
:107FB80083F8382093F83B2093F83C1083F83D5021
:107FC8002A44D2B283F83B200A4483F83C2048E193
:107FD800052283F8382093F83B2093F83C10DD877E
:107FE8002A44D2B283F83B200A4483F83C2038E183
:107FF800062283F8382093F83B2093F83C102A4453
:10800800D2B283F83B200A4483F83C20DA8F02EB93
:108018000525ADB2B5F5AC7F88BF774ADD8784BF4B
:10802800012182F839100022A3F84020002D40F0E9
:108038001881072283F8382013E193F83B2093F83E
:108048003C102A44D2B283F83B200A4483F83C20EF
:10805800B3F84020B2F5AC7F3CBF6749891802F1FC
:10806800010238BF81F84450D98F92B29142A3F8E7
:108078004020DED9F5E0082283F8382093F83B3019
:10808800AB4200F0EE805C4B012283F839200FE010
:108098005B4C83F8382014F8012D6270594A9442D9
:1080A800F9D193F83C10544AA94206D03F232370D3
:1080B800554A536801335360D3E0516B92F8390045
:1080C8000131516310B13E232370CAE02121217090
:1080D80092F83D10062941D004D8022907D0032977
:1080E80023D0F8BD122959D0302967D0F8BD5021C6
:1080F80021704649946C4C60D46C0C60516D4FF4FF
:108108007A7491FBF4F1424C218092F89C11414A17
:1081180019B1117841F0020102E0117821F0020151
:108128001170012283F89D218DE05321217092F86E
:108138004910CE0705D592F84820D51E6A426A41F3
:1081480000E0024602F0010183F89C11002A7AD16E
:1081580030490A7822F002020A7074E04F21217037
:1081680092F84F10CC0705D592F84E20D11E4A42FE
:108178004A4100E0024602F0010183F89C1122B94D
:1081880024490A7822F002020A70234A93F87310ED
:108198001170224AB3F87010118054E056212170F2
:1081A8001F49946D0C8042F21074D16D91FBF4F16B
:1081B8001C4C2180012182F89E1144E04921217044
:1081C80092F84810184A102988BF102111701749D1
:1081D80014780022A24233D2154D0E7A5655154D09
:1081E8004E7A5655144DCE7A5655144D11F80C6FDB
:1081F80056550132EEE700BF041C0020C4290020B8
:108208005C0300204803002028080020381B0020B9
:10821800341B0020301B0020361B00200A010020E0
:10822800321B0020C0120020D8120020481C002059
:10823800D9120020E9120020F912002009130020A9
:10824800DA6A0132DA6293F89D310B4A93B192F8F7
:108258009E317BB1002182F89D1182F89E1118464B
:10826800F8BD0020F8BD1279432A7FF448AD0222F8
:10827800227544E5F8BD00BF041C00200449054BE5
:108288000968187000225A6199611A77704700BF0F
:10829800BC2900202808002010B5121A07EE902AE1
:1082A8005B1A2DED028BF8EEE78A07EE903A184B31
:1082B800059CB8EEE78AD3ED007A28EE278A28EEE7
:1082C800080AA8EEA80A0DF0A3FEDFED127A049BB7
:1082D80020EE270AF0EE480ABCEEC00A83ED000A39
:1082E800B1EE680A0DF0F0FCDFED0B7A9FED0B7A2A
:1082F800E0EE077ABDEC028BFDEEE77A17EE903AD6
:10830800002BBCBF03F50C43A033236010BD00BF96
:10831800AC0000202C7D8E3F00A00C46A00CB3457D
:1083280044F25063984203DDA0F50C40A038704732
:10833800034B9842BCBF00F50C40A030704700BF0B
:10834800B0B9FFFF73B51A4C036823600B6863600C
:10835800184D0068184EFFF705FB184B009395E879
:10836800030094E80C000196FFF796FF144B32685F
:108378001A606868636813491B1A07EE903A124B33
:10838800286893ED007A23681B1A0B600F4BF8EEF0
:10839800E77A1A600E4B67EE877A1B68FDEEE77A7C
:1083A800DA880C4BC1ED017A1A8002B070BD00BFAB
:1083B80094280020381B0020A02800209C2800209A
:1083C800DC280020A4280020AC000020D4280020AD
:1083D80088100020D02800204279DFED2A5A2A4B45
:1083E8009FED2A5A07EE902AF8EE677AC27BC7EE0D
:1083F800A57AB2EE047AC3ED007A07EE902AF8EE79
:10840800677A234ADA60C7EEA57AC3ED017A8179E3
:10841800204B07EE901AF8EE677A017CDA60C7EE17
:10842800877AC3ED007A07EE901A817E06EE101A5D
:10843800F8EE677AB8EE466AC7EEA57A86EE056A60
:10844800C3ED017A83ED026AC179134B06EE901AE7
:10845800417CDA60F8EE666AC6EE876A07EE101AA3
:10846800C17EC3ED006A07EE901AB8EE477AF8EEBF
:10847800677A87EE257AC7EE857A83ED017AC3EDB0
:10848800027A70470000C842AC28002000007A44F5
:108498000000FA44BC280020E028002010B50C4C4D
:1084A80023789B0713D50B4B1B78042B0FD90A4A4B
:1084B8000A4B106852685A601860FFF753FA084B65
:1084C8001A88084B1A80237843F00103237010BDE3
:1084D800301B0020361B0020381B0020C41200204F
:1084E80034130020F02800201C4B1B681B0307B521
:1084F80030D51B4A1B4BD2ED007A1B788DF8003023
:10850800B2EE047A67EE877A174B9FED187A1B78DC
:108518008DF80130FCEEE77A0A2017EE903AD2ED9A
:10852800017A8DF8023067EE877A6946FCEEE77AC1
:1085380017EE903AD2ED027A8DF80330FCEEE77A26
:1085480017EE903A8DF80430094B1B788DF80530FA
:1085580001F034FE03B05DF804FB00BF9829002049
:10856800AC2900208A290020A829002000007A448C
:108578008E290020054A137883F001031370044AFA
:1085880000231360034A1360AEE700BF8E29002062
:10859800A4290020A029002007B5232006F017F8F9
:1085A8006820752101220DF10703FCF7EBFC28B1C7
:1085B8009DF80700A0F168035842584103B05DF8E0
:1085C80004FB00BF704708B51F4A18B95368022258
:1085D8001A8208BD0020516810800B7813F07F03C1
:1085E8000DD14B7A990644BF0221117013F0400F48
:1085F800137814BF43F0010323F0010315E0012BA6
:108608001FD0022B1ED14B7913F0800F03F00F03FC
:108618004FEA830303F1804303F5B8431B6806D090
:1086280003F03003102B07D10123137004E003F487
:108638004053B3F5805FF6E793681B699847024893
:1086480008BD104608BD00BFA81D002010B5064C87
:1086580018B9636801221A8210BDA3689B689847FD
:1086680060680C3010BD00BFA81D002010B5064C76
:1086780018B9636801221A8210BDA3681B6898475D
:1086880060680A3010BD00BFA81D0020084BDA68DA
:10869800D10709D4DA68D20608D4DB6813F0040FCE
:1086A80014BF032004207047012070470220704740
:1086B8000020024010B50446B0F9000008F005FBA0
:1086C800B4F9020008F001FBB4F90400BDE8104059
:1086D80008F0FBBA10B50446006808F0F6FA6068BE
:1086E80008F0F3FAA068BDE8104008F0EEBA2DE9EA
:1086F800F74F012001F092FB002488B3012C2FD8FA
:10870800194E4FF04C0909FB04FA06EB0A0808F168
:108718005407BD7815B10134E4B2EEE790F90030A2
:1087280090F804E01846114B03228DE8240001213B
:108738002A4653F82E3001F04DF9834660B106F110
:108748000C00504429464A460CF0ADFF01231C4456
:10875800C8F80CB0BB70E4B2012001F043FBCCE7D1
:1087680003B0BDE8F08F00BFA81D0020207E0108DF
:1087780010B5184C002120461A220CF094FFA4F5DD
:10878800FA70142380F8F63105230022042180F8BA
:10879800FA3180F8FC3180F8023280F8043280F82F
:1087A8000A3280F80C325223012480F8FB1180F839
:1087B800FD2180F8031280F8052280F80B1280F85A
:1087C8000D2280F8F43180F8FE2180F80642A0F8E6
:1087D800F84110BD3815002010B5FFF757FF4FF4CA
:1087E8003024012806D11CB1FFF750FF013CF8E7FF
:1087F800052010BD002C08BF052010BD70B5064629
:10880800441E14F8011F89B1094D28460CF081FF58
:108818000028F6D005F1080398423FBF054B401BDE
:10882800C018A31B38BF80F88A31EAE770BD00BFC3
:10883800329E010844130020031EB8BF2D2210B534
:10884800B8BF58420C46B8BF01F8012B0A2202F003
:1088580065FA00230370204610BD07B51C4B03F1D1
:10886800A802C3F8A4201B4A92F892215AB1012AFF
:1088780014D1032183F8AA10072183F8AC2083F8C8
:10888800AB100C2208E0022183F8AA10032183F818
:10889800AC2083F8AB10072283F8A8200E4B0F4AB0
:1088A8001A60402001F0BAFA70B10122002390F951
:1088B800000040218DE80C00094A4FF4E13301F033
:1088C80089F8003018BF012003B05DF804FB00BF31
:1088D800A81D0020441300201C0000205516010884
:1088E800E91701080120002107F084BBF0B51C4AF4
:1088F80092F8AD30D2F8B05092F8B47092F8C060E7
:1089080092F8CCE0022B0ED805EBC304591CA31C2B
:10891800C9B206D02346A48814F0010F01D0204222
:1089280005D10B46EEE782F8AD300020F0BD93F993
:1089380002307CB29C4201D1002307E074B29C4211
:108948000CD04FFA8EF49C42EBD1022382F8AD1082
:108958000C2101FB0322D2F8B800F0BD0123F5E792
:10896800A81D002030B5002202F1805303F5B8534A
:108978009B0042F400441D6840F60F7144F08004E7
:10898800294001322143042A1960EDD1024B40F0FD
:108998008000186030BD00BF4C5C00402DE9F843F2
:1089A800324D6E68328A377ABAB9042F15D13048F9
:1089B8000378012B0CD12F4B19682F4B89B20B442C
:1089C8005B0019681A603023A5F8D830027049E0B6
:1089D8001023A5F8D830072744E0B48AB369A24227
:1089E80094BF04270227944228BF14461FFA84F82C
:1089F800404698471F4A13689BB203F1005303F59A
:108A080040535B0004F1010E1B689BB203F1005355
:108A180003F540534FEA6E0E5B000021714500F1EB
:108A2800020009D010F8019C10F802CC4CEA092C7D
:108A380023F821C00131F1E712680F4B92B21344B9
:108A48005B001A681C60338AC8EB03033382738A9D
:108A580098443023A5F8D8304FF44053A6F8128034
:108A6800A5F8DA306B681F72BDE8F883A81D0020EE
:108A7800FD2D0020505C0040023000200E4B0F4AB4
:108A88001B689BB203EBC00002443E294FEA420236
:108A980009D94B09C80604BF03F1FF339BB29B02F7
:108AA80043F4004304E04B08C90748BF01339B0265
:108AB80011681360704700BF505C0040063000200A
:108AC80008B50B4B002093F83010FFF7D7FF094B80
:108AD8005A68107A082801BF4FF48052A3F8DA20A8
:108AE8001022A3F8D820A0F109035842584108BD24
:108AF8001C000020A81D002038B5444D6A68107875
:108B080010F07F0004D1537A23F02003537238BD4C
:108B1800022879D15388002B77D11379002B74D18F
:108B2800537923F08000840004F1804101F5B841B5
:108B380013F0800F096814BF01F0300101F44051AF
:108B4800032861D800295FD0927A002A5CD004F10A
:108B5800804404F5B8441906226825D502F030028D
:108B6800102A4CD103F07F039B0003F1804303F5E7
:108B7800B8431A68510641BF196840F60F720A4097
:108B880042F4004244BF42F0C0021A601A6822F45C
:108B9800E04222F0400292B282F0300242F40042F7
:108BA80042F080021A602AE002F44052B2F5805F77
:108BB80025D128B9164B93F83010FFF75FFF11E065
:108BC8009B0003F1804303F5B8431A68520441BF80
:108BD800196840F60F720A4042F4404244BF42F01E
:108BE80080021A60236823F4804323F070039BB249
:108BF80083F4405343F4004343F080032360AB689D
:108C08005B699847002038BD022038BDA81D0020A8
:108C18001C0000200023036043608360838103619C
:108C280043618361C36103624362836270478A68F8
:108C3800036810B50C6A14430A6914434A6914435B
:108C48008A691443CA6914434A6A14438A6A23F432
:108C5800FF4323F070032243134303608B8943606F
:108C68000B6883604B68C36010BD02684FF6FE73E3
:108C7800134003600023036043608360C360294B93
:108C8800984201D1284A27E0284B984201D1264A28
:108C98002AE0274B984201D1234A2DE0254B9842E0
:108CA80001D1214A30E0244B984201D11E4A33E0D9
:108CB800224B984204D11C4A536843F470032EE0B7
:108CC8001F4B984204D1184A536843F0706326E05A
:108CD8001C4B984204D11C4A536843F00F031EE012
:108CE8001A4B984204D1184A536843F0F00316E02F
:108CF800174B984204D1144A536843F470630EE04A
:108D0800144B984204D1104A536843F4704306E068
:108D1800114B984204D10C4A536843F470235360B2
:108D2800704700BF08000240000002401C000240DB
:108D38003000024044000240580002406C000240EB
:108D48008000024008040240000402401C04024063
:108D5800300402404404024058040240036A23F0ED
:108D680001030362036A70B5446882690D6822F4DE
:108D7800803222F0730215438A8923F002031343D9
:108D88008A881343134A90420FD002F5006290423A
:108D98000BD002F54062904207D002F58062904203
:108DA80003D002F5806290420DD1CA89CE8823F0A3
:108DB800080313430A8A24F4407414434A8A23F0AC
:108DC8000403334314438A68446085614263036241
:108DD80070BD00BF002C01409D4A536803F00C038E
:108DE800042B2DE9F04105D0082B06D099490160E4
:108DF800B3B916E0974B036012E053685468C3F3A5
:108E08008343991CE30349BFD36A934B914C03F006
:108E18000F0344BF0133B4FBF3F34B43036000E09B
:108E2800002351688D4FC1F30311394491F8345030
:108E38000168EDB221FA05F444605668C6F30226CB
:108E48003E4496F8346024FA06FEC0F808E05668F6
:108E5800C6F3C2263E4496F83460F6B2F440C460C5
:108E6800D2F82C80C8F3041808F00F0C07EB4C0C50
:108E780018F0100FBCF844C01FFA8CFC07D0BCF1E6
:108E8800000F04D0B3FBFCFCC0F810C000E0016187
:108E9800D2F82CC0CCF3442C0CF00F0807EB480791
:108EA8001CF0100FB7F84470BFB204D01FB1B3FB69
:108EB800F7F7476100E04161176BFF065ABF654F3E
:108EC80087618161176BBF065ABF624FC761C16175
:108ED800176B7F065ABF5F4F07620162176BFF056A
:108EE80006D5994204D1AE4202D14F00476200E054
:108EF8004462176BFF0406D5994204D1AE4202D1F1
:108F08004F00876200E08462176BBF0506D599425F
:108F180004D1AE4202D14F00C76200E0C462176BB1
:108F28007F0506D5994204D1AE4202D14F0047646D
:108F380000E04464176B3F0506D5994204D1AE4260
:108F480002D14F00876400E08464176BBF0406D524
:108F5800994204D1AE4202D14B00C36400E084645C
:108F6800156B3B4BAD0701D1046315E01C6B04F096
:108F78000304012C01D101630EE01C6B04F003040F
:108F8800022C02D14FF4004305E01B6B03F00303EE
:108F9800032B01D12F4B0363146B2D4B14F4403F6B
:108FA80002D1C0F834E018E01C6B04F44034B4F586
:108FB800803F01D1416310E01C6B04F44034B4F5E8
:108FC800003F02D14FF4004306E01B6B03F440332B
:108FD800B3F5403F01D11F4B4363146B1C4B14F492
:108FE800402F02D1C0F838E018E01C6B04F440248C
:108FF800B4F5802F01D1816310E01C6B04F4402488
:10900800B4F5002F02D14FF4004306E01B6B03F4C4
:109018004023B3F5402F01D10E4B8363146B0C4BE7
:1090280014F4401F02D1C0F83CE021E01C6B04F4AA
:109038004014B4F5801F01D1C16319E01C6B04F41E
:109048004014B4F5001F0BD14FF400430FE000BFEC
:109058000010024000127A0000093D001C000020A8
:109068001B6B03F44013B3F5401F01D1134BC363CB
:10907800126B134B12F4400F03D1C0F840E0BDE867
:10908800F0811A6B02F44002B2F5800F02D101643C
:10909800BDE8F0811A6B02F44002B2F5000F02D16C
:1090A8004FF4004306E01B6B03F44003B3F5400F95
:1090B80001D1024B0364BDE8F08100BF00127A00C1
:1090C80000100240F0B500230E681C460125A5409B
:1090D80005EA060EAE452BD10F797A1E012A15D85E
:1090E800856803229A4025EA020282604D798268E7
:1090F8009D4015438560828892B222EA0E028280E2
:109108008A798588A2402A4392B282800322056820
:109118009A40D2431540056005689F402F43076079
:10912800C7681740CA7902FA03F547EA0502C26020
:109138000134102C03F10203C8D1F0BD38B52DED70
:10914800048B4A4C0368C4F8DC308388A4F8E03008
:10915800013A0D46072A42D8DFE802F0040A10183F
:1091680022292F35B4F8DC300B80B4F8DE3013E058
:10917800B4F8DE300B80B4F8DC3005E0B4F8DC304D
:109188005B420B80B4F8DE305B4205E0B4F8DE30B9
:109198005B420B80B4F8DC306B80B4F8E0301DE043
:1091A800B4F8DC305B420B80B4F8DE3012E0B4F87F
:1091B800DE300B80B4F8DC300CE0B4F8DC300B8027
:1091C800B4F8DE3005E0B4F8DE305B420B80B4F86A
:1091D800DC305B426B80B4F8E0305B42AB80244B00
:1091E80093F86430002B3ED1B5F9003094ED3C0A79
:1091F800D4ED397A09EE103AB5F9023008EE103A92
:10920800B8EEC88AB5F90430B8EEC99A28EE000A53
:1092180008EE903AA7EE890AF8EEE88AD4ED3F7A8C
:10922800A7EEA80A0CF04EFC94ED3D0AD4ED3A7A6C
:10923800288028EE000AA7EE890AD4ED407AA7EE26
:10924800A80A0CF03FFC94ED3E0AD4ED3B7A688006
:1092580028EE000AA7EE890AD4ED417AA7EEA80AFB
:109268000CF030FCA880BDEC048B38BDA81D002094
:109278001C00002008B50A4890F8093100EB4303A8
:109288000A22B3F8181189B2A0F8201100F59470D9
:1092980005F073FA80B208F06DFB024B188008BD28
:1092A800A81D00201C1B0020F8B504460E461746D2
:1092B8000025204620210CF02CFA0446D0B10134B8
:1092C80020460CF08BFAB0F5617F05DB40F63403DD
:1092D8009842A8BF184601E04FF46170A0F561708C
:1092E800192390FBF3F00DB9307000E070703B78F3
:1092F80001333B700DB90125DBE72046F8BD30B5D9
:1093080005460C461346294622460248BDE8304029
:1093180001F005BE189F01087FB504780646E4B938
:10932800354B1B6803EB8403192193F87B0093F8F2
:109338007C6093F8792093F87A304FF4617511FBCB
:10934800005011FB0651009001912C482146013430
:1093580001F0E5FD142CE3D14BE00CF03FFA1328A3
:10936800054641DC244B701C1C68202100238DF825
:109378000F300CF0CEF91E35064670B10136304676
:109388000CF02CFA1A289FBF04EB850358709DF83F
:109398000F30013398BF8DF80F30304620210CF084
:1093A800B8F9064670B1013630460CF017FA0D28A8
:1093B8009FBF04EB850398709DF80F30013398BF69
:1093C8008DF80F3004EB85043046E11C0DF10F02D7
:1093D800FFF76AFF9DF80F30042B0AD0601C0021AC
:1093E80004220CF060F904E0054800211322FFF77D
:1093F80086FF04B070BD00BF98120020379F010897
:109408004C9F0108014806F09BBE00BF529F01080F
:10941800F8B50478064674B9304DB5F8C621B5F8E4
:10942800C8312F482146013401F079FD042C05F19B
:109438000405F2D1F8BD2B490CF03EF9A8B9274B29
:109448004FF47A714FF4FA62A3F8C611A3F8C82151
:10945800A3F8CA11A3F8CC21A3F8CE11A3F8D02100
:10946800A3F8D211A3F8D421F8BD30460CF0B6F910
:10947800032805462BD8304620210CF04AF904462B
:1094880030B1013420460CF0A9F90126074600E066
:109498000646204620210CF03CF910B9BDE8F840FA
:1094A800B0E701300CF09AF9012EF7D1A7F2EE22BD
:1094B80040F2DC539A42F1D8A0F2EE229A42EDD85B
:1094C800064B703503EB8503DF801881F8BD06482D
:1094D80000210322BDE8F84011E700BF4413002033
:1094E800609F0108739F0108B5AC01082DE9FF4191
:1094F80004780546002C39D17348744D06F020FED7
:10950800D5ED057AF5EE407AF1EE10FA00F0D88044
:1095180021466F4801F003FD95ED050A684601F004
:1095280093FB01466B4801F0FAFC95ED060A684684
:1095380001F08AFB0146674801F0F1FC95ED070A46
:10954800684601F081FB0146624801F0E8FC95EDB0
:10955800080A684601F078FB013401465E4801F0CC
:10956800DEFC0C2C05F11005CAD1A9E05B490522E7
:109578000CF0E6F840B9554B03F1C00200215961DF
:1095880010339342FAD19BE02846554904220CF047
:10959800D7F804462846002C40D120210CF0B9F811
:1095A800002800F08D80451C28460CF0C0F80746BE
:1095B8004C4B53F824601EB94B4806F0C1FD7FE0C0
:1095C80028463146FAB20CF0BBF801340028EFD136
:1095D8003E4B03F1C0029E4600215961103393426D
:1095E800FAD1424B03EBC4029846D2F804C0BCF14E
:1095F800000F04D131463E4801F091FC57E00027A6
:1096080018F834309F42F5DA3B010EEB030563444A
:109618000FCB143585E80F000137F1E70CF0DEF8C1
:109628000B28064647DC284620210CF072F8054630
:1096380050B10135284601F07DFA244B03EB06139F
:1096480083ED050A012400E00446284620210CF099
:1096580060F8054648B10135284601F06BFA1B4B06
:1096680003EB061383ED060A0134284620210CF08B
:1096780050F8054648B10135284601F05BFA134B0E
:1096880003EB061383ED070A0134284620210CF06A
:1096980040F810B9FFF7B6FE12E0013001F04AFABF
:1096A8000A4B032C03EB061686ED080AF2D1114883
:1096B800FFF71CFF04E0104801210C22FFF71FFEF2
:1096C80004B0BDE8F08100BF799F01084413002071
:1096D800949F01089A9F0108C9A90108739F01086E
:1096E8009E9F0108E0980108A39F0108489E010871
:1096F800B29F0108D79C01084C9F0108F0B5047877
:1097080087B006461CBB514B1968062303FB04119E
:10971800192091F8CA5091F8CB7091F8CE2091F8A1
:10972800C9304FF4617610FB056510FB07600095A2
:10973800019091F8CC000290C831454849790391CD
:109748002146013401F0EBFB0C2CDCD17CE00CF061
:1097580045F80B28044672DC3C4B701C1D68202120
:1097680000238DF817300BF0D4FF064680B1013680
:1097780030460CF033F803289FBF062303FB04533D
:1097880083F8CE009DF817309CBF01338DF8173051
:10979800304620210BF0BDFF074680B1013738461F
:1097A8000CF01CF80D289FBF062303FB045383F815
:1097B800C9009DF817309CBF01338DF81730062675
:1097C8006643A9193846CA310DF11702FFF76CFD37
:1097D80020210BF09EFF074670B1013738460BF089
:1097E800FDFF14289FBF9DF817307619013386F8BE
:1097F800CC0098BF8DF81730384620210BF089FF30
:1098080078B101300BF0EAFF0D289FBF062303FB58
:10981800045383F8CD009DF817309CBF01338DF8B1
:1098280017309DF81730062B0ED0062202FB045085
:109838000021C9300BF037FFFFF7E4FD04E00548CD
:1098480000210B22FFF75BFD07B0F0BD9812002046
:10985800BE9F01084C9F01082DE9F347047806468E
:109868004CB9204601A9FEF7E7FF0134FFF7F4FFE2
:10987800122CF6D17BE00BF0B1FFC5B2112D71D8D7
:109888003C4C05F1D00704EB4703701C202193F8EA
:109898000280394E0BF03DFF034630B9A8F10202B1
:1098A800D2F1000848EB020845E000F1010A5978B6
:1098B80030460BF02EFF60B1032D8CBF032300232D
:1098C800801B334453FA80F090F80490B9F1030FE9
:1098D80002D1FFF797FD4AE0A9F10203D3F100088E
:1098E80050464FF0200148EB03080BF012FFD8B1A7
:1098F800B8F1000FEDD001300BF070FF40F2ED230E
:1099080080B2984205DD40F6CA039842A8BF1846BF
:1099180001E040F2EE2004EB4703A0F2EE2019220A
:1099280090FBF2F0D87002E0B8F1000FD1D104EB4F
:10993800470383F8029004EB4704A378F25CB8F17C
:10994800000F0AD0E3780D48294640F2EE24192585
:1099580005FB034301F0E3FA09E02946084801F052
:10996800DEFA04E0074800211122FFF7C8FC02B024
:10997800BDE8F08744130020447E0108DE9F0108FB
:10998800F09F0108B5AC010810B50446204604F064
:10999800E5FE18B90A2004F01AFEF7E710BD0C4BD3
:1099A8005A6882421A4607D01B69834206D0D36997
:1099B80083420BD1022302E0002300E001230021AF
:1099C800C1620C2000FB032319725960704700BF65
:1099D8005C1E00202DE9F04F06468A4890F90040A9
:1099E80087B0B44288469DF8445011461A469DF8FF
:1099F800403009D090F90C40B44207D090F9184093
:109A0800B44209D1022702E0002700E001270C2414
:109A180004FB0700047A0CB10020EFE0012E00F0EF
:109A2800DC80142E05D0002E40F0E78000957648A3
:109A3800D5E0DFF814A2DAF8183043F00103CAF8C9
:109A48001830DAF814304FF0904543F40033CAF870
:109A580014304FF0010903224FF4805B04A94FF042
:109A680090408DF815200392CDF810B08DF8149021
:109A78008DF816908DF81740FFF724FBA5F828B04D
:109A8800C82004F0A4FDC5F818B0DAF81430039A19
:109A980043F40033CAF8143028464FF4C0534FF04B
:109AA800020B04A904938DF815208DF814B08DF8D5
:109AB80016408DF81740FFF705FB6B6A23F47043D7
:109AC8006B626B6A43F460436B626B6A23F47023C6
:109AD8006B626B6A43F460236B624C4B4C4D4FF4E2
:109AE80080221A6002F18042A2F53F3212232B63D2
:109AF800082385F83530136885F8369023F48023D9
:109B08001360536823F48023536095F8343003F1CD
:109B1800804303F582331A6842F480221A602A6B64
:109B28003C4B22F01F0002F01F02C15809FA02F252
:109B380021EA0202C2502A6B374922F01F0002F0C4
:109B48001F0250F801E009FA02F22EEA020242501E
:109B58002A6B22F01F0102F01F02C85809FA02F20C
:109B68000243CA502D4B2E4A1C60DAF81C3043F4CD
:109B78000003CAF81C302B4B04A8DA608DF810607B
:109B88008DF811B08DF812408DF8139007F0CCF8CD
:109B98002A238DF810309DF813308DF811908DF828
:109BA80012401BB104A807F0BFF804E01E4B4FF4A5
:109BB8008062C3F884201D4B1D4C1C60022385F86D
:109BC80040301C4A1C4B1D496B6511601B68984747
:109BD8001B4B2B60A4F1380006E01A48009502F0F0
:109BE80097FE00283FF418AF064B06710C2202FBC3
:109BF800073787F80880786000E0204607B0BDE89E
:109C0800F08F00BF5C1E00200038014014040140A2
:109C1800581F0020080401400C040140D8004242AB
:109C28000005FA0500ED00E000E100E0AC1D0020B1
:109C3800901F0020B01D002020000020840000207C
:109C4800507E010800440040001002400C4B1B6885
:109C580093F90220824209D093F90A20824207D060
:109C680093F91220824208D1022002E0002000E08D
:109C7800012003EBC000023070470020704700BF8E
:109C8800581E0020F0B5027887B0AAB94C4C04F1F0
:109C980018064C4B94F9F61193F900208A4273D0B8
:109CA80093F90C208A426FD093F918308B426BD00D
:109CB8000834B442EDD181E0002204920592451C9B
:109CC8000BF08CFDC4B260B2FFF7C0FF074618B1B5
:109CD8008DF81040012400E00446284620210BF0AE
:109CE80018FD054638B1013528460BF077FD0134DB
:109CF800ADF81200E4B20026284620210BF009FD39
:109D0800B0B3451C28460BF069FD00222E4951F8D6
:109D1800223083425FFA82FE04D00132082AF5D14C
:109D2800002300E0734651F82320824220D1022EFE
:109D38000FD0032E12D05A1E012ED2B204D0042AFC
:109D480013D88DF814300EE0042A0ED88DF815308B
:109D580009E0052B09D88DF8173004E09A1E052A6A
:109D680003D88DF816300134E4B20136042EC3D17D
:109D7800052C04D807B0BDE8F040FFF743BB04AB9F
:109D880003CB3860796019E094F8FB010E4B94F826
:109D9800FA5153F82000B4F8F821009094F8FD0126
:109DA80053F82000019094F8FC0153F82000029029
:109DB80053F82530054801F0B2F879E707B0F0BD4F
:109DC800441300205C1E0020207E0108FF9F01082C
:109DD80038B1438811EA030003D08B420CBF01203D
:109DE8000220704730B50B4B0B491C6891F858207E
:109DF800022A0BD8134604EBC303551CEAB29D880C
:109E08002842F5D081F85820981C30BD81F8582098
:109E1800002030BD581E0020581F0020024B002291
:109E280083F85820DEE700BF581F00202DE9F047CF
:109E3800877890F803C0214DBBB2C7F1640E03EBDD
:109E480083065C42C3F178005FFA8EFE7600CCF19F
:109E58006408A4B280B2A3B20FFA83F9B9F1000F73
:109E680005DC002B14BFBA464FF0010A00E0F246A9
:109E780013FB03F303FB0CF21AFB0AF392FBF3F355
:109E8800434403FB09F30A2293FBF2F333449BB2E6
:109E980025F8023FB1F800904A880A34C9EB020A53
:109EA800A4B21AB202FB0AF24FF47A73844292FB0C
:109EB800F3F34B442B80CED1BDE8F087B01F0020D0
:109EC8002E4B2F4A1B68126810B51A602D4A11686C
:109ED800596051689268DA602B4A99601168196173
:109EE800516892689A61294A59611168D961516823
:109EF80092685A62264A19621188198551885985CB
:109F08009188D288DA85234A9985118819865188DB
:109F1800598692889A86204A1188D9865188198745
:109F28001946928821F83A2F1C4A1078002282425A
:109F380006DA1B4C34F8124021F8024F0132F6E7DA
:109F4800184A1288A3F86420174A1288A3F86620D2
:109F5800164A1188A3F86C1051889288A3F87020CB
:109F6800134AA3F86E1012689A66124A1288A3F868
:109F78007220114A5289A3F85E2010BDFC290020E6
:109F8800D82D0020DC250020E8250020F42500201D
:109F98003C1300207C1200202613002058260020A5
:109FA8009C120020C81E00203411002082120020BC
:109FB80030130020B8120020881200202DE9F84341
:109FC8000E4B93E8800305460E460024B44213DA8C
:109FD8007B1933F9140008EB050333F9142009EB56
:109FE800050333F914301344022293FBF2F3C01A29
:109FF80006F06BFE0134E9E7BDE8F883FC29002090
:10A0080070B5472006F0B0FD174B1B681B0307D53A
:10A01800164B174A5B6810681B68C01A06F046FEA4
:10A02800144E154C154D307806F040FE236828680C
:10A03800C01A06F04AFE63686868C01A06F045FE52
:10A048000F4B188806F032FE0E4B188806F02EFECD
:10A058000D4B188806F02AFE337823742B68A3600A
:10A068006B68E36070BD00BF682B0020FC290020EE
:10A07800D82D0020361B0020E8290020381B00209E
:10A08800341B0020321B0020C01200207FB5264C54
:10A09800264E274D2749284A284B20B128480088B2
:10A0A800B0F5805F31D23088ADF8040028781E4DB5
:10A0B80091F8201012788DF806008DF807108DF8A9
:10A0C80008201B788DF8093001A8294606220BF0D4
:10A0D800CFFA30B30198BDF808302860AB80532020
:10A0E80006F042FD208806F0E1FDA07806F0DEFDCE
:10A0F800E37801932379029301A86379039306F027
:10A108003BFD0F4B00221A800BE03088208091F82D
:10A118002010287812781B78A070E1702271637182
:10A12800DDE704B070BD00BFCC1F0020F41B002089
:10A13800301B0020602D0020AB0F002010100020E5
:10A14800882B0020A0F17D03012B70B504460D4635
:10A158000A4E05D830687D2104F00CFB84F02004F9
:10A168003068214604F006FB35B12B881C4404EB0B
:10A17800142404F0FF042C8070BD00BFE41B0020F1
:10A188000A4A138801331380094A1368013313609C
:10A19800084A138801339BB2202B01BF0023138088
:10A1A800054A138808BF013313807047882B0020A5
:10A1B800702B0020742B0020762B002038B53A4BEA
:10A1C8001B78083B012B05460C466BD8452006F04A
:10A1D800CBFC284606F0C8FC0C2D23D004D80A2D49
:10A1E8000AD014D835B138BD0E2D4BD02ED3FF2D43
:10A1F80050D038BD206849E0207806F0B5FC627977
:10A208006378002A14BF80200020184300E02078DB
:10A2180006F0AAFCA07806F0A7FCE07806F0A4FCFB
:10A2280020793BE0B4F9000006F036FDA07806F08E
:10A238009BFCE07806F098FCB4F9040006F02CFDCD
:10A24800B4F90600BDE8384006F026BD63782078EA
:10A258008BB180F0800006F087FCA468E0B206F0BD
:10A2680083FCC4F3072006F07FFCC4F3074006F024
:10A278007BFC200E12E006F077FC6068BDE83840F1
:10A2880006F023BD206806F011FD6068BDE838407F
:10A2980006F00CBD054806F045FC0020BDE8384036
:10A2A80006F062BC38BD00BFD82900201EA00108F6
:10A2B8002DE9F04FB74BB84F1A888BB00193002A9D
:10A2C80040F0A380B7F8CE07B44E42F20103C21A99
:10A2D80050425041FFF7DAFEFFF7F2FD346849209B
:10A2E80006F042FCAE4B2546186806F0DFFC55F830
:10A2F800040B06F0DBFC2846FEF7ECF904F110002D
:10A30800FEF7E8F904F11C094FF01008A54D0123E8
:10A318002A6803FA08F3134203D0D9F8000006F0BC
:10A32800D4FC08F10108B8F1130F09F10409EDD1C3
:10A3380004F12800FEF7BEF9B7F84431B4F92E004D
:10A34800C01A06F0B3FC2B68DB0408D5964BB4F8AA
:10A3580064001B88181AC0F30D0006F0A7FC2B68D0
:10A36800980403D5B4F8660006F0A0FC2B685905DC
:10A3780003D504F16C00FEF79DF92B681A0502D588
:10A38800A06E06F0A2FC2B681B0403D5B4F872007B
:10A3980006F08CFC04F13000A046FEF78BF904F1BE
:10A3A8003600FEF787F9B7F8443138F93C0FC01A80
:10A3B80006F07CFC01277D4B1B789F4208DA38F9B0
:10A3C800020FB4F93C30C01A06F07FFC0137F2E7FF
:10A3D8002B68980505D5B4F95E00A0F2DC5006F0AC
:10A3E80074FC326872487260B260121A9110714A35
:10A3F8004A43531C032293FBF2F202EB42029A1ADD
:10A40800742303FB02033360C9E16B4B6B4A1B687F
:10A4180011688B4206D00AA9002041F8203D13603C
:10A42800FFF7CCFE019B97F8CE171B8897F8CF074C
:10A438000B44013BB3FBF0F200FB12338B4280F07C
:10A448007981564C0120FFF721FEFFF739FD502096
:10A458002668656806F088FBA268236810681B6890
:10A46800626803441068A3EB400006F02EFC6A689B
:10A4780073689B1A0293AA68B3689B1A0393EA68E5
:10A48800F36802A89B1A0493FEF724F92A69336932
:10A498009B1A02936A6973699B1A0393B369AA6941
:10A4A80002A89B1A049306F067FB06F11C0905F144
:10A4B8001C0B1027A0463B4801210368B9401942EC
:10A4C800824606D0D9F80000DBF80030C01A06F042
:10A4D800FCFB0137132F09F104090BF1040BEAD136
:10A4E80006F1260005F12601002331F9024F30F963
:10A4F800022F121B02AC44F823200133042BF4D1A1
:10A508000322002702ABBF0053F82230FFB26BB121
:10A5180003F108010F2902D847F0010706E080334C
:10A52800FF2B94BF47F0020747F0030712F1FF32F1
:10A53800E8D2384606F018FB00240DF10809A346B6
:10A5480007F00302022A10D0032A17D0012A4AD1A1
:10A55800BBF1000F41D0D9F8000000F00F002043F4
:10A5680006F002FB4FF0000B3DE0BBF1000F0CD0F2
:10A57800D9F80000C0F3031020432CE0BBF1000F12
:10A588001ED199F8010006F0EFFA99F8000006F0DC
:10A59800EBFA28E0742B002044130020FC2900204B
:10A5A800702B0020682B0020642B002058260020E8
:10A5B800082A002035C2724F7C2B0020782B0020FF
:10A5C800D9F80000C0F30330204306F0CDFAD9F8DB
:10A5D8000000C0F3071006F0C7FAD9F800402401BC
:10A5E800E4B24FF0010B09F1040906AB99454FEAB3
:10A5F8009707A5D1BBF1010F02D1204606F0B4FAA6
:10A60800DAF8003013F480541FBFB6F86420B5F8A8
:10A618006410521A029218BF012499040AD50AAA92
:10A6280002EB8401B5F86600B6F86620121A41F804
:10A63800202C01345A0513D502AA02EB840E06F128
:10A648006A0705F16A00002237F9021F30F902CFC4
:10A65800CCEB01014EF822100132032AF4D1033465
:10A668001F0508D50AAA02EB8400A96EB26E521A19
:10A6780040F8202C013418040BD50AAB03EB8402F4
:10A68800B5F87210B6F872305B1A42F8203C013403
:10A6980000E0F4B1012C03D1029806F016FB18E093
:10A6A800631E002002AA400052F82320C0B20AB15B
:10A6B80040F0010013F1FF33F4D206F055FA0027F9
:10A6C80002AB53F8270008B106F0FFFA0137A7429A
:10A6D800F6DB30200321FFF771FC36200321FFF75A
:10A6E8006DFC314B3C201978FFF768FCDAF8003034
:10A6F800990506D5B6F95E00B5F95E30C01A06F0C0
:10A70800E4FAD8F800202948D8F80430C8F804201A
:10A71800121A9110264AC8F808304A43531C0322DB
:10A7280093FBF2F202EB42029A1A742303FB020330
:10A73800C8F800301F4B1B681A0630D51E4C1F4D39
:10A7480022682B689A420BD162686B689A4207D1DB
:10A75800019B1B88102B11D1194B1B885B060DD14F
:10A76800482006F001FA206806F0AFFA606806F0A3
:10A77800ACFA23682B6063686B600EE0114A0F4BDC
:10A7880011782A7C914208D10F4A9968106888424A
:10A7980003D15268DB689A4201D0FFF731FC06F01A
:10A7A800B3F90BB0BDE8F08F58260020082A002026
:10A7B80035C2724F98290020C4120020E8290020D1
:10A7C800762B0020361B0020381B00202DE9F84F7F
:10A7D8000C9E3A4CC2EB030B0B9BF61A63680029DC
:10A7E80014BF4FF0060A4FF0040A0133054690469D
:10A7F80013D1236853455ED2314A324852F8232098
:10A80800032B98BF294606F09DF9636801336360FE
:10A818002D4B002205469A7113E0002511E02B4AC2
:10A828001278954240DA0B9BE3B109FB06F2995C7A
:10A8380001228A40264909680A4213D16368013314
:10A848006360D4F804900A9B1C4F9945E7DB2BD131
:10A858000A2006F089F93B6801333B604FF0FF336B
:10A868007B6021E0184A917921B12C2006F07CF90F
:10A87800013501E001219171226809FB0BF308EB16
:10A88800030752B958F8030006F04CF997F9041079
:10A898004B1C0544D2D00F4802E03A440E481179C7
:10A8A80006F050F90544C9E7206850452CBF002040
:10A8B8000120BDE8F88F0020BDE8F88F802B00202C
:10A8C8002883010829A00108CC1F002014010020BA
:10A8D800682B002038A00108E1A9010830B585B02F
:10A8E80004AC002524F8025D0091ADF8060021466D
:10A8F8001020FFF727FC9DF806002146FFF722FCF1
:10A908009DF807002146FFF71DFC9DF80000214631
:10A91800FFF718FC9DF801002146FFF713FC9DF88E
:10A9280002002146FFF70EFC9DF803002146FFF7C1
:10A9380009FC9DF80E00C043C0B22946FFF702FC8F
:10A9480005B030BD10B5054C206803F010FF18B1F4
:10A95800206803F009FFF6E710BD00BFB41B002014
:10A9680013B5044601A9006807F0D6F8132007F0CC
:10A978000FF9BDF9040007F0F9F81B2007F008F9F2
:10A98800BDF9060007F0F2F8232007F001F9236863
:10A99800002BB4BF53204E2007F0E8F801A96068E7
:10A9A80007F0BAF8122007F0F3F8BDF9040007F031
:10A9B800DDF81A2007F0ECF8BDF9060007F0D6F824
:10A9C800222007F0E5F86368002BB4BF5720452024
:10A9D80007F0CCF802B010BDF0B50124B0FBF4F5D7
:10A9E8008D4201D34C43F9E70026D4B1B0FBF4F50E
:10A9F80004FB1500B4FBF1F41EB9002D01DC002C9A
:10AA0800F3D1092D03F1010EEFB204DD002A14BFC2
:10AA18003725572500E030253D441D700136734623
:10AA2800E3E71C70F0BDF0B50124B0FBF4F58D42EE
:10AA380001D34C43F9E70026D4B1B0FBF4F504FB8D
:10AA48001500B4FBF1F41EB9002D01DC002CF3D184
:10AA5800092D03F1010EEFB204DD002A14BF3725DA
:10AA6800572500E030253D441D7001367346E3E765
:10AA78001C70F0BD03685A1C0260197070472DE9FC
:10AA8800F843089E002B07468846144614BF4FF02B
:10AA980030094FF02009334613F8012B0AB925462F
:10AAA80003E0002CFBDD013CF6E7002D04DD384611
:10AAB8004946C047013DF8E724EAE4743546A01B3F
:10AAC800284415F8011B11B13846C047F7E7BDE81F
:10AAD800F883024B186803F04DBE00BF40110020F8
:10AAE80090ED017A07EE901AB5EE407AF1EE10FA81
:10AAF80001BFF8EEE77A9FED0E7A67EE877AB7EE38
:10AB0800007A04BFC7EE277AC0ED017A90ED017A8A
:10AB1800D0ED007A30EE877A30EE670AC0EE870A09
:10AB2800E0EE807AB0EE670AC0ED007A704700BFA9
:10AB3800DB0FC94010B50278202A034600F1010056
:10AB4800F9D0092AF7D02D2A03D10346BFEE000A0F
:10AB580004E02B2A08BF0346B7EE000ADFED387A77
:10AB68001A46134612F8010BA0F13001CCB2092C99
:10AB78000AD807EE101AB8EEC77AF2EE046AA7EE02
:10AB8800A67AF0EE477AECE72E2816D1F2EE046AA0
:10AB98001146B0EE666A0B4611F8012B303AD0B276
:10ABA80009280AD807EE102AB8EEC77A87EE267A5F
:10ABB80066EE866A77EE877AEDE71A7802F0DF02AA
:10ABC800452A35D15A782D2A02D10233012004E0D2
:10ABD8002B2A14BF013302330020013B002213F853
:10ABE800011F3039CCB2092C03D80A2404FB021205
:10ABF800F5E7B2F59A7F28BF4FF49A721346B7EE7D
:10AC0800007A072B05D9DFED0F6A083B27EE267A75
:10AC1800F7E702F007032BB1F2EE046A27EE267A73
:10AC2800013BF8E7F0EE476A20B1C7EE877A03E008
:10AC3800F7EE006A67EEA67A20EE270A10BD00BF7D
:10AC48000000000020BCBE4C30B52DED028B87B053
:10AC5800B0EE408A0C220021054603A80AF023FD25
:10AC6800B5EEC08ADFED2A7AF1EE10FACCBF38EEE5
:10AC7800278A38EE678ADFED277A28EE278A694621
:10AC8800FDEEC87A17EE904A84EAE470A0EBE4700F
:10AC9800FDF7D2FD002CACBF20232D2368468DF88C
:10ACA8000C300AF044FD012807D130238DF80D300F
:10ACB8008DF80E308DF80F300CE0022805D13023C6
:10ACC8008DF80D308DF80E3004E0032804BF3023D2
:10ACD8008DF80D30694603A80AF00CFD03A80AF0A8
:10ACE80026FD0338C4B2224603A928460AF04CFDC3
:10ACF80000232B55284608490AF0FCFC03AB2846DC
:10AD080019190AF0F7FC284607B0BDEC028B30BDD4
:10AD18006F12033A00007A445CA0010870B5064639
:10AD280015460846B6FBF2F414B12046FFF7F6FFC5
:10AD380005FB1464024B1B5D00F8013B70BD00BFAE
:10AD48005EA001082DE9F04F814689B08A46164673
:10AD58001C4600253178002900F0DD80252902D025
:10AD68000136484675E07278302A08BFB278A2F1F9
:10AD7800300319BFB71C4FF0000BF71C4FF0010B45
:10AD8800092B4FF0000819D8A2F13003D9B20929CC
:10AD980005D80A2202FB083817F8012BF4E7A2F1BC
:10ADA8006103052B02D8A2F1570305E0A2F1410384
:10ADB800052B03D8A2F137030A2BEADD6C2A31D11F
:10ADC8003A78642A07F1010600F083800BD8252A17
:10ADD8003DD003D8002A00F09E80BBE7582A0CD04B
:10ADE800632A19D0B6E7732A22D002D86E2A37D040
:10ADF800B0E7752A5CD0782AACD1271D2068A2F16B
:10AE0800580462424FF01001624155E02CD9582A8B
:10AE180032D0632A2AD13E4648462178271DD0479A
:10AE280001350FE0642A64D00ED9732A14D13E4646
:10AE3800236800934846514642460023FFF71FFE09
:10AE4800271D05443C4685E7252ADFD13E4648466E
:10AE58002521D04701357DE70AD86E2A06D13E461E
:10AE6800236804341D6075E7002A54D03E4671E714
:10AE7800752A26D0782AF9D1A2F1580304F1040CD6
:10AE88005A422068CDF80CC04FF010015A4105AB6A
:10AE9800FFF7A2FDDDF80CC03E46644605AB009303
:10AEA8004846514642465B46FFF7E9FD054451E7EF
:10AEB8002068271D0A21002205ABFFF7B4FD3C4698
:10AEC800ECE704F1040CCDF80CC020680A2100223C
:10AED800DDE72068002804F1040708DA2D238DF83F
:10AEE800143040420DF115030A210022E5E705ABB5
:10AEF800FAE72068002804F1040C0ADA2D238DF8FB
:10AF0800143040420DF11503CDF80CC00A2100227F
:10AF1800BEE705ABF8E7284609B0BDE8F08F0FB4E7
:10AF280013B50B4904AB08680A4953F8042B0968A0
:10AF38000193FFF707FF0446074B186803F00EFC60
:10AF48000028F9D0204602B0BDE8104004B0704790
:10AF58008C010020880100204011002080EAE07365
:10AF6800A3EBE0738B4206DB002801DD401A704733
:10AF780002D00844704700207047FDEEC07A17EEF3
:10AF8800903A2033402B43D8DFED237AB4EEE70A1A
:10AF9800F1EE10FA04DDDFED217A30EE670AF3E70F
:10AFA800DFED1F7AB4EEE70AF1EE10FA04D5DFED13
:10AFB8001B7A30EE270AF3E7DFED1A7AB4EEE70AD8
:10AFC800F1EE10FA04DD30EE670A37EEC00A0AE047
:10AFD8009FED157AB4EEC70AF1EE10FA44BF30EED1
:10AFE800270A37EE400A60EE007ADFED106A9FED1F
:10AFF800107AA7EEA67ADFED0F6AE7EE876A9FED73
:10B008000E7AA7EEA67A20EE276AA6EE070A704700
:10B018009FED0A0A704700BFDB0F4940DB0FC940AC
:10B02800DB0F49C0DB0FC93FDB0FC9BF9A7C2E3647
:10B03800FAAF4FB93587083CA4AA2ABE0000000021
:10B04800DFED027A30EE270A97E700BFDB0FC93F32
:10B0580038B52DED068B90ED008AB0EE480A0C4607
:10B068000546FFF7EDFFB0EE40AAB0EE480AFFF73D
:10B0780084FFD5ED018AB0EE409AB0EE680AFFF77A
:10B08800DFFFB0EE408AB0EE680AFFF776FFD5ED35
:10B0980002AAF0EE408AB0EE6A0AFFF7D1FFF0EE9E
:10B0A800409AB0EE6A0AFFF768FF60EE0A6A69EE36
:10B0B800297AF0EE665AE7EEA85A29EE8A6A29EE4E
:10B0C800007A69EE889A29EE489A28EE400A28EE16
:10B0D8000A8AC4ED035AF0EE465AE7EE685AE6EEDD
:10B0E800A87AA6EE687AC4ED009AC4ED028A84EDC7
:10B0F800059A84ED088ABDEC068B84ED010AC4ED3F
:10B10800045A84ED067AC4ED077A38BD10B52DEDE2
:10B11800048B8AB090ED009AD0ED028A90ED018AF6
:10B128000446084601A9FFF793FFDDED047A9DED7B
:10B13800017A68EE277AE9EE077A9DED077AE8EE5C
:10B14800877A9DED027AC4ED007ADDED057A68EE26
:10B15800277AE9EE077A9DED087AE8EE877AC4ED5A
:10B16800017ADDED067A28EE278ADDED037AA9EE6D
:10B17800278ADDED097AA8EEA78A84ED028A0AB04B
:10B18800BDEC048B10BD074B1A8822EA00009042E0
:10B1980010B518801C4602D0012003F075FA2088EB
:10B1A80010BD00BFF41B0020064B1A8810439042C4
:10B1B80010B518801C4602D0012003F065FA2088DB
:10B1C80010BD00BFF41B0020024A936823EA000068
:10B1D800906070474413002008B5104B1A7800237C
:10B1E800D9B2914207D20E4951F8231009680020BC
:10B1F80008600133F4E7322003F0E9F9094B1B68D2
:10B208005A0309D5084B9B685B0305D440F2DC5010
:10B21800BDE8084003F0DBB908BD00BF5826002090
:10B228002826002098290020441300202DE9F34106
:10B2380006F0F6FB454A6923137040F2D473538035
:10B24800BE231371EF2382F8D137002382F8D23757
:10B2580019461646F25C0133514040F2D4729342CB
:10B26800F8D13A4B83F8D217394B1A69120604D52C
:10B27800384A5A6002F188325A6004270020013F98
:10B2880017F0FF0750D0324B3422DA60002444B163
:10B29800002356F804800193FDF79EFA0428EED1A6
:10B2A80017E0FDF799FA0428E9D1294D2B6943F0F5
:10B2B80002032B61284B6B612B6943F040032B6120
:10B2C800FDF78AFA2B69042823F002032B61DFD0EB
:10B2D800D5E71F4D2B6943F001032B6104F100638F
:10B2E80003F57E331FFA88F21A80FDF775FA0428F1
:10B2F80010D11A4B23440193019B4FEA1848A3F835
:10B308000080FDF769FA2B69042823F001032B61FB
:10B3180005D0B4E72B6923F001032B61AFE70434B0
:10B3280040F2D4739C42B2D1094A1369042843F00D
:10B338008003136102D105F019F910B9052003F053
:10B34800BBF906F057FB02B0BDE8F08144130020BA
:10B35800002002402301674500F8030802F80308AB
:10B3680010B50E4C206803F075F82068047A0022A6
:10B3780002FB02F3193B634303F6C4135343192139
:10B3880093FBF1F3064921F812300132072AEFD175
:10B398000449BDE81040FEF749BD00BFBC120020BB
:10B3A80010110020881400202DE9F04105F0DEF886
:10B3B80010B9042003F080F9B14CB24D06F030FB0F
:10B3C800B14940F2D47220460AF062F994F8A837DD
:10B3D800022B84BF002384F8A83794F8A8274FF4D9
:10B3E800CC7101FB02F303F5387023442044286034
:10B3F80093F8340303F54C73022801FB024284BF1F
:10B408000020187192F83433A04A13700C2202FB02
:10B4180003439F4A03F2AA731360A36846F2090222
:10B428001A401AB9964A43F400539360A368D807A0
:10B4380003D54FF40050FFF7C7FEA368590409D598
:10B448000820FFF7C1FE4FF40050FFF7BDFE0120B2
:10B45800FFF7BAFEA3681A0706D54FF40050FFF7A6
:10B46800B3FE0120FFF7B0FEA3689B0406D54FF496
:10B478008030FFF7A9FE4020FFF7A6FE012284F8DE
:10B48800112294F8E0217E4B2AB193F8E42112B1FD
:10B49800002283F8E4217F4B7F4E1E604FF0000CA2
:10B4A800674604EB0C03B3F8F8E14FEA5E0101F0DC
:10B4B80077314FEA9E0303F03333C1EB0E00C11A14
:10B4C8004FEADE0303F01133CB1A03EB23131EF00C
:10B4D800010803F00F324FF0FF0392FBF3F3C3EBC5
:10B4E800032318BF0137A2EB030318BFFFB2012BD8
:10B4F8000ADD022B40F0C180B8F1000F00F0BD80DA
:10B508001EF0BC0F00F0B9800CF1080CBCF1180F4C
:10B51800C7D1013F012F00F2B080FFF721FF302291
:10B5280000215E485E4F0AF0BEF85E4BD5F80080F9
:10B538001F605D4B002108F17900C3F8008002F01C
:10B54800C9FF5A4B80F001001870594B07F12602C9
:10B558001A60584B07F1CC021A6098F8000003F003
:10B5680045FB2868544B00F5C5721A60FCF734FF98
:10B57800524B94F8D801DFED526A07F194021A6031
:10B588006421504BC82211FB00225A6000229A60A5
:10B59800DA601A615A619A61DA6183F8202083F8C7
:10B5A8002120494B07F12C021A602B68474A93ED7A
:10B5B800187A03F219111160454A03F289111160D2
:10B5C800444A07F108011160434A1760434A07F1EA
:10B5D800A0011160424A07F1AA011160414967EED2
:10B5E800266A0E60B4F86611B6EE007A07EE901A75
:10B5F80087EE267AB4F86811101DF8EE677AC2ED66
:10B60800027A07EE901A93F85C10117193F878108B
:10B61800517194F8E3111174F8EE677AB3F81611C2
:10B62800C2ED037A07EE901A2F49086053612F4A3A
:10B6380003F1640111602E4A2E4982ED007AF8EE7A
:10B64800E77A9FED2D7A2D4A0B60C7EE277A2C49B1
:10B658009FED2C7A67EE877AC2ED007A03F16802D3
:10B668000A60294903F211130B60284B1F60284B0D
:10B67800BDE8F0411A6006F0BDB9FDF779F84CE76E
:10B68800441300209812002000F8030844290020E1
:10B69800BC120020542D0020CE140020441000209D
:10B6A80088140020781000207C100020140000204E
:10B6B800540800208806002088100020C82D00208B
:10B6C800DB0F4940602D0020AC0800202C20002012
:10B6D800B40A00209C270020A0270020C8090020C9
:10B6E800D41F00208C0A0020DC0800201409002048
:10B6F800100900202408002000006144C40900202B
:10B70800180800204C3D0F44B4090020BC09002053
:10B718001407002008B5FFF789FDFFF745FE012053
:10B72800BDE8084002F0B0BF38B500240B4D6059A1
:10B73800254404F005FD696811B10948FFF7EFFBDE
:10B74800A96811B10748FFF7EAFB0748103404F06D
:10B75800F7FCB4F5D87FE9D138BD00BF40830108B4
:10B7680083A0010889A0010887AA0108F0B585B05F
:10B77800044609F0DCFF082826D1621EE01D1F4997
:10B7880012F8013F09681944497801F003010229B8
:10B7980008BF203B82421370F1D1254604F1080707
:10B7A80015F8016B1648314609F0B3FF20B1284659
:10B7B800314609F0AEFF10B1FDF724FE1CE0BD4292
:10B7C800EED12046FDF71AF80E4804F0B9FC002324
:10B7D8000D4A1A4404A992F88A210A440849595C76
:10B7E80002F80C1C0133082BF2D1002307488DF80E
:10B7F8000C3001A9FFF793FB05B0F0BD180100203C
:10B80800329E01088FA0010844130020C9A901082D
:10B81800234B244C1D68206880B5FEF7B5F82846F0
:10B82800FEF7B2F8206841798B0704D4036841F029
:10B8380002015B6998471C4B4FF488521A854FF4F4
:10B8480088421A85206802F092FFA0B1164E4FF484
:10B858008853B361134B186802F086FF0746FCF75C
:10B868000FFA08B103F0B0FA2846394602F082FF11
:10B878004FF488533385284602F079FF0028E1D039
:10B88800094ED4F800804FF48847B761284602F083
:10B898006BFF0146404602F06DFF3785D2E700BFD7
:10B8A80060290020EC1F0020001000482DE9F04717
:10B8B800054609F03CFF314E0446D6F8088090B999
:10B8C8002F4804F03DFC2F4B53F8241049B10123B5
:10B8D800A34013EA080F02D02B48FFF720FB0134DE
:10B8E800F1E72A4822E028462949224609F028FF9C
:10B8F80058B92848284C04F023FC54F8041F0029A0
:10B90800EFD02148FFF70BFBF7E72B782D2B03BF70
:10B91800013504F1FF344FF0010A4FF0000A4FF0EF
:10B928000009184B53F8297027B91C48BDE8F0479F
:10B9380004F006BC28463946224609F001FFC8B97A
:10B94800012000FA09F0830501D51548EEE7BAF1A0
:10B95800000F03D0FFF738FC124803E040EA080064
:10B96800B060114804F0ECFB39461048BDE8F047D8
:10B97800FFF7D5BA09F10109D3E700BF4413002046
:10B9880095A00108F08401089FA0010887AA010872
:10B99800A3A00108A8A00108EC840108A39F01083E
:10B9A800B4A00108C2A00108CBA00108C8A90108D9
:10B9B80010B5084804F0C4FB074B00241C715C63F5
:10B9C800064B1C7003F05AF804F09EFD044B1C60F3
:10B9D80010BD00BFD3A00108EC1F0020FE2D0020E1
:10B9E8006029002070B5064600240B4BE518AA888C
:10B9F80016420AD0E1580948FFF791FA2846002173
:10BA080004F02BFB064804F09BFB143440F6BC43BF
:10BA18009C42EAD170BD00BF248C0108FFA0010838
:10BA280087AA0108F0B504788BB005460CB100244C
:10BA380036E04B4B19680E2303FB041101F58C709B
:10BA4800B1F91D51B1F91921B1F91B31009591F8DE
:10BA58002051019591F82151029590F90700039022
:10BA680001F590713F4891F9021004912146013483
:10BA7800FFF755FA082CDCD170E02D2B14D1072CD8
:10BA88001BDC284609F0AAFE0AAB661C03EB44043B
:10BA980024F8100C15F8013F303B092BFAD934462D
:10BAA8002B78002BE9D104E0A3F13002092A09D848
:10BAB800E5E7082CBDF8182009D00BB0BDE8F04028
:10BAC800FDF7A0BC202BF8D101352646E7E7072A69
:10BAD800F3D8BDF81A00224BA0F2EE2189B240F249
:10BAE800DC55A9421B68E8D8BDF81C10A1F2EE2469
:10BAF800A4B2AC42E1D8BDF81E6004B237B2A74286
:10BB0800DBDB0DB2AF42D8DCA542D6DBBDF8247032
:10BB180007F16404A4B2C82CCFD8BDF826E00FFA08
:10BB28008EF4112CC9DCBDF82050B42DC5D8BDF851
:10BB38002240B42CC1D812B24FF00E0C0CFB0233C9
:10BB4800A3F81901A3F81B11A3F81D6183F820516C
:10BB580083F8214183F81F7183F822E10BB0F0BD0F
:10BB68009812002009A10108F0B504468FB02046BC
:10BB780009F0DDFDC5B225BBAC48AD4C04F0E0FAD8
:10BB880094F8D61009B9AB4854E049B294F8D420D7
:10BB980094F8D530009194F8D710019194F9D81001
:10BBA800029194F9D910039194F8DA100491A248FB
:10BBB80029460135FFF7B3F9102D04F10704DFD149
:10BBC800E1E720469D49052209F0BAFD0546B8B9C6
:10BBD80029469B48702209F066FD9A4B1968284649
:10BBE8000E2303FB001301300022082883F82321C9
:10BBF80083F8242183F8252183F82621F0D113E145
:10BC080020469149042209F09BFD05462046002D57
:10BC18004AD1202109F07DFD002800F00581461C4D
:10BC2800304609F084FD2C460746884B53F82450CB
:10BC38002DB987480FB0BDE8F040FFF770B930461E
:10BC48002946FAB209F07CFD01340028EDD1784A82
:10BC580002F170011646002382F8DA3082F8D630F5
:10BC680082F8D53082F8D43007328A42F3D1794944
:10BC780001EBC40191F80822934210DAD1F80C7252
:10BC8800C3EBC302B0183A4400F1D4011768C0F8F6
:10BC9800D4709088888092798A710133E7E72946C1
:10BCA8006D48FFF73CF990E06C49072209F048FD20
:10BCB80005462046002D4AD1202109F02AFD0646D6
:10BCC80009F035FDC4B274BB6548FFF728F9214671
:10BCD80064480134FFF723F90E2CF8D15548FFF7D3
:10BCE8001EF9002460482146FFF719F90025554A36
:10BCF8005E4811680E2202FB04120123D2F82321A8
:10BD08005B49AB4013425B4B05F1010508BF19467F
:10BD1800FFF705F90E2DEAD146480134FFF7FFF881
:10BD2800082CDFD180E03046534909F05BFD2C46F2
:10BD380000284CD0022C4FD009F050FD06AB4E49DC
:10BD480043F82400002009F04DFD0134F0E74A498A
:10BD580009F048FD002460B1082C38D009F03EFDF8
:10BD680006AB454943F82400002009F03BFD0134A7
:10BD7800F1E7082C2BD1069B0F2B28D8DDF81CE007
:10BD8800BEF1070F23D8089F0D2F20D8099E06F172
:10BD98006402C82A1BD80A9DFF2D18D80B9864285E
:10BDA80015D80C99642912D8884210DA0D9C032CF6
:10BDB8000DD8324AC3EBC303134483F804E05F7120
:10BDC8009E71DD71187259729C722D4CCFE60FB0BE
:10BDD800BDE8F040FDF716BB069B072B20D8079956
:10BDE8000D291DD80278722A0DD06E2A18D1154A4D
:10BDF80012680E2000FB032301228A40D3F8231186
:10BE080021EA020209E00F4A12680E2000FB032310
:10BE180001228A40D3F823110A43C3F8232101E001
:10BE2800FDF7F0FA0D4CA2E60FB0F0BD31A1010804
:10BE38004413002087AA01085CA10108739F010828
:10BE480018140020981200209E9F0108E09801080D
:10BE5800A39F010840830108B29F010829A1010896
:10BE68008DA0010878A10108E1A901087DA10108B8
:10BE7800E8AD0108A2AE010881A101081414002050
:10BE8800D79C01082DE9F743047805468CB9324D53
:10BE980095F8A312B5F8A02295F8A2322F48009180
:10BEA80021460134FFF73BF8102C05F10405EFD1CA
:10BEB8004EE009F093FC0F28044636DC2846202182
:10BEC80009F027FC264EE4B2D6F83880451CA400B9
:10BED8000027284609F082FC5FFA87F9B9F1010FBB
:10BEE80083B208D0B9F1020F0BD0B3F5B47F24D2D6
:10BEF800B26B13530AE0FF2B1FD8B36B234498701F
:10BF080004E0FF2B19D8B36B2344D87028462C21A2
:10BF180009F0FFFB054608B1013502E0B9F1020F4F
:10BF28000BD10137032FD4D112E00E4800210F2284
:10BF380003B0BDE8F043FDF7E2B908EB04000021C7
:10BF4800042209F0B0FB03B0BDE8F043FDF75ABA8C
:10BF580003B0BDE8F08300BF4413002083A10108AB
:10BF6800EC1F00204C9F01082DE9F04304788FB0A6
:10BF78000546002C59D17C4B0021142209A807AE94
:10BF8800D3F83C8009F08FFB07223046002109F0E6
:10BF98008AFB05A80023A700059308EB0705838003
:10BFA8001A467249B5F802E031F813C01CEA0E0FC0
:10BFB8000AD00DF1380C0E3102F1010E6244595CC1
:10BFC80002F81C1C5FFA8EF20133072BE9D100211D
:10BFD8000B46674AB5F802E011F802C01CEA0E0FDA
:10BFE8000AD00DF1380C063203F1010E63448A5C65
:10BFF80003F8242C5FFA8EF301310629E9D118F8E9
:10C0080007305C498DE841006A78029209A81A094C
:10C0180003F00F0305F0E6F82146574809AA013452
:10C02800FEF77DFF202CA6D19BE009F0D7FB1F2847
:10C03800044600F3898028462021E4B209F069FB10
:10C048001F2C02D9FDF7DEF98BE0474BDB6B03EBC6
:10C058008404451C00212046042209F024FB002703
:10C06800464B09AE304600210A2217F803905FFAC2
:10C0780087F809F018FB002315F8012B32B10A2BB9
:10C0880004D04A4502D0F2540133F5E74A4561D15C
:10C0980008F1FF33032B09D8DFE803F0100502424B
:10C0A8000DF1230037E00DF123011FE0304609F0C0
:10C0B80095FB2378C0B243EA001006E0304609F049
:10C0C8008DFB237800F00F001843207034E0013313
:10C0D800062B0BD02A4800F2F3269E5D9642F6D135
:10C0E800034493F8ED2263881343638011F8012F0A
:10C0F80012B30023EEE70133072B0CD0204A02F2DB
:10C10800E6269E5D8E42F6D102EB4303B3F8D822B1
:10C1180063881343638010F8011F69B10023EDE7BA
:10C12800304609F05BFB0F2804DC304609F056FB6B
:10C13800607001E0002363700137052F90D101245E
:10C1480002F0E8FD6CB97DE70E4800211F22FDF7DB
:10C15800D6F806E020460021042209F0A4FA0024BB
:10C16800EEE70FB0BDE8F083EC1F00201886010849
:10C178002D86010897A10108A6A1010839860108A2
:10C18800408301084C9F01082DE9F0412DED048BF7
:10C19800B1498AB0044609F08FFAB0490028204610
:10C1A8000CBF0126072609F087FAAD49002820466A
:10C1B80008BF022609F080FA002808BF0426F10704
:10C1C80040F1EF80A748A84C03F0BAFF002003F025
:10C1D800C3FDA64803F0B4FFA54803F0B1FF637997
:10C1E800A44AA548013B254652F82310FEF797FEBE
:10C1F800A248FEF794FE4FF00008274695ED058A01
:10C20800B5EE408AF1EE10FA04D19D48FEF787FE9C
:10C21800002570E09B48D5ED069A95ED079AD5ED77
:10C22800088A4146FEF77BFEB5EEC08AF1EE10FAA9
:10C2380002D5202003F07CFFB0EE480A06A8FEF7DE
:10C2480003FD01469048FEF76AFEF5EEC09AF1EE4E
:10C2580010FA02D5202003F06BFFB0EE690A06A899
:10C26800FEF7F2FC01468848FEF759FEB5EEC09A83
:10C27800F1EE10FA02D5202003F05AFFB0EE490A79
:10C2880006A8FEF7E1FC01467F48FEF748FEF5EEFA
:10C29800C08AF1EE10FA02D5202003F049FFB0EE73
:10C2A800680A06A8FEF7D0FC08F10108014677489D
:10C2B800FEF735FEB8F10C0F05F110059ED1A4E785
:10C2C80049B294F8D42094F8D530009194F8D71056
:10C2D800019194F9D810029194F9D910039194F826
:10C2E800DA1004916A4829460135FEF718FE102D28
:10C2F80004F1070403D094F8D6100029E0D165486A
:10C30800654C03F01DFFD7F8088054F8041F19B1D5
:10C318006248FEF704FEF8E70D46614B53F82540E6
:10C3280054B10123AB4013EA080F03D05D482146FE
:10C33800FEF7F5FD0135F0E75B4803F001FF214604
:10C348007B180AAA93F88A311344584A8A5C03F87E
:10C35800102C01310829F3D1002306A954488DF87F
:10C368002030FEF7DCFD534803F0EAFE5248FDF7A3
:10C3780089FC524803F0E4FE4F48FFF7F5FD5048AA
:10C3880003F0DEFE4C48FFF77DFD4E48FEF7C7FD83
:10C398004020FFF727FB4C4803F0D2FE4648FDF744
:10C3A8005BFAB20739D5494803F0CAFE484803F09A
:10C3B800C7FE414803F010FD464803F0C1FE3E4861
:10C3C800FCF7AAFF444803F0BBFE3B48FDF796F98B
:10C3D8004248FEF7A4FD3848FDF71AF8404803F034
:10C3E800AFFE3548FFF71EFB00270E257D430024CE
:10C3F8003C4A126C2A440123D2F80A20A340134273
:10C408001ED101340E2CF3D10137082FEDD12D4860
:10C41800FEF785FD8020FFF7E5FA730716D5324849
:10C4280003F08EFE314803F08BFE234803F0AEFC88
:10C438002448FEF774FD4FF48070FFF7D3FA05E047
:10C44800394622462A48FEF76AFDDAE70AB0BDEC0B
:10C45800048BBDE8F08100BFB2A10108C2A50108A4
:10C46800B9A10108BFA1010844130020CDA101080A
:10C47800DFA10108E0980108EBA10108F6A1010875
:10C4880003A2010810A201088CA00108C9A901088B
:10C4980028A2010818A20108EC84010847A2010893
:10C4A800F084010855A2010862A20108329E010821
:10C4B8006EA2010877A20108D79C010886A201088C
:10C4C80092A2010887AA0108A0A20108ADA201084A
:10C4D800C0A20108CEA20108D8A20108E7A201085B
:10C4E800F5A20108EC1F002001A3010812A301080E
:10C4F80024A30108026D036B70B50446D5699BB986
:10C50800A90611D5C36A1BB1908C80B298470BE07D
:10C51800E169928C40694E1CD2B2E6614254E169ED
:10C52800E268914228BFE361616BA1B92A0612D57E
:10C53800636AA26A9A42236D09D0501CA669A06258
:10C54800B25C1A852369984205D3A16203E01A6890
:10C5580022F080021A602B0742BF236D08221A625C
:10C5680070BD026BC168034610B5406942B11A6CD0
:10C578008C1A013A005D08BF0A46C0B21A6410BDA1
:10C588001A6A805C01328A4228BF0022C0B21A624D
:10C5980010BD436B13B190F844007047836A406A3A
:10C5A8001B1A584258417047036B13B15B68016C02
:10C5B80001E0C369016A8B423CBFC2689B18581AE4
:10C5C800C0B27047836A8169426B1944D160416A7D
:10C5D80099429DBF0169CB1A5360CB1A96BF0023BD
:10C5E800536083624FF0000380F84430136888BFBB
:10C5F800816243F0010313607047436A8269D15432
:10C60800436A02690133934228BF00234362436BA4
:10C618001BB11B68DB0705D4D4E7026D136843F030
:10C628008003136070474171F8F756B98160F8F7D5
:10C6380053B92DE9F0410369C76805460E461F4006
:10C64800002F35D0B7FA87F24FF00043D340DB43D1
:10C658002B611F40A2F11B03042BF1D8DFE803F084
:10C66800221F1C190300746A24B1013C0023A4B2E0
:10C67800736201E0EC6AA4B2D6F82080B8F1000F2A
:10C68800DED0D8F80030404621469847D8F80480D4
:10C69800F4E73068696B07E07068A96B04E0B0687C
:10C6A800E96B01E0F068296C036889B29847C7E72D
:10C6B800BDE8F08101480249BBE700BF0004004023
:10C6C800AC2600204FF080400049B2E784260020C5
:10C6D80010B5054C05482146FFF7ABFF04F1F00102
:10C6E8000348BDE81040A4E75C260020002C014068
:10C6F80000440140014802499BE700BF002C01406B
:10C708005C260020224B10B5224C5A43224BB3FB27
:10C71800F2F203880139013AA04289B292B29BB27F
:10C728000ED004F50064A0420AD0B0F1804F07D0C3
:10C73800A4F59834A04203D004F58064A04202D145
:10C7480023F070039BB2154CA04206D004F5806418
:10C75800A0421CBF23F440739BB203800D4BC162FF
:10C76800984202850FD003F5006398420BD003F579
:10C778004063984207D003F58063984203D003F5DD
:10C788008063984201D1002303860123436110BDD1
:10C7980040420F00002C014000A24A040010004053
:10C7A800164B800A984226D00AD84A3B984218D09D
:10C7B8000133984217D0B0F5801F1AD10120704775
:10C7C8000F4B984211D004D8033B984211D1042052
:10C7D80070470C4B98420AD00133984209D1072080
:10C7E80070470220704703207047052070470620D5
:10C7F8007047FE2070470020704700BF4B001000B4
:10C808005000100051001000F8B504680646204694
:10C818000F461546FFF7C4FF07284BD8B27A910890
:10C8280047B902238B40D4F80CE0DB439BB203EA00
:10C838000E03E3600A23204A03FB001342F8237027
:10C84800043342F8235015463FB1B17AE2688908AB
:10C8580002238B409BB21343E360282202FB005261
:10C868002032EFF31286502383F3128803B203EBCE
:10C878008303DB0003F10C011C3329442B4451F8DA
:10C88800047F17B117600A6804329942F7D1002370
:10C898001360F3B283F31188282303FB0050036A63
:10C8A8001BB1E36843F0010303E0E2684FF6FE734F
:10C8B8001340E360F8BD00BF5C260020004819E67D
:10C8C80030200020004815E6842000200D4B0E483B
:10C8D8004FF400525A600D4A11684FF6FE730B4030
:10C8E8001360D0F8882011684FF6FE730B40136070
:10C8F800826FC36F9A4201D0543063E6012380F8F7
:10C908009830704700000240302000204400024068
:10C918002DE9F0471E46A54B8CB0984289469046B3
:10C928009DF8507040F08B80A14BA24A5A6503F1E4
:10C93800A8029A6603F5D472DA664FF480721A6612
:10C948005A669D4AC3F88420143AC3F88820A2F591
:10C958004842203AC3F8A0200432C3F89C20C3F808
:10C968005C80C3F8A400954B9A6942F480429A61AE
:10C978005A6942F001025A6102238DF808300323F4
:10C9880017F0010A8DF809304FF000038DF80A30CE
:10C9980014BF022301233A078DF80B3019D54FF045
:10C9A80090444FF4007501958AF001038DF80A3020
:10C9B800636A23F0F0036362636A43F0700363629F
:10C9C800204601A9FCF77EFBBAF1000F27D1A5612B
:10C9D80025E0B30710D50CA94FF4007341F82C3D9E
:10C9E8004FF09040436A23F0F0034362436A43F0F8
:10C9F80070034362FCF766FBF50710D50CA94FF4EA
:10CA0800806341F82C3D4FF09040436A23F47063F3
:10CA18004362436A43F4E0634362FCF753FB0E232B
:10CA28008DF800300022012368468DF801308DF81A
:10CA380002208DF80330624C04F076F974E0614B03
:10CA4800984240F003815A4B5A4A1A604FF4807258
:10CA5800DA601A6103F52A725A6103F56A729A61FB
:10CA6800564AC3F808801865D36943F40033D36184
:10CA780002238DF80830032317F0010A8DF80930D6
:10CA88004FF000038DF80A3014BF022301233C073E
:10CA98008DF80B3017D54C4C202501958AF00103F1
:10CAA8008DF80A30236A23F470032362236A43F45F
:10CAB800E0032362204601A9FCF704FBBAF1000F4A
:10CAC80023D1A56121E0B0070ED50CA9202341F898
:10CAD8002C3D3D48036A23F470030362036A43F460
:10CAE800E0030362FCF7EEFAF1070ED50CA9402328
:10CAF80041F82C3D3448036A23F070630362036AEB
:10CB080043F0E0630362FCF7DDFA26238DF800307A
:10CB18000022012368468DF801308DF802208DF837
:10CB2800033004F001F9224CC4F82C9000250123AD
:10CB380084F844302562E561A56265626671C4F8CF
:10CB48000880A7712046F7F7C7FEF20745D5236B83
:10CB5800002B3BD001A8FCF75DF8E36C01934FF480
:10CB680080530A9380230693E368ADF8103020239E
:10CB78000993206B636902930B95059507950895B2
:10CB88000395FCF772F801A9206BFCF750F8236BAA
:10CB9800216D1A6842F001021A608A6842F0400268
:10CBA8008A605B689BB2236417E000BF00380140CD
:10CBB80030200020FC860108580002400010024086
:10CBC8008420002000440040000C0048236D2022EF
:10CBD8001A621A6842F020021A60B3072FD5636BF5
:10CBE80043B301A8FCF716F8A36C01934FF48053E4
:10CBF8000A93802306932369ADF81030002510238B
:10CC0800606B03930B950595079508950995FCF7B7
:10CC18002CF8606B01A9FCF70AF8636B1A6842F0FC
:10CC280002021A60226D5D605D60936843F08003C4
:10CC3800936004E0226D136843F080031360226D53
:10CC4800136843F001031360204600E000200CB095
:10CC5800BDE8F0872DE9F74FA74C01F091FC266855
:10CC68006568A768861BF643451BC71BED43FF4352
:10CC7800F60F8046ED0FFF0F2EB93FB9002D00F0DB
:10CC88008682B9462CE04FF0000929E0B14627E03A
:10CC980003EB8A0BBBF802301A050ED413F4805F3D
:10CCA8001DBF964A9BF801101268954A954B14BF10
:10CCB80052F82120126843F82A20BBF80230D80520
:10CCC80016D499050AD5904B1B7813F0040F0CBFA6
:10CCD8008E4A8F4A8B4B126843F82A2009F10109C2
:10CCE800207B8C495FFA89FA82450B68D0D326E00D
:10CCF800894A5046594601F09DFF884B1B885A06C1
:10CD080003D550465946864A16E0580703D550467B
:10CD18005946844A10E0190703D550465946824AB5
:10CD28000AE09A0703D550465946804A04E0DB07D3
:10CD3800D4D57F4A5046594601F07CFFCEE7DFF84C
:10CD480008E20093BEF906307822A3F57A735343BC
:10CD58004FF47A7293FBF2F303F22B130193002240
:10CD6800F3465FFA82FE864517D2009B03EB820EDC
:10CD7800BEF802E01EF4806F0DD0DFF88891019BA9
:10CD880039F822E040F2671A9E449EFBFAFC0AFB3F
:10CD98001CEE29F822E00132E3E74DB308F5C3336E
:10CDA800A0336360637B544A13BB9373614B1B6866
:10CDB80013F0020F0AD0DFF894E19EF800E0BEF10C
:10CDC800000F03D04FF0010E82F80EE0DA0506D509
:10CDD800594BDB781BB1A37B43F00203A3734A4B87
:10CDE8001B7813F0050F02BFA37B43F00403A37362
:10CDF80094F80EE0BEF1000F03D13F4B5B7B002B94
:10CE08004FD094F80DC01CF0010FACF10C031DD1EC
:10CE1800BCF1030F07D8DFF8E8903C4A1EF0040F76
:10CE280008BF4A4600E0364AACF1040CBCF1070FD3
:10CE380005D8DFF81CC11EF0010F18BF6246DBB22F
:10CE4800032B0ED81EF0020F3C4B06E0DBB2032B7F
:10CE580006D82F4B2A4A1EF0020F18BF1A4600E0C8
:10CE6800274A4FF0000C5FFA8CF383420DD20B680F
:10CE780003EB8C035B881B0642BF224BD2F8009061
:10CE880043F82C900CF1010CEDE785B1BEF1000FD1
:10CE980008D0637B184A0133DBB2142B06D1002378
:10CEA80004E025B1637B002BF3D100E05373002E1F
:10CEB80052D0234AB2F90250B2F90020002DB8BF6F
:10CEC8006D42002A4FF03203B8BF524295FBF3F58A
:10CED80092FBF3F2EDB2D3B2AB4238BF2B46194AFC
:10CEE80013B192FBF3F300E0134643442360E37B62
:10CEF800014A7BBB01232EE0D824002024200020F7
:10CF0800A49B0108FA0E0020FB2D00206C9A010852
:10CF18005C9A01082820002014870108F41B0020CF
:10CF28001A87010820870108268701082C8701082D
:10CF38003287010898290020602D0020749A010882
:10CF48003C130020400D0300802C00207C1B002097
:10CF58007C9A01080023D3738E4D8F4B2D78E27B8A
:10CF6800ADB9002F00F00E818C4B267B1A788C4BC4
:10CF78008C4D93F800C08C4BD3F800E00B6802F09E
:10CF880004020021D2B203EB86060F46B5E01AB9B7
:10CF9800864A1A61002508E0854AFAE70A68AB0064
:10CFA800D6187688760604D40135EBB28342F5D3D9
:10CFB800D7E7804EB6F90060192E25DD12F803E098
:10CFC80094F814C026690EF00F09E1450CDCDFF86F
:10CFD800C8C19CF815C0BCEB1E1FDEBFDFF8D8E146
:10CFE800D6F800C043F80EC012F803E094F816C053
:10CFF8000EF00F09E14533DBDFF89CC19CF815C042
:10D00800BCEB1E1F2CDC26E0193629DA12F803E0E7
:10D0180094F814C026690EF00F09E1450CDCDFF81E
:10D0280078C19CF817C0BCEB1E1FA2BFDFF888E1CF
:10D03800D6F800C043F80EC012F803E094F816C002
:10D048000EF00F09E1450BDBDFF84CC19CF817C067
:10D05800BCEB1E1F04DBD6F800E0574E43F806E091
:10D06800544EB6F90260192E1BDD12F803C094F86D
:10D0780014E026690CF00F09F1450CDCDFF8189173
:10D0880099F81590B9EB1C1FDEBFDFF82CC1D6F854
:10D09800009043F80C90D25C02F00F0CF4451EDDB2
:10D0A80082E7193680DA12F803C094F816E0266988
:10D0B8000CF00F09F1450CDBDFF8DC9099F81590BE
:10D0C800B9EB1C1FDEBFDFF8F0C0D6F8009043F8BC
:10D0D8000C90D25C02F00F0CF445FFF665AF94F8A3
:10D0E80017E0BEEB121FA2BF334A36689E505BE7BB
:10D0F8005888000504D404330435B342F8D122E03B
:10D108004AB101EB0C0A06209AFBF0F900FB19A0C2
:10D1180001280DDC01E057B9012793F801900EEBC7
:10D1280089003EF829A090F80290C07803E01746DD
:10D13800002081468246013125F802AC85F800902E
:10D148006870C9B2D7E7164A1378013B13F0FF039A
:10D1580008BF06231370114B1B785B0741BFBBF94F
:10D168000630A3F57A7303EBC3034FF47A7243BF17
:10D1780093FBF2F30133DBB20123104A92FBF3F382
:10D188004344A36003B0BDE8F04FF7F707BD03B011
:10D19800BDE8F08FAB0F0020D8240020FB2D002025
:10D1A800A8000020FC0E002024200020789A010806
:10D1B800A49B01083C130020FA0E0020400D030038
:10D1C8002DE9F04F2DED0A8B89B08046059390F834
:10D1D8005030049102921BB1322BA8BF322300E0D9
:10D1E800012307EE903AF8EEE7BADFEDA87AA84BEC
:10D1F8009FEDA8CA1B88C7EEABBA002B08BF012356
:10D2080007EE903AB8EEE7AAA34B03932AEE0CCAAE
:10D218001A887BEE8CBA12F0020FCCEE2BBA27D00C
:10D228009E4AB2F90030B2F9022083EAE37182EA39
:10D23800E270A1EBE371A0EBE27088420446B8BF4C
:10D248000C46B4F5E17F16DA88429FED95BA05DD04
:10D25800002AD8BF524207EE902A04E0002BD8BF1C
:10D268005B4207EE903AF8EEE77A87EE8BBA04E075
:10D278009FED8CBA01E0B7EE00BADFF858A2DFEDF7
:10D28800899ACDF804800AF1080B0AF110070AF10F
:10D298001C090024F0EE69AA834931F914307F494A
:10D2A80009EE103AB8EEC99A31F91430F5EE047A5D
:10D2B80029EE279A08EE103A039BBDEEC99A198801
:10D2C800F8EEC97A9FED799A89074FEA440627EE66
:10D2D800899AB8EEC88A00F08180754931F914300E
:10D2E80007EE903AF8EEE77AB0EE007AE8EE077AC1
:10D2F800029B5842FDEEE77A17EE901A814203DB53
:10D308008B42A8BF0B4618466A49059B715E401AB6
:10D3180033F91410084407EE900AF8EEE78A04F08F
:10D3280047FD48B16449F2EE049A88EEA90A085DFF
:10D3380003F044FD60EE298A98F81C30DFED5F6A3F
:10D348000AEE903A98F8083007EE903AF8EE677AC5
:10D35800F8EE6AAA68EEA77AB1EE047A67EEA67AC2
:10D368002AEE877AFDEEE77A17EE901AF1EE477A01
:10D37800FDEEE7AA1AEE903A994208DBFDEEC7AA3D
:10D388001AEE903A8B42A8BF0B460AEE903AD9EDB6
:10D39800007AE8EE8C7ABBEE0E7AF4EEC77AF1EEFC
:10D3A80010FAF8EEEAAA09D4B3EE0E7AF4EE477A48
:10D3B800F1EE10FAC8BFF0EE477A01E0F0EE477AD6
:10D3C800C9ED007A98F8123009EE903AF8EE699AA9
:10D3D80067EEA97ADFED3A9A67EEA99A039B198856
:10D3E800CA0779D43048305E0028B8BF4042B0F54B
:10D3F800206F02DD0020386026E0019B9FED317A26
:10D408005B7868EE077A07EE103AB8EE477A87EE4F
:10D41800877AD7ED007A37EE497AE7EE0C7A9FEDF6
:10D428002A7AF4EEC77AF1EE10FA09D49FED277A3A
:10D43800F4EE477AF1EE10FAC8BFF0EE477A01E051
:10D44800F0EE477AC7ED007A019BD7ED007ADB7AD8
:10D4580008EE903AF8EE688A8B0768EEA77ADFED57
:10D468001C8A67EEA88A3BD538EE6A8AF0EE6A7A9B
:10D47800EBEE087A78EEE98AB0EE678AF0EE697A20
:10D48800EBEE287AF0EE678A2AE000BF83F9223EA5
:10D4980050120020BD378635F41B00203C130020B5
:10D4A8000000E143000000007C120020CDCC4C407D
:10D4B800F42D002090290020388701086F12033CC2
:10D4C8000AD7A33D0000A043000040C3000040432A
:10D4D8000AD7233CF0240020F0EE698AB0EE6A8A6D
:10D4E80089499FED8A7A635C98F8511007EE903A63
:10D4F800F8EEE77A67EEC97AA7EE878A59B18448C9
:10D50800844DB0EE480A00EBC400D5ED000AFDF7E3
:10D51800E7FAB0EE408A9AED007ADBED007A7E49B0
:10D52800AAEC019A39EE477A635C7C4D87EE0C7A57
:10D53800043709F1040909EE103A37EE677AB8EEB4
:10D54800C99AEBEE877A38EE280AEBEC017A67EE97
:10D55800897A9FED739A27EE899A30EE490A08F086
:10D56800B1FABDEEC88A6F49A85318EE103AFDEE1D
:10D57800E88AB1EE499A18EE902A41F82430BDEEB7
:10D58800C99A694B694E43F8242019EE102A46F8C7
:10D598002420019A06910132019207930CB90124C3
:10D5A8007AE6049A624B9479B3F90430640028341B
:10D5B8005C43604BB3F9043000EE103ABAEECF0A80
:10D5C80008F080FA6411201A002C07EE900AB8BF00
:10D5D8006442322CF8EEE76A574A02DD0023936072
:10D5E80026E0BDEECAAA1AEE103A23F0030307EEAE
:10D5F800903AB8EEE7AADFED517A98F80D30CAEE06
:10D60800277A07EE103AB8EE477A936826EE877ABB
:10D6180067EE277AFDEEE77A17EE901A0B44484931
:10D628008B42A8BF0B4647498B42ACBF93609160C1
:10D6380093685B13B3F5807FA8BF4FF480736FF0D6
:10D64800FF029342B8BF134607EE903AF8EEE78A16
:10D65800FDEEE67A98F8032017EE903A53439B11B3
:10D6680007EE903A384B1B78032BB8EEE78A14D9AB
:10D67800B8F84E20B2F5FA7F0FD2FDEEC87A5342C1
:10D6880017EE901A994204DB914217EE903AA8BF20
:10D69800134607EE903AB8EEE78A98F8511081B130
:10D6A8004B0803D09942A8BF194600E00121194B45
:10D6B8002648D3ED000AB0EE480AFDF711FAB0EE9D
:10D6C800408A78EE287AFDEEE77ACDED017ABDF84A
:10D6D8000430AB801BB200EE103AB8EEC00A08F076
:10D6E800F1F9069BA880BDEEC88AFDEEE88A83EDB5
:10D6F800028A079BC3ED028A0023B36009B0BDEC20
:10D708000A8BBDE8F08F00BF14250020A69B443B80
:10D71800702500208825002017250020D42500200A
:10D72800F7CC9238DC250020E8250020F4250020DD
:10D738003C1300207C1200208C25002000803B45F3
:10D74800FEFFFF0F020000F0582600208025002071
:10D758002DE9F04F2DED028B87B000260493C14BC5
:10D768000391B3F90280B3F900300292B8F1000FC7
:10D77800B8BFC8F10008002BB8BF5B429845B8BFD6
:10D788009846B8F5FA7F0746A8BF4FF4FA78009094
:10D79800B2460196B1463446B34D2B88990757D007
:10D7A800B04BB24A33F8143032F91420022013FB7C
:10D7B8000022029B5B429A424FEA440103DB029B30
:10D7C8009342A8BF1346AA4A31F902B0049A32F923
:10D7D8001420CBEB030303EB020B04F0E9FA88B146
:10D7E80007EE90BAA34BB8EEE70AB2EE048A185DCA
:10D7F80080EE080A03F0E2FA20EE080AFDEEC07A8D
:10D8080017EE90BA3B7A642203FB0BF393FBF2F317
:10D818003A7F6FF0040909FB02F94B4504DB02EB80
:10D8280082099945A8BF9946934A52F824100BEBF0
:10D83800010342F210718B42A8BF0B468F498B42FD
:10D84800B8BF0B4642F82430BA7C53431B130193EC
:10D858002D8805F00303012B38D0824B884933F912
:10D8680014A0009B51F824E093F801C0854B33F9CC
:10D87800140080EAE073A3EBE073B3F5206F4FEA7E
:10D88800840616DC0AEB8A031A0192FBFCF30422D5
:10D8980090FBF2F0181A8644BEF57A5FA8BF4FF4E1
:10D8A8007A5E794B9E45ACBF41F824E041F82430BC
:10D8B80002E0002341F824308B597D2693FBF6F6CD
:10D8C800009BDB7A7343402693FBF6F6AA0711D533
:10D8D8000198C8F5FA7208FB0AF308FB06F54FF43D
:10D8E800FA7102FB093302FB005593FBF1F395FB38
:10D8F800F1F505E0EB074DBF019D354653464B4614
:10D90800604A32F91410042291FBF2F25F49615C1B
:10D918004A436FF04F0192FBF1F297F8511013440C
:10D928004FEA440B08EE103A59B1594B5948D3ED18
:10D93800000AB8EEC80A00EBC400FDF7D1F8BDEE46
:10D94800C08A504B544A3BF803003BF902302BF88D
:10D95800020001B2101D0C32CB1A50F824E0042149
:10D9680093FBF1F152F8243040F8241073440B442F
:10D9780097F8501042F824E04FEA840C00EE103A71
:10D9880079B1434A4548D2ED000ACDF814C0B8EE43
:10D99800C00A00EBC400FDF7A3F8DDF814C0BDEE23
:10D9A800C00A3F4A3F49125D3F4810EE103A5343C0
:10D9B800202293FBF2F318EE102A2A44D21A2BF8ED
:10D9C800012018EE102A4CF80020384A4CF8025072
:10D9D800374D5B424CF80530009B013300930CB97E
:10D9E8000124D9E61F4B97F80DE0B3F90440039BD7
:10D9F8009B790F335B0063435B11224C002B4FF084
:10DA08000406B4F9044094FBF6F41D4EA3EB040499
:10DA1800B8BF5B42322BD6F808C00DDC254B0EFB95
:10DA280004CE7345A8BF7346DFF890E07345ACBFDA
:10DA3800B360C6F808E001E00023B360FB785C43FC
:10DA48001D4B1B78032B4FEAA4143AD9B7F84E3074
:10DA5800B3F5FA7F35D25F42BC4231DB9C42A8BFA6
:10DA68001C462EE03C130020F41B0020F42D00205F
:10DA780090290020388701081C250020F0D8FFFFD6
:10DA88008C2500207C12002080C1FFFF1425002077
:10DA9800882500207025002024250020BC25002092
:10DAA80017250020D4250020DC250020E8250020AB
:10DAB800F4250020FEFFFF0F58260020020000F08A
:10DAC8003C46B368846043F34F33B3F5807FA8BF07
:10DAD8004FF480736FF0FF06B342B8BF3346E618C1
:10DAE800936000238E80AB6007B0BDEC028BBDE86D
:10DAF800F08F2DE9F04F2DED028B85B08346029310
:10DB0800B84B01911D88009205F00205ADB295B1A0
:10DB1800B54BB3F90250B3F90030002DB8BF6D42D0
:10DB2800002BB8BF5B429D42B8BF1D46B5F5007FCC
:10DB3800A8BF4FF40075D9460026AB4BAB4C33F861
:10DB48001610AB4B54F8267033F9163083EAE37E8F
:10DB5800AEEBE37E08B2BEF5206F4FEA460A4FEA05
:10DB680040004FEA860812DC4FF0040E93FBFEF3E8
:10DB7800C31A1F44B7F57A5FA8BF4FF47A579D4B75
:10DB88009F42ACBF44F8267044F8263002E00023D8
:10DB980044F8263054F8087099F80B3099F8014089
:10DBA800FF115F438F4B1B8844439B074FEAA7171E
:10DBB8004FEAA41456D0904B33F90A30022011FBD7
:10DBC8000031009B5B42994203DB009B8B42A8BF5C
:10DBD8000B468A493AF90110591A029B33F9163053
:10DBE800CB1808EE103A04F0E3F868B1B8EEC80AAA
:10DBF800834BB2EE048A80EE080A985D03F0DEF8E3
:10DC080020EE080ABDEEC08A7E487F4958F80030E9
:10DC180018EE102A42F2107E13447345A8BF7346CB
:10DC28008B42B8BF0B4648F800309BF808109BF8A9
:10DC38001C00514300EB8000C911C0F1000E714572
:10DC480003DB8142A8BF01468E469BF812104B4366
:10DC58001B13FF1ACEEB04046F436C4303EB6727D7
:10DC68000EEB6424624B04213AF9030090FBF1F1B6
:10DC78006648805D4143A4EBA1129BF8511008EE61
:10DC8800102A69B16248634C0393B8EEC80A00EBE6
:10DC9800C600D4ED000AFCF723FF039BBDEEC08A43
:10DCA8005D4933F80A303AF901002AF801300FFAD1
:10DCB80083FEC0EB0E0E04209EFBF0F001F1040E73
:10DCC8000C3158F80E4058F8013048F80140234408
:10DCD8009BF8501048F80E00034400EE103A59B172
:10DCE8004C4B4E48D3ED000AB8EEC00A00EBC60014
:10DCF800FCF7F6FEBDEEC00A49494A48895D4A4C20
:10DD080010EE103A18EE102A4B435B11D119C91ABC
:10DD18002AF8001048F804204449454A48F8017098
:10DD28005B4248F8023009F101090EB9012604E7FF
:10DD38002D4B2E4EB3F90450019BD6F808E09B7981
:10DD48000F335B006B435B11294D002BB5F9045071
:10DD58004FF0040795FBF7F7A3EB0707B8BF5B4243
:10DD6800322B9BF80D500BDC324B05FB07E5AB4221
:10DD7800A8BF2B46304DAB42ACBFB360B56001E0E5
:10DD88000023B3609BF8035005FB07F32B4D2D7858
:10DD9800032D4FEAA3130CD9BBF84E50B5F5FA7F03
:10DDA80007D26F42BB4203DBAB42A8BF2B4600E061
:10DDB8003B46B568A36045F34F35B5F5807FA8BFEE
:10DDC8004FF480756FF0FF06B542B8BF35465E194F
:10DDD800002386808D60936005B0BDEC028BBDE8A2
:10DDE800F08F00BFF41B00203C1300208C2500207E
:10DDF8007C12002080C1FFFFF42D00209029002014
:10DE0800388701081C250020F0D8FFFF14250020C2
:10DE1800702500208825002038250020BC250020FA
:10DE280017250020D4250020DC250020E825002027
:10DE3800F4250020FEFFFF0F020000F05826002006
:10DE48002DE9F04F2DED028B87B000260493B24BDD
:10DE58000392B3F90270B3F900300190002FB8BFF4
:10DE68007F42002BB8BF5B429F42B8BF1F46B7F541
:10DE7800FA7F8146A8BF4FF4FA77B0460296B346B8
:10DE88003446A64D2B8899075BD0022C59D0A24B5B
:10DE9800A34A33F8143032F91420022013FB00226D
:10DEA800039B5B429A424FEA440103DB039B934284
:10DEB800A8BF13469B4A31F902A0049A32F91420EC
:10DEC800CAEB030303EB020A03F072FF88B107EE03
:10DED80090AA954BB8EEE70AB2EE048A185D80EE78
:10DEE800080A02F06BFF20EE080AFDEEC07A17EE72
:10DEF80090AA99F80830642203FB0AF393FBF2F323
:10DF080099F81C206FF0040B0BFB02FB5B4504DB4C
:10DF180002EB820B9B45A8BF9B46844A52F82430EB
:10DF280042F2107153448B42A8BF0B4680498B4282
:10DF3800B8BF0B4642F8243099F8122053431B13FC
:10DF480002932B8803F00302012A01D1022C3FD14E
:10DF58007848714A30F9140032F914807649019AE8
:10DF680051F824E0567880EAE075A5EBE075B5F540
:10DF7800206F4FEA84021EDC022C16D008EB8801C1
:10DF8800090191FBF6F6042190FBF1F0361AB6442C
:10DF9800BEF57A5F68496948A8BF4FF47A5E86453E
:10DFA800ACBF42F801E0505007E088EAE875A5EBFD
:10DFB800E875642DE2DD002088505F497D265258BF
:10DFC80092FBF6F6019AD27A7243402692FBF6F655
:10DFD8009A0713D5022C11D00298C7F5FA7307FBDC
:10DFE80006F507FB08F203FB0B224FF4FA7103FB5B
:10DFF800005392FBF1F293FBF1F508E0DB0704D53F
:10E00800022C02D0029D5A4601E035464246494B51
:10E0180033F91410042391FBF3F34949615C4B4332
:10E028006FF04F0193FBF1F399F85110D3184FEAB1
:10E03800440A08EE103AB1B1022CB8EEC80A414BB6
:10E0480008D14A0803D09142A8BF114600E0012137
:10E058003D4802E03D4800EBC400D3ED000AFCF760
:10E068003FFDBDEEC08A334B394A3AF803003AF90E
:10E0780002302AF8020001B202F108001432CB1A69
:10E0880050F824E0042193FBF1F152F8243040F8D1
:10E09800241073440B4499F8501042F824E04FEAD6
:10E0A800840C00EE103A79B1264B2A48D3ED000AC9
:10E0B800CDF814C0B8EEC00A00EBC400FCF710FDA0
:10E0C800DDF814C0BDEEC00A234A2449125D10EEE3
:10E0D800103A5343202293FBF2F318EE102A2A44F5
:10E0E800D21A2AF801201E4A18EE101A4CF802100B
:10E0F8001C4A4CF802501C4A5B424CF80230019B07
:10E1080001340133032C01937FF4BBAE07B0BDEC9F
:10E11800028BBDE8F08F00BF3C130020F41B0020E9
:10E12800F42D002090290020388701081C250020A4
:10E13800F0D8FFFF7C1200208C25002080C1FFFF53
:10E148001425002088250020802500207025002027
:10E158004C250020BC25002017250020D4250020B0
:10E16800DC250020E8250020F4250020034B4FF48F
:10E17800085208B19A6170471A8570470010004824
:10E18800034B4FF4085208B11A8570479A617047DB
:10E19800001000482DE9F04F2DED028B85B00746A1
:10E1A8000293A04B1B889807934636D5109B9E4830
:10E1B800DC89B0F900301B1B03F2F31540F2E6329C
:10E1C800954203D8002BB8BF5B4201E04FF4FA73C5
:10E1D800B0F90220121B02F2F31440F2E630844236
:10E1E80003D8002AB8BF524201E04FF4FA729342B2
:10E1F800B8BF1346C3F5FA73052293FBF2F30A225C
:10E20800643B53433A7FD2105343642293FBF2F3A7
:10E21800134423EAE373DBB200E064230093CB1CCE
:10E228000193B8460024019BDFF824A213F8016F7C
:10E238000193022C4FEA440905D1BAF904301B3680
:10E248005E43761146E079493AF8142031F9141002
:10E25800022012FB0011CBF10002914203DB594569
:10E268000A46A8BF5A467249029B31F90950551B04
:10E2780033F91420154403F09BFD88B107EE905A3A
:10E288006C4AB8EEE70AB2EE048A105D80EE080A1E
:10E2980002F094FD20EE080AFDEEC07A17EE905ABF
:10E2A800604A1288D10712D43AF909301B365E4306
:10E2B80093074FEA26160DD5BB7C5D439DF90030C8
:10E2C8005D43642395FBF3F506EB251602E03E7AE1
:10E2D80075432E11584B042533F9093093FBF5F596
:10E2E800564BE25C924698F80120751B51466A43EA
:10E2F8004A43642192FBF1F297F85110D21108EECB
:10E30800102AA9B1022CB8EEC80A08D14A0803D0CD
:10E318009142A8BF114600E00121494802E0181DBA
:10E3280000EBC400D3ED070AFCF7DAFBBDEEC08AA8
:10E33800DFF808E1434B98F80B6018880EF12003CA
:10E3480000FB05F253F82410D21206FB0216B6F5AC
:10E35800001F3D4AA8BF4FF400169642B8BF1646A4
:10E368000EF12C0243F8246052F8243042F824506D
:10E37800EB1A0EF138014FF6FF720009B2FBF0F00C
:10E3880043430EF1440051F8245050F8242040F83B
:10E3980024509B112A4441F8243097F850101A440D
:10E3A8004FEA840C761300EE102A79B10EF1500072
:10E3B800B8EEC00A00EBC400DEED070ACDF80CC0C9
:10E3C800FCF78EFBDDF80CC0BDEEC00A98F81530DE
:10E3D80010EE102A18EE101A5A43534653431A46A1
:10E3E8003144642392FBF3F3184A1B12194422F8B0
:10E3F800091018EE100A02F1080101344CF8010066
:10E4080002F114012032032C4CF801604CF8023060
:10E4180008F101087FF407AF05B0BDEC028BBDE839
:10E42800F08F00BFF41B0020802C0020F42D00206A
:10E4380090290020388701087C1200206C250020D4
:10E4480080250020501200200000E0FFD425002085
:10E458003C13002010B544780078002202FB02F338
:10E46800193B634303F6C413534340F6C4114343B3
:10E4780093FBF1F3034921F812300132072AEDD159
:10E4880010BD00BF002600200430114B33F91000E6
:10E49800B0F5617F10B506DB40F6330398420246BB
:10E4A800A8BF1A4601E04FF461720C78192340F2B4
:10E4B800833013FB0404944207DA497813FB010301
:10E4C8009342B4BF0020012010BD002010BD00BF42
:10E4D800802C002010B500F1500302788A4203D145
:10E4E8008478C278944204D304309842F5D100204D
:10E4F80010BD012010BD0B4B1B6813F4805F0A4B45
:10E50800B3F9063005D0C089421A934207DD0844A2
:10E5180000E0008A8342B4BF002001207047012038
:10E52800704700BF98290020802C00201FB5094B98
:10E538001B681B030AD58DF8040001230D2001A9CF
:10E548008DED030A8DF80530FBF738FE05B05DF850
:10E5580004FB00BF982900201FB5084B1B681B034C
:10E5680009D58DF80400029100230D2001A98DF82A
:10E578000530FBF723FE05B05DF804FB9829002061
:10E5880010B50A4A0A4B11689B6800BF126891428D
:10E59800F7D1084AD2F8A4404FF47A7000FB04F28D
:10E5A800D31AB3FBF4F300FB013010BDBC290020E3
:10E5B80010E000E06C25002038B50446FFF7E0FFC6
:10E5C8000546FFF7DDFF401BA042FAD338BD10B562
:10E5D80004462CB14FF47A70FFF7EEFF013CF8E7E0
:10E5E80010BD024A1368013313607047BC2900202C
:10E5F800024BD3F8A83003B1184770476C250020A8
:10E60800014B1B68184700BFDC2D002010B5002007
:10E61800FFF7F6FF074B00241C7003F023FA064BA4
:10E6280083F8AC40C3F8B040A3F8B440C3F8B8408E
:10E6380010BD00BF842D00206C25002010B510B936
:10E64800BDE81040E2E700230C225A430C4C111994
:10E65800125D824203D00133102BF5D110BD094B56
:10E66800D3F8B80018B14A784078824206D200221E
:10E67800C3F8B810A3F8B420C3F8B02010BD00BF89
:10E68800848A01086C25002010B540001428A8BF12
:10E6980014200023074A022199540B449918142482
:10E6A800834201F8014CF5DBFF21D1540F20BDE86E
:10E6B8001040C3E7702900202DE9F84380460B2558
:10E6C800013D3FD0224B4FF488429A614FF4885263
:10E6D8001A8508F1010632274FF005091C4CA38A58
:10E6E8009BB283F48843A382A38A9BB283F48853A2
:10E6F800A3820120FFF784FF3846FFF768FFA38A4B
:10E708009BB283F48843A382A38A9BB283F4885381
:10E718000020A382FFF774FF3846FFF758FFB9F1CE
:10E72800000F08D0B9F10109D8D14FF4FA70FFF7FA
:10E738004EFFFA27D2E7013ED0D14FF47A70FFF7A7
:10E7480046FFBDE7034B044ADA60BDE8F88300BF23
:10E758000010004800ED00E00400FA0503681B699A
:10E7680018470368DB68184703689B6818470368FD
:10E778005B68184703681B6818472DE9F84FB0F91C
:10E788000230934218BF00232DED028B18BF03708F
:10E79800057804460E469146002D40F08B8007EE22
:10E7A800902A9FED770AF8EEE77AB6EE008A27EE10
:10E7B800800ADFED747A20EE270AA04620EE080AC8
:10E7C80007F0F6F9DFED706A60EE266AB7EE006AC8
:10E7D800B0EE667AA0EE007A40F2DC536365D0EEC4
:10E7E800006A1023A4F8523037EE067A76EE866A6D
:10E7F800C6EE077A1823A4F85030274684ED046A39
:10E8080027EE807A27EE007A77EE075A84ED017AB0
:10E81800C4ED025A70EE005A84ED037AB8EE007A1D
:10E82800A5EE807A27EE877A67EEA67A84ED057AD8
:10E83800C4ED067ADFED557A98ED047A27EE277A4B
:10E84800F0EE678AB5EEC07AF1EE10FA4CBF77EEBB
:10E85800487A77EE087A013517EE900A03F020FD22
:10E86800D8ED017A67EEA87AC7E90E01F5EEC07A0D
:10E87800F1EE10FA4CBF77EEC87A77EE887A08F195
:10E88800040817EE900A03F00BFD032DC7E90801F1
:10E8980007F10807CED1A6F2DC531B042367E36710
:10E8A8006367C4F88030A367C4F884300123A4F8F0
:10E8B80002902370D4F85490B4F95280636A276A9E
:10E8C800206FE26FD4F840C0D4F88010C4F88020DC
:10E8D800C9EB060606FA08F64FEAE67B734307FB20
:10E8E8000B332667A7FB06671F44636C656F606779
:10E8F8004FEAE27B53430CFB0B3EACFB0223734411
:10E90800B61A67EB0307E36AA26AC4F884104FEAF1
:10E91800E07B434302FB0B3EA2FB00237344B61883
:10E928005F41E36CA06CB4F95020A5674FEAE17B26
:10E938004B4300FB0B33A0FB01011944636B361AF0
:10E94800206B4FEAE57B05FB03F300FB0B3367EB1A
:10E958000107A0FB050119448019794103F076FCF1
:10E9680008F1FF3201239340E067C01841EBE371DF
:10E97800424603F06BFCBDEC028B4844BDE8F88FBF
:10E988006F12833ADB0F4940F404B53F0000804B17
:10E998002DE9F8430024244B93F8EC60E0B2B04230
:10E9A8000DD203EB8003214AD3F8BC3032F81010A3
:10E9B8001BB10B2801D8DB6898470134EBE71C4BE7
:10E9C8001B685B032DD500242346E2B2B24228D24D
:10E9D800DFF8549009F1BC074FEA840857F824205F
:10E9E80055689D4215D02846FDF7DAFEEFF31283ED
:10E9F800502282F3128828216A6A01FB00900132B2
:10EA0800C0F814216A6942F001026A61DBB283F33B
:10EA1800118857F808301B6800221A6001342B4609
:10EA2800D3E7BDE8F88300BF6C2500209C120020C6
:10EA38009829002008B50E4B1B6813F4805F0D4B16
:10EA480014BFD3F83022D3F8342293F8EC1092880C
:10EA58000023D8B2884204D2074820F81320013393
:10EA6800F7E7FFF795FF3220BDE80840AFE500BFA4
:10EA7800982900206C2500209C1200200A4B1A6857
:10EA88000A4B30B502F48052D3F83042D3F83452EE
:10EA980000230AB1A18800E0A988054820F81310CE
:10EAA80001330C2BF5D130BD982900206C250020AE
:10EAB8004629002070B5124D0024214605F2392060
:10EAC800702285F8384206F0EEFD2146D5F8AC32C2
:10EAD8000B4A0B4493F9020080B102F239241E68F4
:10EAE8000E5108199C8884809B79837192F838327A
:10EAF80007310133702982F83832E7D170BD00BF81
:10EB08006C250020094B1A680E2303FB0020437A6A
:10EB1800FF2B07D0064A12789A4203D9054A32F8E1
:10EB2800130000E0808800B2704700BF2C2000204E
:10EB3800501E0020802C002038B5294C2DED048B68
:10EB480094EDAC8AB0EE480A0546FCF779FAF0EE87
:10EB5800408AB0EE480AFCF710FA94EDAD9AB0EE90
:10EB6800408AB0EE490AFCF76BFAF0EE409AB0EE34
:10EB7800490AFCF702FA95ED017AD5ED027A95ED8E
:10EB8800006A68EE676A27EE088AE7EE286A68EE88
:10EB9800000A67EE807AE6EE290AB0EE660AE7EE2A
:10EBA800A80A07F091F8DFED0F7A20EE270ADFEDCB
:10EBB8000E7A80EE270AD4EDAE7A30EE270AF2EE0E
:10EBC800047A80EE270A06F07DFFBDEC048B83B241
:10EBD8001A0444BF00F5B47083B218B238BD00BF40
:10EBE8006C2500200000E144DB0F494001380A4B46
:10EBF800042804D8DFE800F00507090B0D00074AD0
:10EC080008E0074A06E0074A04E0074A02E0074A24
:10EC180000E0074A1A6070470C01002049DE00082E
:10EC28009DE10008DD1D0108FBDA000859D700083E
:10EC3800C9D1000810B54B88DC0641BF2F4B1479A9
:10EC48001B6853F8244044BF2D4B43F820404B88A1
:10EC58009B0641BF294B54791B6853F8244044BF95
:10EC6800274B43F820404B881C070ED5254B0C78C2
:10EC78001B78B3EB141FA1BF204BD4781B6853F843
:10EC88002440A4BF1E4B43F820404B889B070ED559
:10EC98001D4B0C781B78B3EB141FDFBF174B547850
:10ECA8001B6853F82440DCBF154B43F820404B88C1
:10ECB800DC070FD5154C0B78247803F00F03A3421B
:10ECC800DFBF0E4B14781B6853F82440DCBF0C4B95
:10ECD80043F820404B885B070FD50B780C4909781F
:10ECE80003F00F038B42A1BF044B92781B6853F8C3
:10ECF8002220A4BF024B43F8202010BD242000206E
:10ED0800FA0E0020EF240020ED240020EC2400203F
:10ED1800EE240020254A264826490023F0B5156828
:10ED280003700B701C461A462E1976884EB92F5D53
:10ED38003FB9037000230A704B7007781C461A46C7
:10ED48000CE0360548BF013204F1040403F1010365
:10ED580048BFD2B2802CDBB2E6D1EAE7E0B2B842D3
:10ED68000CD215F8240006099E4200F00F00A8BF37
:10ED7800731C9042A8BF421C0134EFE78A704B70A5
:10ED8800C2F3470102F001020A444C1E0A490B482B
:10ED98000A70C3F3470203F00103134404700849DF
:10EDA800501E084A08701370F0BD00BF28200020CC
:10EDB800E424002028280020EE240020EC24002051
:10EDC800EF240020ED2400202DE9F04FC24BDA6833
:10EDD8002DED028B1A61C14A1168D960C0490B68D0
:10EDE80043F020030B60BF4B1978012990460CBFF4
:10EDF800002201221A70BC4B1A78910789B040F1A1
:10EE08003D83BA490978042940F23883B84909781A
:10EE180001F0040101F0FF0011B922F001021A709B
:10EE28001B78DB0702D408B1F9F738FBB149CA7877
:10EE3800531C052293FBF2F202EB82029A1AAE4BA4
:10EE4800CA701B78039392000023AC4CDFF8CCC245
:10EE5800DFF8D8925CF8231091FBF9F504F108006B
:10EE680004F1100640F82350A54844F8231000FB8D
:10EE7800051142F2107091FBF0F080B226F81300F1
:10EE88004FF0140E04F1140604F13C0A0EFB036E55
:10EE98005AF823605EF802704EF80210F61B3144EF
:10EEA80044344AF82310052691FBF6F109FB0511B5
:10EEB80044F82310039C012C4FEA830BE24605D14A
:10EEC8000238B0F5797F98BF4BF80C100BB90123C5
:10EED800BBE7884CD8F80030226D9FED8A7A8A4EBD
:10EEE8008A4D9B1A07EE903AF8EE677AD8F8003008
:10EEF8002365C7EE877A7C4B1B78B7EE008AF4EE61
:10EF0800C87AF1EE10FA58BFF0EE487A13F0010310
:10EF1800C4ED157A12D005AA00927D4B06AA01927B
:10EF28000CCB9AE80300F9F7B7F96421059A069B18
:10EF3800B2FBF1F293FBF1F3328000E033802B80D7
:10EF480094F858306B48002B3BD0D0ED157AC26D41
:10EF5800DAF80030C8EE276A9B1A026E022507EE1F
:10EF6800103AB8EEC77ADAF8043027EE267A9B1AF8
:10EF7800FDEEC77AB0F9662017EE901A07EE903AC0
:10EF8800644BB8EEE77AD3ED007A67EE277A67EE3E
:10EF9800A67AFDEEE77A17EE903A02FA83F3B0F913
:10EFA800642093FBF5F302FA81F29BB292FBF5F22F
:10EFB80092B2A0F86A30A0F86820A0F86630A0F8ED
:10EFC8006420012384F85830534BDAF804101B8866
:10EFD800DAF80000474D514E216603F03003E06532
:10EFE800002B00F04B8205F17403009305F17803C0
:10EFF8000193EA6E2B6FF9F74FF972682B6F9B1A22
:10F0080007EE903A434B326893ED007AEB6EF8EED8
:10F01800E77A9B1AEB67384B67EE877A1B78FDEE29
:10F02800E77A012BC5ED207A03D0022B00F0DF80B0
:10F0380024E2D5ED287A3A4BD5ED215A95ED255A9B
:10F0480095ED156A95ED264AD5ED274A35491D688F
:10F05800B1EE677ABDEEC77AFDEEE77A17EE10EAF1
:10F0680017EE90CA0020304A91ED007A52F82070CD
:10F0780007EE907AF8EEE77AA2F1140367EEA57A24
:10F0880033F81060FDEEE77A283217EE903A9B1BB2
:10F098009BB222F810301BB207EE903AF8EEE77AEE
:10F0A8003B4467EE857A4400FDEEE77ACDED037ABE
:10F0B80007EE903AF8EEE77ABDF80C8067EE847AAE
:10F0C800A7EE867AFDEEC77A17EE902A724531DBF5
:10F0D8006245A8BF62462EE028080020BC2900200F
:10F0E8002C1B0020C2120020301B0020361B0020E1
:10F0F800FB2D002028280020841000202C28002028
:10F10800806967FF00007A44AA1B0020AC1B00201E
:10F11800C4120020AC000020F41B0020381B002083
:10F1280088100020B8100020A4280020809698009D
:10F13800DB0FC940724607EE902AF8EEE77A5FEDDA
:10F14800046AC1ED007AFDEEE77A313617EE903A9F
:10F1580043449AB2AB78D1ED027A07EE103AB8EE92
:10F16800477A4B684F6027EE267AFB1A88EE077AB3
:10F17800B6B2622E06EE903AF8EEE66A37EE067AF6
:10F18800C6EE866A86EE077A76EEE76AE7EE267AB4
:10F19800C1ED047AC1ED027A0FD964EEA77ABA4EAE
:10F1A800FDEEE77A17EE903AB3F5FA6FA8BF4FF481
:10F1B800FA63B342B8BF334600E0002313441BB2DE
:10F1C80040F6B8329342A8BF1346B04A9342B8BF3C
:10F1D8001346AF4AA352AF4A142303FB002351F846
:10F1E800142B1A60002840F0498101203BE7AA4B04
:10F1F800D5F874801F68D4F878903E89DFEDA78A27
:10F208004FEA58039E4228BF1E46B5F8A8301AB2E6
:10F218009642C3BFD5ED157A9FEDA17A67EE877A3E
:10F22800B6B2C1BFFDEEE77A17EE906AF618B6B22D
:10F23800C8BFA5F8A860D4F8AC50C5EB09052846A6
:10F24800F9F76EF80028D8BF404241F29312904275
:10F25800CCBF0020012088B307EE905AB8EEE70A29
:10F2680020EE280AFBF789FE07EE908AF8EE677A07
:10F2780040F6B83320EE270AFDEEC07ACDED037ACA
:10F28800BDF80C20A4F8B02012B29A42A8BF1A46C2
:10F298007E4B9A42ACBF09EB02034B4448F6A042AE
:10F2A800934203DDA3F50C43A03B04E0002BBCBF55
:10F2B80003F50C43A033C4F8B43001E0C4F8B490AB
:10F2C800D4F8B450C5F50C53283307EE903AF8EE4D
:10F2D800E77A67EEA88AB0EE680AFBF7B1FE8DED13
:10F2E800070AB0EE680AFBF748FED4ED317AD4ED90
:10F2F8002E4AD4ED155A94ED2F4A94ED305A6549AB
:10F308008DED060AB1EE677ABDEEC77AFDEEE77AB3
:10F318000DF1180E17EE10AA17EE90BA0020614AE8
:10F32800FEEC016A32F91030DFF88C9107EE903A62
:10F3380007EE106AF8EEE77AB8EEC77A3C32D6EEF6
:10F34800877A4FEA400CFDEEE77ACDED037ABDF9F6
:10F358000C30B3F57A7FA8BF4FF47A734B45B8BF2A
:10F368004B461FFA83F922F810900FFA89F207EE3C
:10F37800902AF8EEE77A27EEA47ABDEEC77A8DEDEB
:10F38800037A27EE847AD1ED007ABDF80C90E7EE87
:10F39800257AFDEEE77A17EE902A524503DB5A45A7
:10F3A800A8BF5A4600E0524607EE902AF8EEE77AE0
:10F3B8009FED3D6AC1ED007ABA7891ED027A06EECA
:10F3C800902AF8EE666A4A684B6066EE866A9A1A70
:10F3D800C8EE266A143106EE102AB8EEC66A76EE32
:10F3E800A56A86EE256AC5EEA66A36EE476AA6EED7
:10F3F800867A01ED017A01ED037A25EE077ABDEEF2
:10F40800C77A17EE103ABDEEE77A4B4417EE102A8A
:10F4180013441BB240F6B8329342A8BF13461B4AA6
:10F428009342B8BF13461A4A2CF802301F4A1423D5
:10F4380003FB0023C3ED007A08B901206FE73B798D
:10F4480023B1642395FBF3F5194B1D803B88984540
:10F458000DD9D4F8AC30A06FC01AF8F761FF80EA74
:10F46800E072A2EBE07242F210739A4206DD114B91
:10F4780001221A700E4BB4F8C8201A8009B0BDECEE
:10F48800028BBDE8F08F00BF30F8FFFF48F4FFFFA4
:10F498000C110020E010002088100020D30237391A
:10F4A8000000C84290280020DB0FC940B810002097
:10F4B800801000208410002018FCFFFFF0B5974D45
:10F4C8002B78023B87B0082B00F29581DFE813F018
:10F4D80009002E004E0063007B008D0009016E01BB
:10F4E80079018F4B8F4C1A68636864339A4240F2F3
:10F4F800828100268C4B8D4A1B789E420ADA23684B
:10F50800884FD05C30B101F02FFB3B6801330136E6
:10F518003B60EFE72168834B525C002A40F06B8127
:10F528001A604FF0FF325A60032354E125230093F9
:10F538007F4B019303F10C0202924920A3F10A02C6
:10F5480050210233FBF742F9002840F05481794BEF
:10F558001B6813F080024FF0FF31724B03D083E831
:10F568000300042337E11A6059602AE0724A022333
:10F578000021009301910291482002F10803FBF752
:10F5880025F9002840F03781664B4FF0FF321860AC
:10F598005A6005231FE107230093684B019303F189
:10F5A8000C0202924720A3F1080200210433FBF762
:10F5B8000DF9002840F01F815A4B4FF0FF321860B8
:10F5C8005A60062307E15E4A052300210093019152
:10F5D8000291532002F10803FBF7F8F8002840F0E5
:10F5E8000A81504B18600723F5E04E4C236813B985
:10F5F8006360012323604C4B1A7863681344402BE3
:10F60800A8BF4023132B636040F3F580454B1B686C
:10F618000D2B00F2E780DFE803F060070B0E1219EC
:10F6280023282D3134404B51464801F07BFA51E0F4
:10F63800454846493FE046484649474A48E0474B1F
:10F64800474893F8CE1793F8CF2741E0434B4548F6
:10F6580093F8A8270C2101FB023393F8AA172AE094
:10F668003E4B4148B3F8441125E03C4B3F48B3F8C2
:10F67800461120E03E4B3F4819691CE03E483F4B8D
:10F6880018E03F4B1B68D80404D5344B3D4893F829
:10F698007C1110E00C2323601FE0304B3A4893F8AC
:10F6A800801193F8812193F87F3101F04BFA11E032
:10F6B8003648374B198801F045FA0BE01D4B1B689B
:10F6C80019050AD5254B3348B3F88411B3F98221BB
:10F6D80001F038FA6368181A606023680133236000
:10F6E80089E02D4B1B689A0114D52C4B1B888BB9CC
:10F6F8002B4B1B6804932B4B0E201B68059304A906
:10F70800FAF75CFD284B4FF480521A8009232B70BE
:10F71800FAF7CEFDFAF734FD6DE000BFD8290020D6
:10F72800BC290020802B0020140100203C87010800
:10F73800A6870108982900205889010870890108BE
:10F74800BC89010833A7010850A70108259D0108B5
:10F7580068A70108109D01081C9D0108441300209A
:10F768007FA7010893A70108A0A70108B2A701086D
:10F77800902D0020C4A70108D7A701081600002073
:10F78800682B0020E4A70108F4A7010810A80108C5
:10F79800642B00201EA801085C120020742B002096
:10F7A800702B0020D82D0020882B0020134B1B78AD
:10F7B800002BADD0124B1B689B01A9D408232B70DA
:10F7C800A8E7104B1A68104B5B68C8339A4204D9F3
:10F7D80001F080F901232B700DE001F095F9002864
:10F7E800F6D108E001F090F928B1084B4FF48052A7
:10F7F8001A800923EFE707B0F0BD00BF6C2B00208B
:10F808005C120020BC290020802B0020882B0020BF
:10F8180082B01B4B1B4A8DF807101968106860B33B
:10F828001268052A29D1184A106810BB9DF80810DB
:10F838009DF8073043EA012314490B80144B1968DB
:10F84800144B89B20B445B001968012119601368D5
:10F858000B441360104A136823F4E04323F0400379
:10F868009BB283F0300343F4004343F080031360FA
:10F8780003E01A68521A312AD5D902B0704700BF7E
:10F88800BC290020E02D0020F428002080610040E1
:10F89800505C00400A300020045C0040014B58686E
:10F8A800C0B27047F42800200120704770477047A5
:10F8B80020B9034B1B6808221A8270470148704719
:10F8C800AC1D0020B000002020B9034B1B680822A3
:10F8D8001A82704701487047AC1D0020B000002014
:10F8E80021B901288CBF02200020704702207047F0
:10F8F80010B5094B1A68D378042B0BD8074C518ADA
:10F90800DB00234418B99B895B1A138210BD9B68DE
:10F91800581810BD002010BDAC1D0020B0000020FC
:10F92800054B1968054B4A8A18B99B8D9B1A0B829F
:10F938007047986A10447047AC1D0020B000002042
:10F94800054B1968054B4A8A18B99B8E9B1A0B827E
:10F958007047186B10447047AC1D0020B0000020A1
:10F96800074B1B681B7803F07F03212B06D100F09F
:10F97800DF00022814BF02200020704702207047D1
:10F98800AC1D0020212810B508D1114B1B681B782D
:10F9980003F07F03212B10D0022010BD2028FBD1BB
:10F9A8000B4B0C4A1B6810701B7803F07F03212B4C
:10F9B800094B18BF00230BB9EEE7084B044A12683D
:10F9C80000249361548220469847204610BD00BF0A
:10F9D800AC1D0020FF2D0020B9F80008D1F8000860
:10F9E8007047034B1A78202A04BF00221A70704708
:10F9F800FF2D0020014B04221A607047E02D0020E3
:10FA0800034B9B7A13B1034B05221A60704700BF62
:10FA1800901F0020E02D0020F7B51C4B5A681D46AA
:10FA28000AB95C6800E00124187A0021CAB2A2422F
:10FA380001F1010107D202AE2F1816443A44527A56
:10FA480006F8042CF2E75A68121B5A601A7A5D68A5
:10FA580022441A729DB903204021F9F70FF80C4A85
:10FA6800136823F4804323F070039BB283F440535C
:10FA780043F4004343F080031360044B1D72002CD1
:10FA8800CBD09DF8040003B0F0BD00BFF4280020DF
:10FA98000C5C00402DE9F843664B674E1B68DFF8A5
:10FAA800B881664A00254FF0C0099D7283F8099015
:10FAB800DD723560D8F8003023F4EC4323F070038E
:10FAC80043F400739BB2C8F80030D8F8003023F430
:10FAD800E04323F040039BB248F2800483F0100314
:10FAE8002343C8F80030336812FA83F35B004027D9
:10FAF8001A681F6033689BB203F1005303F5405343
:10FB08005B0028461A6880221A60D8F8003023F46F
:10FB1800F8731B051B0D2343C8F80030484B93F8B6
:10FB28002C10F8F7ABFFD8F80030464A464923F4C2
:10FB3800804323F070039BB283F440532343C8F8F7
:10FB48000030136823F4EC4323F070039BB2136076
:10FB5800336811FA83F35B0003201968C3F8009037
:10FB680013683A4923F4E04323F040039BB283F03F
:10FB7800200323431360136823F4804323F07003A6
:10FB880023439BB21360536823F4EC4323F07003C0
:10FB980043F4C0639BB25360336811FA83F35B008C
:10FBA80019684FF480711960536823F4804323F077
:10FBB800700323439BB25360536823F4E04323F05C
:10FBC80040039BB283F0200323435360D8F80C30E2
:10FBD8001F4A23F4EC4323F070039BB2C8F80C309F
:10FBE800336812FA83F35B0039461A684FF4887257
:10FBF8001A60F8F743FFD8F80C3023F4804323F059
:10FC080070039BB283F440532343C8F80C30D8F8F0
:10FC18000C3023F4E04323F040031C43A4B2C8F89B
:10FC28000C402846F8F79EFE0A4B01221A60BDE8F0
:10FC3800F88300BFAC1D0020505C00400430002059
:10FC480020000020045C0040083000201030002014
:10FC58001C300020E02D0020005C0040134A144BAB
:10FC680050681B68181810B5146808D01149082284
:10FC7800F7F74FFC204610490422F7F74AFC0F4BD0
:10FC88001A68002393720E4A012111600D4913600E
:10FC98004FF4E0500B6010600B480B604FF4364196
:10FCA800A0F84A101160094A136010BDB0F7FF1F91
:10FCB800ACF7FF1FEA000020FA000020AC1D00206E
:10FCC800405C0040445C0040F4280020E02D002007
:10FCD800104B93F84C2013B51C46C2B90E4B1B6849
:10FCE800ABB11A681AB10D49486902434A619A884A
:10FCF800ADF8042002228DF807209868002201A997
:10FD08008DF80620F5F728F8012384F84C3002B066
:10FD180010BD00BFF4280020080300200010024096
:10FD28000A4B10B519684FF6FB720A401A60084A68
:10FD3800927A1C46074B0AB1052200E001221A609C
:10FD480000F094FE4FF43643236010BD405C004041
:10FD5800901F0020E02D002007B5064B0093064BAE
:10FD680001930649064A074B0748FBF7D8F803B042
:10FD78005DF804FB1C9D0108259D010867A9010881
:10FD880071A90108109D010847A9010808B5037861
:10FD980033B90C4B0C481978BDE80840FBF7BFB8DD
:10FDA80005F01CFD02280CD8064B1870074B0C22D6
:10FDB80002FB0030064B02301860FBF7D1FA054809
:10FDC800E5E708BD4429002078A90108EC1A0020BD
:10FDD800BC120020D79C010808B503783BB90B4B2F
:10FDE8000B4893F8A817BDE80840FBF798B805F04A
:10FDF800F5FC022808D8054B83F8A807FBF716FA84
:10FE0800FBF7D2FA0348E8E708BD00BF4413002017
:10FE18007CA90108D79C010838B5037803BB214B9E
:10FE28001B6801330F2B07D81F490C2202FB031252
:10FE38001C4695682DBB00E01C4601340F2C01DDE3
:10FE4800002400E005D818490C2202FB041295682A
:10FE5800BDB99C42F1D11548BDE83840FBF75FB801
:10FE680005F0BCFC0F28044605D80F4A0C2303FBF9
:10FE780000239D682DB921460D48BDE83840FBF7A1
:10FE88004EB8084B1C60FEF7C1FB21462A460948BC
:10FE9800FBF745F80C235C43034B185DBDE838407D
:10FEA800FEF7CCBB04010020848A010889A9010857
:10FEB8009FA90108B7A9010873B5037813B9F9F721
:10FEC800A1FA3DE01F4901AA05F0E9FC002401461A
:10FED8002646254699B134B1012C08D1084605F0CB
:10FEE8007DFC064603E0084605F078FC0546154902
:10FEF800002001AA05F0D3FC01340146EAE70B2DE6
:10FF080002D911480C220BE0022C10D1A6F57A7305
:10FF1800B3F57A7F07D90D484FF47A714FF4FA6236
:10FF2800F9F7EDF90CE00A4B03EB45035E80084B4B
:10FF3800084803EB45032946B3F90220FAF7EFFF17
:10FF480002B070BD81A101084C9F0108E4A401081A
:10FF580044290020CEA9010838B50D4C23688342F6
:10FF6800054606D1F9F71BFD204600214C2205F075
:10FF78009AFBE36CAB4209D12846F9F710FD054816
:10FF880000214C22BDE8384005F08DBB38BD00BFCC
:10FF9800B41D0020001E0020034B1A68D379591C99
:10FFA8001344D171187A7047D41B002010B5FFF79D
:10FFB800F3FF84B2FFF7F0FF04EB002080B210BD1E
:10FFC80010B5FFF7F3FF0446FFF7F0FF04EB00401E
:10FFD80010BD064B10B5044621461868FEF7CAFB4B
:10FFE800034B1B6898796040987110BDD81B00209E
:08FFF800D41B002038B50446BB
:020000040801F1
:1000000024200D46FFF7E9FF4D20FFF7E6FF002C07
:10001000084C14BF21203E20FFF7DFFF2368002299
:1000200028469A71FFF7D9FF236893F84900BDE885
:100030003840D2E7D41B002001460020DEE710B58F
:100040000446C0B2FFF7C9FF200ABDE81040C4E76C
:1000500010B5044680B2FFF7F2FF200CBDE8104057
:10006000EDE737B582888368044610060D4641BF28
:100070002B4991F8A8174FF4CC7000FB0133D10540
:1000800044BF2849097802F03F0244BF01EB410117
:1000900003EB8103042A12D006D8012A0DD0022ACC
:1000A00032D193F9001030E0102A0AD0202A0AD069
:1000B000082A29D1B3F9001027E0197825E019881A
:1000C00023E0196821E093ED000A6846FAF7C0FDC5
:1000D00001461548FAF727FF05B3D4ED037A6846C1
:1000E000B8EEE70AFAF7B4FD01461048FAF71BFF2D
:1000F00094ED040A6846B8EEC00AFAF7A9FD014675
:100100000A48FAF710FF09E000210948FAF70BFF47
:1001100025B10848E1682269FAF705FF03B030BD50
:1001200044130020442900208CA0010885A0010868
:10013000E1A90108DDA90108024B0146D869FEF7D3
:100140001DBB00BF4429002010B5441E14F8011F38
:1001500021B1034BD869FEF711FBF7E710BD00BFD3
:1001600044290020F7B52B492B4B08782B4D1C68F0
:100170002B4B05EB80001A882A4BD0F8C0101B7857
:10018000294800914FF47A71B4FBF1F1FAF7CBFEF4
:1001900026484821FAF7C7FE254B1F680026F3B210
:1001A00005EB8302D2F8D010E9B101249C403C4217
:1001B00017D0220715D01F4AD25C0B2000FB032367
:1001C000164A1D4802EB8303D3F8F020FAF7ABFE82
:1001D000022C06D1194B93F8281011B11848FAF7E0
:1001E000A2FE0136DBE71748FFF7AEFF164B1748B4
:1001F0001A68174B9A420CBF164B174B1A88174BAD
:10020000198892B240F2D47303B0BDE8F040FAF717
:100210008ABE00BF7C1B0020BC290020848A010804
:100220001C1B002008010020E4A9010827AA0108DE
:100230002C1B00201001002037AA010844290020AF
:100240003FAA010887AA01085412002043AA010806
:1002500000540040581200205A1200205012002072
:100260002DE9F0410024804625460F4EA75941460E
:10027000384605F09FFA58B139460C48FAF753FE54
:1002800030190021FFF7EDFE0948FFF75DFF01354A
:10029000143440F6BC439C42E7D11DB90548BDE883
:1002A000F04151E7BDE8F081248C010803A1010869
:1002B00087AA0108A39F01082DE9F04F2DED028BBD
:1002C00083B0054605F037FA064620B1012818D15B
:1002D0002B782A2B15D15C48FFF736FF00245B4DA5
:1002E0005B486159FAF71FFE28193146FFF7B9FE3E
:1002F0005848FFF729FF143440F6BC439C42EED126
:100300009CE028463D2105F008FA002800F08F8087
:100310000346994613F8012D202AFAD0441C2046A2
:1003200005F060FA80462046FAF708FCC5EB09099B
:10033000B0EE408A0026DFF834A1142202FB06F456
:100340000AF5D07B54F80B70384605F0F4F90346F3
:100350001A4628463946019305F0F6F9019B002814
:100360005BD15FFA89F29A4257D10AEB0402D2EDCF
:100370006B7AF8EEE77A0BEB0405B4EEE78AF1EE60
:1003800010FA48DBD2ED6C7AF8EEE77AB4EEE78A41
:10039000F1EE10FA3FD8B2F8A431D2F8A82113F048
:1003A000200F08BF08EE108A1C0641BF2A4991F8A9
:1003B000A8174FF4CC7404FB0122D90544BF274988
:1003C000097803F03F0344BF01EB410102EB8102D6
:1003D000042B18EE100A0BD004D8013B012B0ED8C9
:1003E00010700CE0102B05D0202B06D0082B06D166
:1003F000108004E082ED008A01E082ED008A394637
:100400001748FAF790FD2846002103B0BDEC028B97
:10041000BDE8F04F25E6134803E00136A32E8AD14C
:10042000114803B0BDEC028BBDE8F04F8CE62846C6
:1004300003B0BDEC028BBDE8F04F11E703B0BDEC9B
:10044000028BBDE8F08F00BF75AA0108248C01085B
:1004500003A1010887AA01084413002044290020B1
:100460008AAA010895AA0108A39F0108848A0108A5
:1004700070B50546284605F05EF9064658B9194B91
:1004800019485A79194B03EB8203BDE87040D3F841
:10049000581EFAF748BD28461549324605F054F96A
:1004A00060B91448144CFFF74FFE54F8041F19B1FB
:1004B0001248FAF738FDF8E7114805E00024114B1F
:1004C00053F8241019B91048BDE870403CE628469E
:1004D000324605F039F901340028F0D1014B0B4DBB
:1004E0005C71C7E744130020B5AA0108848A01089B
:1004F000A3A00108C1AA0108DC9801089FA0010877
:1005000087AA0108E0980108A39F0108D79C010869
:1005100008B50748FFF718FE064BD869F9F738FA0F
:10052000FEF78CFAFAF75CFE034B044ADA6008BD6A
:10053000D4AA01084429002000ED00E00400FA05D7
:1005400008B50548FFF700FE00F038F8FAF772FE2C
:10055000BDE80840DCE700BFE0AA010808B5044890
:10056000FFF7F2FDFAF766FEBDE80840D0E700BFEE
:10057000F6AA01080F4B1A78692A17D1598840F258
:10058000D472914212D11A79BE2A0FD193F8D12791
:10059000EF2A4FF000000BD113F8012B5040064A10
:1005A0009342F9D1B0FA80F04009704700207047BB
:1005B000704700BF00F80308D4FF03082DE9F04F8F
:1005C0002DED028BEA4D002140F2D47285B0284611
:1005D00005F06DF8E74B05F538721A60E64A00231E
:1005E0001370E64A05F2AA71116069222A7003228B
:1005F0006A714FF48072AA604FF41672A5F86621F2
:10060000FA22A5F86821BC22A5F864214FF4FA72F9
:100610002021A5F86E21012285F8622185F86A1152
:1006200085F87E216E2185F88621052285F87C11CA
:1006300085F81F220A2140F2DC5285F87D11A5F8C9
:1006400098212B2140F24C4285F87F11A5F89A2180
:10065000212140F26C7285F88011A5F89C2123219C
:1006600040F2753285F88111A5F89E214FF4C871CA
:1006700040F64302A5F8A021A5F882112A462C468F
:10068000032BCCBF0121002103F1010382F8A21149
:1006900014BF1E217521122B82F8A31102F1020250
:1006A000EED14FF4FA63A4F8C831A4F8CC31A4F821
:1006B000D031A4F8D43140F27E41052340F27E5679
:1006C00084F8E231A4F84411C82340F23A71A4F846
:1006D0004C6140F2EA5601274FF47A784FF0320B22
:1006E000A4F8E631A4F846114FF4C87340F2DC5187
:1006F000A4F84E61DFF87CA2A4F8EA3140F2B456C7
:100700001E201922A4F84A11A4F85061A4F8C68149
:10071000A4F8CA81A4F8CE81A4F8D28184F8E47147
:1007200084F8E57184F8E871A4F84881A4F852B11E
:1007300084F89501039084F8E32101920291A4F8D2
:10074000543184F8E17184F8EE71A4F856B184F85C
:10075000F171F8F711F8DAF80030039827740026E1
:10076000E773A673A681D87218735520019AD870C2
:100770000F205871DA712220212298715A740E20AC
:1007800053224FF0170E1874DA7635200A224FF0F4
:10079000280983F815E083F816E098764FF02D0EBF
:1007A0005A209A740192642283F80DE018721A7725
:1007B0001E7083F8019083F80290DE7583F804B010
:1007C0009E731E76DE735E7683F8099083F814E0DC
:1007D0004FF4FA7EA3F84EE04FF03C0E83F851E060
:1007E0004FF0110E83F850E0DFF8ACE1C3F838E0C9
:1007F000C3F83CE0DFF8A4E1C3F828E04FF0780C40
:10080000DFF89CE183F80AC0C3F834E0DFF894C154
:10081000DFF894E19FED5A8AC3F82CC0C3F830C0CA
:10082000C3F848E0F7EE087ADFF880C102999F77B5
:100830004FF04B0E83F85260C3ED087AC3ED097A8E
:1008400083ED108AC3F844C083F84CE084F8AA070B
:10085000A4F8B4174120042184F8AB0784F8ACB79E
:1008600084F8AD6784F8B16784F8B26784F8AE673E
:1008700084F8AF6784F8B067A3F85860A3F85A60AB
:10088000A3F8566083F85C10152183F868103D4981
:10089000D9663D4919673D495967C3F860C083F877
:1008A000649083F8659083F878703948F7F7AAFF69
:1008B000DAF80030019A83F811614FF44871A3F817
:1008C000161183F8126183F8139183F8147183F879
:1008D000186184F8D821C82284F8D9216422A4F8A8
:1008E000DA8184F8DC61A4F8DE2119460E2202FBCD
:1008F00006326FF0170082F81901032082F81A01FE
:100900006FF02F0082F81B01072082F81C016FF0A6
:10091000230082F81D01052082F81E0101365A20AD
:1009200081F8200181F821016422FF20082E81F83E
:100930001F2181F8220101F10E01D7D1002183F896
:100940008911C821A3F88A11142183F88C11A3F806
:1009500090211E214FF4967283F88D11A3F89221F5
:100960000121282283F88E11A3F89421094B1FE05E
:10097000441300209812002044290020BC120020BB
:10098000000000009A99193FF6287C3F3D0A773F06
:10099000DCB50108041400208FC2F53C0000604063
:1009A0006666663FCDCCCC3E000040400000A040D3
:1009B00085ED058A10359D42FAD12A480021402252
:1009C00004F075FE0023284D284C59591A19043398
:1009D0000868C2F8A002382BF5D104F50870002190
:1009E000802204F064FE05F13801702204F50870DD
:1009F00004F052FEFEF792F9DAF8006000230125B8
:100A0000314604F58F604FF4CC7284F8D03784F807
:100A1000CE5784F8CF5704F03FFE04F5C26031464C
:100A20004FF4CC7204F038FE114B1B681A68C4F8FE
:100A3000B6275A68C4F8BA279A68C4F8BE271A6855
:100A4000C4F8C2275A68C4F8C6279A68C4F8CA27E7
:100A5000022384F8CC5484F8643605B0BDEC028BD4
:100A6000BDE8F08FE4150020A89901084413002088
:100A7000BC1200201549D1F8883043F47003C1F846
:100A80008830134B1A6842F001021A605868114A04
:100A900002405A601A6822F0847222F480321A608E
:100AA0001A6822F480221A605A6822F4FE025A6000
:100AB000DA6A22F00F02DA62186B074A02401A6300
:100AC00000229A604FF000638B60704700ED00E0F9
:100AD000001002400CC07FF8CCFC00FF38B5094B79
:100AE00093F8D05765B9084C2068F8F75CFF074BBE
:100AF00025601B78022B03D1BDE83840F7F7FBBD1A
:100B000038BD00BF44130020E4290020E029002064
:100B1000044B93F8D0371BB9034B1868FDF722BE7E
:100B20000020704744130020E429002038B5054612
:100B30000446204614F8011B21B1034B1868FDF749
:100B40001DFEF6E7401B38BDE42900200FB407B5B1
:100B500004AB064953F8042B01930020FAF7F6F88A
:100B600003B05DF804EB04B0704700BFDB0C010874
:100B7000024B01461868FDF701BE00BFE4290020C2
:100B8000F8B5011F06460023083051F8042F02F182
:100B900020043F2C3AD802F108040F2C06D8023268
:100BA000032A04D9002B08BF012300E0022381425D
:100BB000EBD1012B30680ED0022B1AD0736803F0F2
:100BC00003039B0000F0030043EA0010B36803F046
:100BD0000303184317E000F00F0040F04000FFF758
:100BE000C7FFB068736800F00F0040EA0310C0B29E
:100BF00009E000F03F0040F08000FFF7B9FF3079D6
:100C0000FFF7B6FF307ABDE8F840B1E706F10C0710
:100C100034463A46002552F8043D03F18001FF298D
:100C20004FEA850510D903F50041B1F5803F02D2A6
:100C300045F0010508E003F50003B3F1807F34BF00
:100C400045F0020545F00305B242E4D165F03F00EE
:100C5000C0B2FFF78DFF05F00303022B207807D009
:100C6000032B0CD0012B13D1FFF782FF60780FE02C
:100C7000FFF77EFF6078FFF77BFFA07808E0FFF7C3
:100C800077FF6078FFF774FFA078FFF771FFE078D7
:100C90000434FFF76DFFBC424FEAA505DBD1F8BD78
:100CA00010B50446C0B2FFF763FFC4F30720BDE8E8
:100CB00010405DE710B504467F2C06D964F07F0034
:100CC000C0B2FFF755FFE409F6E7E0B2BDE8104017
:100CD0004EE7430083EAE070ECE7084648E700BFD0
:100CE00040F2E9330F4A1289920704D4013B9BB2C8
:100CF000002BF7D10BE00C4A40F2E93310700949A0
:100D00000989C9070AD4013B9BB2002BF7D1074AD6
:100D1000138801339BB21380FF2070471078C0B254
:100D2000704700BF003001400C300140882900208E
:100D30000C4B0D49DA684378D243C2F30222C2F168
:100D40000402934002781B010A44DBB282F80033AC
:100D500003780122580903F01F0302FA03F341F854
:100D60002030704700ED00E000E100E073B505467B
:100D7000002100680122FBF7C9FC2A6813889BB296
:100D800043F001031380EB7A8DF804300124002630
:100D900001A88DF805408DF806608DF80740FFF733
:100DA000C7FFEB7A1B2B0BD1192301A88DF8043058
:100DB0008DF805408DF806608DF80740FFF7B8FF05
:100DC00002B070BDF0B5BE4CA3782DED028B013B97
:100DD000012B85B000F26F81E578854240F06B8190
:100DE0002379022B00F06781B64B5B5D6371A379B9
:100DF0006D00F2EE048A1BB16319B3F9083009E003
:100E00006319D4ED037AB3F90830F1EE677AC4EDD3
:100E1000037A5B4208EE103A2369A94EB8EEC88AFD
:100E20001A0388EE288A35D5D6ED037AFDEEE77AE7
:100E300028EE280A17EE903AD6ED057A8DF80A309A
:100E4000FDEEE77A17EE903A8DF80B3004F084FE51
:100E5000FCEEC07A96ED060A17EE903A20EE280ACC
:100E6000ADF8083004F078FEFCEEC07A96ED070A83
:100E700017EE903A20EE280AADF80C3004F06CFE24
:100E8000FCEEC07A0C2017EE903A02A9ADF80E30B5
:100E9000F9F798F9D4ED077A894BF5EE407AF1EE3F
:100EA00010FA60D1D3ED067AB4EEE78AF1EE10FACB
:100EB00004DDDA6883ED068A5A61E8E0F5EEC07A6F
:100EC000F1EE10FA40F3E38093F8202042B1022AB9
:100ED00000F2DD805A6B83ED078AFA329A63D6E01E
:100EE000D3ED037A38EE678AF7EE007AB4EEE78A3C
:100EF000F1EE10FAACBF01210021D3ED0A7A69B1FD
:100F00009FED717A27EE877ADFED707AB4EEE77A9B
:100F1000F1EE10FA58BFF0EE477A03E09FED6C7ADD
:100F200067EE877AC3ED0A7A2369654A1B0311D5F8
:100F30008DF808105379116B0B440B205A788DF8FB
:100F40000920DA7A8DF80A205B7D8DF80B3002A932
:100F5000F9F738F90123226B84F8203063791344C0
:100F60000022DA7291E0B4EEE78AF1EE10FA48BF9F
:100F700083ED078AA16B636B94ED067AD4ED076A63
:100F8000591AC943C90F77EE667A59B9B7EE006AA4
:100F9000F4EEC67AF1EE10FA79DDB4EEE68AF1EEFF
:100FA00010FA74DDD4ED056A454BB4EEE67AF1EE45
:100FB00010FACCBF0126002666B1D3ED097A9FED69
:100FC000427A67EE877A9FED427AC3ED097AD3EDD4
:100FD0000B7A0AE0B0EE007AF4EEC77AF1EE10FA7E
:100FE00008DDD3ED0B7A9FED387A67EE877AC3ED93
:100FF0000B7A07E0D3ED097A9FED357A67EE877AB1
:10100000C3ED097AD4ED097A206B627967EEA87A8C
:101010001044FCEEE77ACDED017A9DF80430437080
:10102000D4ED0B7A2769FCEEE77A3F03CDED017A28
:101030009DF8042042750ED546EA41018DF808104E
:101040008DF80930C37A8DF80A300B2002A98DF88B
:101050000B20F9F7B7F894F82020194B022A11D188
:10106000D3ED0A7A9FED1B7A196B67EE877A00221F
:1010700083F82020FCEEE77A5A7917EE903A0A447A
:10108000D37202E0022283F82020F7F777FAA279E0
:101090000B4B0AB1104A00E0104ADA602544D4ED47
:1010A000037AB5F9083000EE103AB8EEC00A80EEC7
:1010B000280A37EEC00A05B0BDEC028BF0BD00BFB8
:1010C00088290020809A0108EC51783F6F12833AFA
:1010D0000AD7833F00007A440000A0410000A0C16D
:1010E0002B4BF0B52B4D1E6805F110002F78F3192E
:1010F0002C46597801F00401013501F0FF0219B1C5
:101100008542F3D10020F0BD224D631B022B0ADD86
:101110001AB102EB82025200D2B215F8013B303B09
:101120001A44D2B2F1E70021AC420AD919B101EB5D
:1011300081014900C9B215F8013B303B1944C9B2DD
:10114000F2E72E2F16D101340420002325787719D9
:1011500003EB83037F785B007F079BB244BF303D86
:101160005B1900F1FF3044BF01349BB210F0FF0067
:10117000ECD100E0002308484143642000FB031346
:101180000620B3FBF0F3054800FB0230F0BD00BFC2
:1011900018010020C429002040420F0080969800CA
:1011A00030B500231A4610498C1894F83C40BCB165
:1011B0002E2C06D1013298B18C180444002584F8F5
:1011C0003C5011440A2491F83C106343A1F13004CF
:1011D000092C9CBF303B5B180E2A03D80132E2E792
:1011E000184630BD002030BD882900200EB40FB550
:1011F0000749019006AB01A8064A0393F9F7A6FD3B
:10120000019B00221A7004B05DF804EB03B0704734
:101210007DAA000897A101082DE9F04FAE490B788F
:1012200013F0010F87B003F0040200F07981002A67
:1012300040F08381A948066816F0806640F07D8101
:10124000980700F16D8143F004030B70A44BA54F88
:101250001A88A54B1A803B681B0340F11D81A34BE4
:1012600080201E70F7F746FB08B1FEF779FEA04C10
:101270002578012D40F010819E4B93F8CE1721B1B7
:1012800093F8CF270AB1914203D3012283F8CE27E6
:1012900011E096460846BEF1000F06D090FBFEFC1A
:1012A0000EFB1C0C7046E646F5E791FBF0F183F867
:1012B000CE1792FBF0F283F8CF2793F8D0271AB11C
:1012C0008C4A002182F8D017626893F8D09702EB1D
:1012D000C20241F669018A4284BF40F2E241B2FB98
:1012E000F1F285498CBFD2B204220A70B9F1000F25
:1012F0001FD18020F8F796FD8046D0B18021F8F705
:101300006BFD98F806207D4B207253F8223098F937
:101310000000DFF8DC81B3F5613F0CBF0222002240
:1013200002218DE8060080214A46F8F757FBE0606D
:1013300008B90023AFE0494608F11000142204F078
:10134000B6F908F13003C8F8243008F1A403C8F84E
:10135000283008F58C73C8F82C30694B39681B8825
:10136000A8F88C31634B93F8942193F8CE8793F8C7
:1013700086A1002A634A10685A7993F8CF37A2F100
:10138000190EC1F3C03C18BF4FF0010CDEF100078D
:1013900047EB0E07012A14BF3A4601225A4F049226
:1013A00098455A4BD7F800E01B78039301F4006985
:1013B000C0F3800BC1F34001C0F3C0002CBF4FF05D
:1013C00000084FF0010805976A1ED2B2531E132B76
:1013D0003DD8DFE803F00C0C0C0C0C0C0C0C0AAC28
:1013E000AE292B3F37121212393F049BA2E0039B18
:1013F0009342B4BF0023012328E09EF80030022B63
:101400000BD10EEB820353ED027AF5EE407AF1EE4A
:1014100010FA14BF0123002318E00EEB02035B79DE
:10142000003318BF012311E00B4683E0B9F1000F30
:1014300004D00AF1FF377B427B4100E04B4603F0CA
:10144000010377E0634675E0434673E013B101237F
:1014500093401E43142D02D80135EDB2B4E7059B2D
:10146000C4F89061186819217930FDF737F8002326
:10147000C4F89831A4F89C31A4F89E31C4F8A8317E
:10148000234BD4F8A4211B68C4F8AC3184F8940130
:10149000C4F8A021022323701D4B164A1B6892F842
:1014A000E2214FF47A7101FB02331A4A13600D4BAB
:1014B0001B681A0609D5184B1B789B0705D5174BD7
:1014C0001B78042B01D9062000E0052007B0BDE8F9
:1014D000F04FFDF7B7B800BFFB2D00205C120020D5
:1014E000341300209829002082100020551E00206F
:1014F000D82900204413002014010020207E010878
:10150000C81E00202C1B0020981200205826002006
:10151000BC29002034100020301B0020361B002086
:101520005AB9012007B0BDE8F04FFDF7B1B8034646
:1015300000E05B46002B8AD18EE707B0BDE8F08F54
:1015400010B5154A1378590725D523F004031370F5
:10155000124B1B681B0319D5114C2378A3F1080209
:10156000012A0BD8FF200021F8F72CFE0D4B1B6839
:10157000C4F8AC31FFF7CCFA0A2306E0012B05D9F9
:101580000A2B03D0FFF7AAFA012323700420BDE839
:101590001040FDF757B810BDFB2D00209829002002
:1015A000D8290020BC29002003788B4286BF024B3B
:1015B00033F81100002070478C2B002070B50022FA
:1015C0001346234914180C44247E83EA0423082478
:1015D00013F4004F4FEA430318BF83F4815304F11F
:1015E000FF3418BF83F0010314F0FF049BB2EFD166
:1015F0000132192AE5D100F1190200F11A050A4455
:101600000D44167E2A7E02EB062292B29A421ED129
:101610000F4B93F83950E2B2AA4215D2431C03EBA8
:101620004203DBB2CA1801330B44127E1B7E03EB6C
:1016300002239BB24FF4AF6253431B1303F548736D
:1016400021F814300134E6E7012381F83A3070BD07
:101650008C2B002003788B420BD9074B1A78074B51
:1016600089001944C86B02B1400800F5777080B258
:1016700070470020704700BF541E00208C2B0020B4
:1016800007299DBF034B03EB8101B1F86C000020DB
:10169000704700BF8C2B0020034B03EB4101B1F8D6
:1016A0008C00C008704700BF8C2B00200A4BDFED78
:1016B0000B7A03EB810191ED2B7AB8EE477AF6EEC7
:1016C000046AE7EE267A82B0FCEEE77ACDED017A85
:1016D000BDF8040002B070478C2B002000005C4471
:1016E000024B03EB4101B1F8F40070478C2B002052
:1016F000024B03EB4101B1F8180170478C2B00201D
:10170000024B03EB4101B1F8180170478C2B00200C
:101710000020704770B5334C0546FCF735FFD4F810
:101720003031C4F83001C31AB3F5FA5FC4F834316C
:1017300082BF002384F8383184F8393194F8383185
:101740002BB9A12D02BF274A012182F8391194F843
:101750003911244A29B1D118EDB201330D7682F83E
:10176000383194F8385194F83A31AB4239D11D4BA5
:1017700093F83B31052B02D0062B03D02CE0002040
:10178000FFF71CFF637E1E2B26D100200246C1B24C
:101790006B1E994219DA21440B7E0821DBB283EAE1
:1017A0000206F60744BF83F01803C3F3460301F1B2
:1017B000FF3154BF5B0843F0800311F0FF01C2F317
:1017C0004702ECD101301A46E1E723441B7E9A42DE
:1017D00002D10320FFF7F2FE002384F8393184F8A8
:1017E000383170BD8C2B002010B50446FCF7CCFEC0
:1017F0000F4BD3F83C21C3F83C01821A41F28831E7
:101800008A42C3F8402184BF002283F8442193F820
:101810004421074913440F2AE4B218BF013283F868
:10182000454112BF81F84421012381F8553110BD93
:101830008C2B002010B50446FCF7A6FE0F4BD3F806
:101840005821C3F85801821A41F288318A42C3F8FC
:101850005C2184BF002283F8602193F8602107494E
:101860001344142A18BF013283F8614112BF81F872
:101870006021012381F8763110BD00BF8C2B002040
:1018800038B50446FCF780FE274A2749D2F878315C
:10189000C2F87801C31AB3F57A6F84BF002382F8C7
:1018A0007C3192F87C3133B9A82C3BD181F87D3161
:1018B000A1F87E3106E0022B02D181F8804101E0DF
:1018C000242B02D8D11881F8814192F88011164D4D
:1018D00001330231DBB249008B4282F87C3118DAE5
:1018E000B5F87E31E0B283EA0020082310F4004FFF
:1018F0004FEA400018BF80F4815003F1FF3318BF56
:1019000080F0010013F0FF0380B2EFD1A2F87E0156
:1019100038BD01318B4201BF002385F87C310123A2
:1019200085F87D3138BD00BF8C2B002010B50446F2
:10193000FCF72AFE104AD2F8A83140F6AC51C31A7F
:101940008B42C4BF002382F8AC3192F8AC31D1187D
:1019500081F8AD4123B90F2C0DD10749C1F8A80179
:101960000133DBB2192B044982F8AC310CBF0123DF
:10197000002381F8C63110BD8C2B0020094B1A685A
:10198000137844F6FB7103EB431300FB0313507809
:10199000C0EB0030B3FBF0F39078B3FBF0F080B213
:1019A000704700BF181B0020124B10B5D3F8C82198
:1019B00002EB40010C7E14B1022C11D00BE0022886
:1019C00005D9032807D10C4B1B68DB0401D5D0894E
:1019D00010BD908A10BD03EB4003B3F8F40010BDB6
:1019E000487E00EB800000EB800000F2EE2080B229
:1019F00010BD00BF8C2B00209829002008B5FCF7F3
:101A0000C3FD074B022283F8D021064AC3F8CC015C
:101A10001268C3F8DC21012283F8F52108BD00BF5C
:101A20008C2B0020BC29002008B5FCF7ADFD084B2D
:101A3000022283F8D021D3F8DC2100F5B71000F59D
:101A4000587002F2DC52C3F8CC01C3F8DC2108BDA7
:101A50008C2B0020044B1B6842F201021A420CBF7F
:101A600001200020704700BF98290020114B93F8F7
:101A7000F821012A10B51C460ED008D3022A0FD136
:101A80000D4A938A9BB283F48853938208E00A4BF1
:101A90004FF488521A8503E0074B4FF488529A613D
:101AA000FCF772FD00F5F42000F59070C4F8FC011D
:101AB00010BD00BF8C2B002000100048022803D06E
:101AC000431E584258417047064B1B681B7823B190
:101AD000054B1868C0F3C0407047044B1878C0F33A
:101AE00080007047880600205C120020FB2D00203B
:101AF00010B50A4C5E280146206805D15D21FCF72F
:101B00003DFE20683E2105E05D2903D1FCF736FE4D
:101B100020683D21BDE81040FCF730BE8C2D002030
:101B200030B50028104C114AB8BF40423C2590FB0C
:101B3000F2F304FB030068430D4D90FBF2F22D68B5
:101B40002D7B25B903EB830303EB830301E0C3EB98
:101B5000031302EB83030B8004FB02024FF47A733E
:101B600092FBF3F24A8030BD806967FF809698004F
:101B7000201B002010B50446C0B2FFF7B9FFC4F324
:101B80000720BDE81040B3E7024B5E211868FCF760
:101B9000F5BD00BF8C2D002038B5064C05465E21F2
:101BA0002068FCF7EBFD20682946BDE83840FCF7CB
:101BB000E5BD00BF8C2D0020674B73B51878674DCD
:101BC000FFF77CFF2B788342044620D0C8B1644BDA
:101BD0001B68E3B193F9000002230093614B1B687B
:101BE0005B78003318BF0123019304214FF416538F
:101BF0000022F7F7F3FE5C4B186040B101232B7015
